Archive member included to satisfy reference by file (symbol)

/usr/local/bin/../lib/gcc/arm-none-eabi/8.3.1/../../../../arm-none-eabi/lib/thumb/v7e-m+fp/hard/libc_nano.a(lib_a-exit.o)
                              /usr/local/bin/../lib/gcc/arm-none-eabi/8.3.1/../../../../arm-none-eabi/lib/thumb/v7e-m+fp/hard/crt0.o (exit)
/usr/local/bin/../lib/gcc/arm-none-eabi/8.3.1/../../../../arm-none-eabi/lib/thumb/v7e-m+fp/hard/libc_nano.a(lib_a-impure.o)
                              /usr/local/bin/../lib/gcc/arm-none-eabi/8.3.1/../../../../arm-none-eabi/lib/thumb/v7e-m+fp/hard/libc_nano.a(lib_a-exit.o) (_global_impure_ptr)
/usr/local/bin/../lib/gcc/arm-none-eabi/8.3.1/../../../../arm-none-eabi/lib/thumb/v7e-m+fp/hard/libc_nano.a(lib_a-init.o)
                              /usr/local/bin/../lib/gcc/arm-none-eabi/8.3.1/../../../../arm-none-eabi/lib/thumb/v7e-m+fp/hard/crt0.o (__libc_init_array)
/usr/local/bin/../lib/gcc/arm-none-eabi/8.3.1/../../../../arm-none-eabi/lib/thumb/v7e-m+fp/hard/libc_nano.a(lib_a-memset.o)
                              /usr/local/bin/../lib/gcc/arm-none-eabi/8.3.1/../../../../arm-none-eabi/lib/thumb/v7e-m+fp/hard/crt0.o (memset)
/usr/local/bin/../lib/gcc/arm-none-eabi/8.3.1/../../../../arm-none-eabi/lib/thumb/v7e-m+fp/hard/libnosys.a(_exit.o)
                              /usr/local/bin/../lib/gcc/arm-none-eabi/8.3.1/../../../../arm-none-eabi/lib/thumb/v7e-m+fp/hard/libc_nano.a(lib_a-exit.o) (_exit)
/usr/local/bin/../lib/gcc/arm-none-eabi/8.3.1/thumb/v7e-m+fp/hard/libgcc.a(_arm_addsubdf3.o)
                              _build/nrf52832_xxaa_print.c.o (__aeabi_dsub)
/usr/local/bin/../lib/gcc/arm-none-eabi/8.3.1/thumb/v7e-m+fp/hard/libgcc.a(_arm_muldivdf3.o)
                              _build/nrf52832_xxaa_print.c.o (__aeabi_dmul)
/usr/local/bin/../lib/gcc/arm-none-eabi/8.3.1/thumb/v7e-m+fp/hard/libgcc.a(_arm_cmpdf2.o)
                              _build/nrf52832_xxaa_print.c.o (__aeabi_dcmpeq)
/usr/local/bin/../lib/gcc/arm-none-eabi/8.3.1/thumb/v7e-m+fp/hard/libgcc.a(_arm_fixdfsi.o)
                              _build/nrf52832_xxaa_print.c.o (__aeabi_d2iz)
/usr/local/bin/../lib/gcc/arm-none-eabi/8.3.1/thumb/v7e-m+fp/hard/libgcc.a(_aeabi_ldivmod.o)
                              _build/nrf52832_xxaa_bsp.c.o (__aeabi_ldivmod)
/usr/local/bin/../lib/gcc/arm-none-eabi/8.3.1/thumb/v7e-m+fp/hard/libgcc.a(_aeabi_uldivmod.o)
                              _build/nrf52832_xxaa_bsp.c.o (__aeabi_uldivmod)
/usr/local/bin/../lib/gcc/arm-none-eabi/8.3.1/thumb/v7e-m+fp/hard/libgcc.a(_udivmoddi4.o)
                              /usr/local/bin/../lib/gcc/arm-none-eabi/8.3.1/thumb/v7e-m+fp/hard/libgcc.a(_aeabi_ldivmod.o) (__udivmoddi4)
/usr/local/bin/../lib/gcc/arm-none-eabi/8.3.1/thumb/v7e-m+fp/hard/libgcc.a(_dvmd_tls.o)
                              /usr/local/bin/../lib/gcc/arm-none-eabi/8.3.1/thumb/v7e-m+fp/hard/libgcc.a(_aeabi_ldivmod.o) (__aeabi_ldiv0)
/usr/local/bin/../lib/gcc/arm-none-eabi/8.3.1/../../../../arm-none-eabi/lib/thumb/v7e-m+fp/hard/libc_nano.a(lib_a-ctype_.o)
                              _build/nrf52832_xxaa_nrf_log_backend_serial.c.o (_ctype_)
/usr/local/bin/../lib/gcc/arm-none-eabi/8.3.1/../../../../arm-none-eabi/lib/thumb/v7e-m+fp/hard/libc_nano.a(lib_a-memcmp.o)
                              _build/nrf52832_xxaa_id_manager.c.o (memcmp)
/usr/local/bin/../lib/gcc/arm-none-eabi/8.3.1/../../../../arm-none-eabi/lib/thumb/v7e-m+fp/hard/libc_nano.a(lib_a-memcpy-stub.o)
                              _build/nrf52832_xxaa_nrf_log_backend_serial.c.o (memcpy)
/usr/local/bin/../lib/gcc/arm-none-eabi/8.3.1/../../../../arm-none-eabi/lib/thumb/v7e-m+fp/hard/libc_nano.a(lib_a-snprintf.o)
                              _build/nrf52832_xxaa_nrf_log_backend_serial.c.o (snprintf)
/usr/local/bin/../lib/gcc/arm-none-eabi/8.3.1/../../../../arm-none-eabi/lib/thumb/v7e-m+fp/hard/libc_nano.a(lib_a-strcpy.o)
                              _build/nrf52832_xxaa_SEGGER_RTT.c.o (strcpy)
/usr/local/bin/../lib/gcc/arm-none-eabi/8.3.1/../../../../arm-none-eabi/lib/thumb/v7e-m+fp/hard/libc_nano.a(lib_a-strlen.o)
                              _build/nrf52832_xxaa_ble_init.c.o (strlen)
/usr/local/bin/../lib/gcc/arm-none-eabi/8.3.1/../../../../arm-none-eabi/lib/thumb/v7e-m+fp/hard/libc_nano.a(lib_a-nano-svfprintf.o)
                              /usr/local/bin/../lib/gcc/arm-none-eabi/8.3.1/../../../../arm-none-eabi/lib/thumb/v7e-m+fp/hard/libc_nano.a(lib_a-snprintf.o) (_svfprintf_r)
/usr/local/bin/../lib/gcc/arm-none-eabi/8.3.1/../../../../arm-none-eabi/lib/thumb/v7e-m+fp/hard/libc_nano.a(lib_a-nano-vfprintf_i.o)
                              /usr/local/bin/../lib/gcc/arm-none-eabi/8.3.1/../../../../arm-none-eabi/lib/thumb/v7e-m+fp/hard/libc_nano.a(lib_a-nano-svfprintf.o) (_printf_i)
/usr/local/bin/../lib/gcc/arm-none-eabi/8.3.1/../../../../arm-none-eabi/lib/thumb/v7e-m+fp/hard/libc_nano.a(lib_a-memchr.o)
                              /usr/local/bin/../lib/gcc/arm-none-eabi/8.3.1/../../../../arm-none-eabi/lib/thumb/v7e-m+fp/hard/libc_nano.a(lib_a-nano-svfprintf.o) (memchr)
/usr/local/bin/../lib/gcc/arm-none-eabi/8.3.1/../../../../arm-none-eabi/lib/thumb/v7e-m+fp/hard/libc_nano.a(lib_a-memmove.o)
                              /usr/local/bin/../lib/gcc/arm-none-eabi/8.3.1/../../../../arm-none-eabi/lib/thumb/v7e-m+fp/hard/libc_nano.a(lib_a-nano-svfprintf.o) (memmove)
/usr/local/bin/../lib/gcc/arm-none-eabi/8.3.1/../../../../arm-none-eabi/lib/thumb/v7e-m+fp/hard/libc_nano.a(lib_a-nano-freer.o)
                              /usr/local/bin/../lib/gcc/arm-none-eabi/8.3.1/../../../../arm-none-eabi/lib/thumb/v7e-m+fp/hard/libc_nano.a(lib_a-nano-svfprintf.o) (_free_r)
/usr/local/bin/../lib/gcc/arm-none-eabi/8.3.1/../../../../arm-none-eabi/lib/thumb/v7e-m+fp/hard/libc_nano.a(lib_a-nano-mallocr.o)
                              /usr/local/bin/../lib/gcc/arm-none-eabi/8.3.1/../../../../arm-none-eabi/lib/thumb/v7e-m+fp/hard/libc_nano.a(lib_a-nano-svfprintf.o) (_malloc_r)
/usr/local/bin/../lib/gcc/arm-none-eabi/8.3.1/../../../../arm-none-eabi/lib/thumb/v7e-m+fp/hard/libc_nano.a(lib_a-nano-reallocr.o)
                              /usr/local/bin/../lib/gcc/arm-none-eabi/8.3.1/../../../../arm-none-eabi/lib/thumb/v7e-m+fp/hard/libc_nano.a(lib_a-nano-svfprintf.o) (_realloc_r)
/usr/local/bin/../lib/gcc/arm-none-eabi/8.3.1/../../../../arm-none-eabi/lib/thumb/v7e-m+fp/hard/libc_nano.a(lib_a-sbrkr.o)
                              /usr/local/bin/../lib/gcc/arm-none-eabi/8.3.1/../../../../arm-none-eabi/lib/thumb/v7e-m+fp/hard/libc_nano.a(lib_a-nano-mallocr.o) (_sbrk_r)
/usr/local/bin/../lib/gcc/arm-none-eabi/8.3.1/../../../../arm-none-eabi/lib/thumb/v7e-m+fp/hard/libc_nano.a(lib_a-mlock.o)
                              /usr/local/bin/../lib/gcc/arm-none-eabi/8.3.1/../../../../arm-none-eabi/lib/thumb/v7e-m+fp/hard/libc_nano.a(lib_a-nano-freer.o) (__malloc_lock)
/usr/local/bin/../lib/gcc/arm-none-eabi/8.3.1/../../../../arm-none-eabi/lib/thumb/v7e-m+fp/hard/libc_nano.a(lib_a-nano-msizer.o)
                              /usr/local/bin/../lib/gcc/arm-none-eabi/8.3.1/../../../../arm-none-eabi/lib/thumb/v7e-m+fp/hard/libc_nano.a(lib_a-nano-reallocr.o) (_malloc_usable_size_r)
/usr/local/bin/../lib/gcc/arm-none-eabi/8.3.1/../../../../arm-none-eabi/lib/thumb/v7e-m+fp/hard/libc_nano.a(lib_a-reent.o)
                              /usr/local/bin/../lib/gcc/arm-none-eabi/8.3.1/../../../../arm-none-eabi/lib/thumb/v7e-m+fp/hard/libc_nano.a(lib_a-sbrkr.o) (errno)
/usr/local/bin/../lib/gcc/arm-none-eabi/8.3.1/../../../../arm-none-eabi/lib/thumb/v7e-m+fp/hard/libc_nano.a(lib_a-lock.o)
                              /usr/local/bin/../lib/gcc/arm-none-eabi/8.3.1/../../../../arm-none-eabi/lib/thumb/v7e-m+fp/hard/libc_nano.a(lib_a-mlock.o) (__retarget_lock_acquire_recursive)
/usr/local/bin/../lib/gcc/arm-none-eabi/8.3.1/../../../../arm-none-eabi/lib/thumb/v7e-m+fp/hard/libnosys.a(sbrk.o)
                              /usr/local/bin/../lib/gcc/arm-none-eabi/8.3.1/../../../../arm-none-eabi/lib/thumb/v7e-m+fp/hard/libc_nano.a(lib_a-sbrkr.o) (_sbrk)

Allocating common symbols
Common symbol       size              file

nrf_nvic_state      0xc               _build/nrf52832_xxaa_app_util_platform.c.o
__lock___atexit_recursive_mutex
                    0x1               /usr/local/bin/../lib/gcc/arm-none-eabi/8.3.1/../../../../arm-none-eabi/lib/thumb/v7e-m+fp/hard/libc_nano.a(lib_a-lock.o)
__lock___arc4random_mutex
                    0x1               /usr/local/bin/../lib/gcc/arm-none-eabi/8.3.1/../../../../arm-none-eabi/lib/thumb/v7e-m+fp/hard/libc_nano.a(lib_a-lock.o)
errno               0x4               /usr/local/bin/../lib/gcc/arm-none-eabi/8.3.1/../../../../arm-none-eabi/lib/thumb/v7e-m+fp/hard/libc_nano.a(lib_a-reent.o)
__lock___env_recursive_mutex
                    0x1               /usr/local/bin/../lib/gcc/arm-none-eabi/8.3.1/../../../../arm-none-eabi/lib/thumb/v7e-m+fp/hard/libc_nano.a(lib_a-lock.o)
__lock___sinit_recursive_mutex
                    0x1               /usr/local/bin/../lib/gcc/arm-none-eabi/8.3.1/../../../../arm-none-eabi/lib/thumb/v7e-m+fp/hard/libc_nano.a(lib_a-lock.o)
__lock___malloc_recursive_mutex
                    0x1               /usr/local/bin/../lib/gcc/arm-none-eabi/8.3.1/../../../../arm-none-eabi/lib/thumb/v7e-m+fp/hard/libc_nano.a(lib_a-lock.o)
ble_lcs             0x14              _build/nrf52832_xxaa_ble_init.c.o
m_gatt              0x1c              _build/nrf52832_xxaa_ble_init.c.o
ble_ics             0x1c              _build/nrf52832_xxaa_ble_init.c.o
ble_scs             0x1c              _build/nrf52832_xxaa_ble_init.c.o
__lock___at_quick_exit_mutex
                    0x1               /usr/local/bin/../lib/gcc/arm-none-eabi/8.3.1/../../../../arm-none-eabi/lib/thumb/v7e-m+fp/hard/libc_nano.a(lib_a-lock.o)
_SEGGER_RTT         0x78              _build/nrf52832_xxaa_SEGGER_RTT.c.o
__lock___dd_hash_mutex
                    0x1               /usr/local/bin/../lib/gcc/arm-none-eabi/8.3.1/../../../../arm-none-eabi/lib/thumb/v7e-m+fp/hard/libc_nano.a(lib_a-lock.o)
__lock___tz_mutex   0x1               /usr/local/bin/../lib/gcc/arm-none-eabi/8.3.1/../../../../arm-none-eabi/lib/thumb/v7e-m+fp/hard/libc_nano.a(lib_a-lock.o)
ble_tcs             0x48              _build/nrf52832_xxaa_ble_init.c.o
__lock___sfp_recursive_mutex
                    0x1               /usr/local/bin/../lib/gcc/arm-none-eabi/8.3.1/../../../../arm-none-eabi/lib/thumb/v7e-m+fp/hard/libc_nano.a(lib_a-lock.o)

Discarded input sections

 .text          0x0000000000000000        0x0 /usr/local/bin/../lib/gcc/arm-none-eabi/8.3.1/thumb/v7e-m+fp/hard/crti.o
 .data          0x0000000000000000        0x0 /usr/local/bin/../lib/gcc/arm-none-eabi/8.3.1/thumb/v7e-m+fp/hard/crti.o
 .bss           0x0000000000000000        0x0 /usr/local/bin/../lib/gcc/arm-none-eabi/8.3.1/thumb/v7e-m+fp/hard/crti.o
 .data          0x0000000000000000        0x4 /usr/local/bin/../lib/gcc/arm-none-eabi/8.3.1/thumb/v7e-m+fp/hard/crtbegin.o
 .data          0x0000000000000000        0x0 /usr/local/bin/../lib/gcc/arm-none-eabi/8.3.1/../../../../arm-none-eabi/lib/thumb/v7e-m+fp/hard/crt0.o
 .bss           0x0000000000000000        0x0 /usr/local/bin/../lib/gcc/arm-none-eabi/8.3.1/../../../../arm-none-eabi/lib/thumb/v7e-m+fp/hard/crt0.o
 .ARM.extab     0x0000000000000000        0x0 /usr/local/bin/../lib/gcc/arm-none-eabi/8.3.1/../../../../arm-none-eabi/lib/thumb/v7e-m+fp/hard/crt0.o
 .text          0x0000000000000000        0x0 /usr/local/bin/../lib/gcc/arm-none-eabi/8.3.1/../../../../arm-none-eabi/lib/thumb/v7e-m+fp/hard/libc_nano.a(lib_a-exit.o)
 .data          0x0000000000000000        0x0 /usr/local/bin/../lib/gcc/arm-none-eabi/8.3.1/../../../../arm-none-eabi/lib/thumb/v7e-m+fp/hard/libc_nano.a(lib_a-exit.o)
 .bss           0x0000000000000000        0x0 /usr/local/bin/../lib/gcc/arm-none-eabi/8.3.1/../../../../arm-none-eabi/lib/thumb/v7e-m+fp/hard/libc_nano.a(lib_a-exit.o)
 .text          0x0000000000000000        0x0 /usr/local/bin/../lib/gcc/arm-none-eabi/8.3.1/../../../../arm-none-eabi/lib/thumb/v7e-m+fp/hard/libc_nano.a(lib_a-impure.o)
 .data          0x0000000000000000        0x0 /usr/local/bin/../lib/gcc/arm-none-eabi/8.3.1/../../../../arm-none-eabi/lib/thumb/v7e-m+fp/hard/libc_nano.a(lib_a-impure.o)
 .bss           0x0000000000000000        0x0 /usr/local/bin/../lib/gcc/arm-none-eabi/8.3.1/../../../../arm-none-eabi/lib/thumb/v7e-m+fp/hard/libc_nano.a(lib_a-impure.o)
 .text          0x0000000000000000        0x0 /usr/local/bin/../lib/gcc/arm-none-eabi/8.3.1/../../../../arm-none-eabi/lib/thumb/v7e-m+fp/hard/libc_nano.a(lib_a-init.o)
 .data          0x0000000000000000        0x0 /usr/local/bin/../lib/gcc/arm-none-eabi/8.3.1/../../../../arm-none-eabi/lib/thumb/v7e-m+fp/hard/libc_nano.a(lib_a-init.o)
 .bss           0x0000000000000000        0x0 /usr/local/bin/../lib/gcc/arm-none-eabi/8.3.1/../../../../arm-none-eabi/lib/thumb/v7e-m+fp/hard/libc_nano.a(lib_a-init.o)
 .text          0x0000000000000000        0x0 /usr/local/bin/../lib/gcc/arm-none-eabi/8.3.1/../../../../arm-none-eabi/lib/thumb/v7e-m+fp/hard/libc_nano.a(lib_a-memset.o)
 .data          0x0000000000000000        0x0 /usr/local/bin/../lib/gcc/arm-none-eabi/8.3.1/../../../../arm-none-eabi/lib/thumb/v7e-m+fp/hard/libc_nano.a(lib_a-memset.o)
Memory Configuration

Name             Origin             Length             Attributes
FLASH            0x000000000001f000 0x000000000005d000 xr
FLASH_STEP_COUNT 0x000000000007c000 0x0000000000003000 xr
FLASH_USER_INFO  0x000000000007f000 0x0000000000001000 xr
RAM              0x0000000020002260 0x000000000000dda0 xrw
*default*        0x0000000000000000 0xffffffffffffffff

Linker script and memory map


.text           0x000000000001f000     0xe6dc
 *(.isr_vector)
 .isr_vector    0x000000000001f000      0x200 _build/nrf52832_xxaa_gcc_startup_nrf52.S.o
                0x000000000001f000                __isr_vector
 *(.text*)
 .text          0x000000000001f200       0x40 /usr/local/bin/../lib/gcc/arm-none-eabi/8.3.1/thumb/v7e-m+fp/hard/crtbegin.o
 .text          0x000000000001f240       0x74 /usr/local/bin/../lib/gcc/arm-none-eabi/8.3.1/../../../../arm-none-eabi/lib/thumb/v7e-m+fp/hard/crt0.o
                0x000000000001f240                _mainCRTStartup
                0x000000000001f240                _start
 .text.exit     0x000000000001f2b4       0x28 /usr/local/bin/../lib/gcc/arm-none-eabi/8.3.1/../../../../arm-none-eabi/lib/thumb/v7e-m+fp/hard/libc_nano.a(lib_a-exit.o)
                0x000000000001f2b4                exit
 .text.__libc_init_array
                0x000000000001f2dc       0x48 /usr/local/bin/../lib/gcc/arm-none-eabi/8.3.1/../../../../arm-none-eabi/lib/thumb/v7e-m+fp/hard/libc_nano.a(lib_a-init.o)
                0x000000000001f2dc                __libc_init_array
 .text.memset   0x000000000001f324       0x10 /usr/local/bin/../lib/gcc/arm-none-eabi/8.3.1/../../../../arm-none-eabi/lib/thumb/v7e-m+fp/hard/libc_nano.a(lib_a-memset.o)
                0x000000000001f324                memset
 .text._exit    0x000000000001f334        0x4 /usr/local/bin/../lib/gcc/arm-none-eabi/8.3.1/../../../../arm-none-eabi/lib/thumb/v7e-m+fp/hard/libnosys.a(_exit.o)
                0x000000000001f334                _exit
 .text.RTC2_IRQ_handler
                0x000000000001f338       0x18 _build/nrf52832_xxaa_main.c.o
                0x000000000001f338                RTC2_IRQ_handler
 .text.startup.main
                0x000000000001f350      0x14c _build/nrf52832_xxaa_main.c.o
                0x000000000001f350                main
 .text.sd_ble_gap_disconnect
                0x000000000001f49c        0x4 _build/nrf52832_xxaa_ble_init.c.o
 .text.sd_ble_gap_appearance_set
                0x000000000001f4a0        0x4 _build/nrf52832_xxaa_ble_init.c.o
 .text.sd_ble_gap_ppcp_set
                0x000000000001f4a4        0x4 _build/nrf52832_xxaa_ble_init.c.o
 .text.sd_ble_gap_device_name_set
                0x000000000001f4a8        0x4 _build/nrf52832_xxaa_ble_init.c.o
 .text.sd_ble_gatts_rw_authorize_reply
                0x000000000001f4ac        0x4 _build/nrf52832_xxaa_ble_init.c.o
 .text.sd_ble_cfg_set
                0x000000000001f4b0        0x4 _build/nrf52832_xxaa_ble_init.c.o
 .text.sd_ble_user_mem_reply
                0x000000000001f4b4        0x4 _build/nrf52832_xxaa_ble_init.c.o
 .text.sd_power_system_off
                0x000000000001f4b8        0x4 _build/nrf52832_xxaa_ble_init.c.o
 .text.conn_params_error_handler
                0x000000000001f4bc        0x4 _build/nrf52832_xxaa_ble_init.c.o
 .text.sys_evt_dispatch
                0x000000000001f4c0       0x18 _build/nrf52832_xxaa_ble_init.c.o
 .text.ble_evt_dispatch
                0x000000000001f4d8      0x110 _build/nrf52832_xxaa_ble_init.c.o
 .text.advertising_start
                0x000000000001f5e8       0x24 _build/nrf52832_xxaa_ble_init.c.o
 .text.pm_evt_handler
                0x000000000001f60c       0xf8 _build/nrf52832_xxaa_ble_init.c.o
 .text.on_adv_evt
                0x000000000001f704       0x30 _build/nrf52832_xxaa_ble_init.c.o
 .text.on_conn_params_evt
                0x000000000001f734       0x34 _build/nrf52832_xxaa_ble_init.c.o
 .text.init_BLE
                0x000000000001f768      0x528 _build/nrf52832_xxaa_ble_init.c.o
                0x000000000001f768                init_BLE
 .text.sd_ble_gatts_service_add
                0x000000000001fc90        0x4 _build/nrf52832_xxaa_ble_lcs.c.o
 .text.sd_ble_gatts_characteristic_add
                0x000000000001fc94        0x4 _build/nrf52832_xxaa_ble_lcs.c.o
 .text.sd_ble_uuid_vs_add
                0x000000000001fc98        0x4 _build/nrf52832_xxaa_ble_lcs.c.o
 .text.ble_lcs_on_ble_evt
                0x000000000001fc9c       0x5c _build/nrf52832_xxaa_ble_lcs.c.o
                0x000000000001fc9c                ble_lcs_on_ble_evt
 .text.ble_lcs_init
                0x000000000001fcf8      0x1c0 _build/nrf52832_xxaa_ble_lcs.c.o
                0x000000000001fcf8                ble_lcs_init
 .text.ble_lcs_data_handler
                0x000000000001feb8       0x60 _build/nrf52832_xxaa_ble_lcs.c.o
                0x000000000001feb8                ble_lcs_data_handler
 .text.sd_ble_gatts_service_add
                0x000000000001ff18        0x4 _build/nrf52832_xxaa_ble_ics.c.o
 .text.sd_ble_gatts_characteristic_add
                0x000000000001ff1c        0x4 _build/nrf52832_xxaa_ble_ics.c.o
 .text.sd_ble_uuid_vs_add
                0x000000000001ff20        0x4 _build/nrf52832_xxaa_ble_ics.c.o
 .text.ble_ics_on_ble_evt
                0x000000000001ff24       0x5c _build/nrf52832_xxaa_ble_ics.c.o
                0x000000000001ff24                ble_ics_on_ble_evt
 .text.ble_ics_init
                0x000000000001ff80      0x1c8 _build/nrf52832_xxaa_ble_ics.c.o
                0x000000000001ff80                ble_ics_init
 .text.ble_ics_data_handler
                0x0000000000020148       0x24 _build/nrf52832_xxaa_ble_ics.c.o
                0x0000000000020148                ble_ics_data_handler
 .text.sd_ble_gatts_service_add
                0x000000000002016c        0x4 _build/nrf52832_xxaa_ble_tcs.c.o
 .text.sd_ble_gatts_characteristic_add
                0x0000000000020170        0x4 _build/nrf52832_xxaa_ble_tcs.c.o
 .text.sd_ble_uuid_vs_add
                0x0000000000020174        0x4 _build/nrf52832_xxaa_ble_tcs.c.o
 .text.ble_tcs_on_ble_evt
                0x0000000000020178      0x28c _build/nrf52832_xxaa_ble_tcs.c.o
                0x0000000000020178                ble_tcs_on_ble_evt
 .text.ble_tcs_init
                0x0000000000020404      0x830 _build/nrf52832_xxaa_ble_tcs.c.o
                0x0000000000020404                ble_tcs_init
 .text.sd_ble_gatts_service_add
                0x0000000000020c34        0x4 _build/nrf52832_xxaa_ble_scs.c.o
 .text.sd_ble_gatts_characteristic_add
                0x0000000000020c38        0x4 _build/nrf52832_xxaa_ble_scs.c.o
 .text.sd_ble_gatts_value_set
                0x0000000000020c3c        0x4 _build/nrf52832_xxaa_ble_scs.c.o
 .text.sd_ble_gatts_hvx
                0x0000000000020c40        0x4 _build/nrf52832_xxaa_ble_scs.c.o
 .text.sd_ble_uuid_vs_add
                0x0000000000020c44        0x4 _build/nrf52832_xxaa_ble_scs.c.o
 .text.ble_scs_on_ble_evt
                0x0000000000020c48       0x60 _build/nrf52832_xxaa_ble_scs.c.o
                0x0000000000020c48                ble_scs_on_ble_evt
 .text.ble_scs_init
                0x0000000000020ca8      0x19c _build/nrf52832_xxaa_ble_scs.c.o
                0x0000000000020ca8                ble_scs_init
 .text.ble_scs_step_count_update
                0x0000000000020e44       0x8c _build/nrf52832_xxaa_ble_scs.c.o
                0x0000000000020e44                ble_scs_step_count_update
 .text.init_LED1
                0x0000000000020ed0        0xc _build/nrf52832_xxaa_gpio.c.o
                0x0000000000020ed0                init_LED1
 .text.turnON_LED1
                0x0000000000020edc       0x10 _build/nrf52832_xxaa_gpio.c.o
                0x0000000000020edc                turnON_LED1
 .text.turnOFF_LED1
                0x0000000000020eec       0x10 _build/nrf52832_xxaa_gpio.c.o
                0x0000000000020eec                turnOFF_LED1
 .text.init_UART
                0x0000000000020efc       0x78 _build/nrf52832_xxaa_uart.c.o
                0x0000000000020efc                init_UART
 .text.putchar_UART
                0x0000000000020f74       0x1c _build/nrf52832_xxaa_uart.c.o
                0x0000000000020f74                putchar_UART
 .text.print    0x0000000000020f90      0x458 _build/nrf52832_xxaa_print.c.o
                0x0000000000020f90                print
 .text.init_SPIM1
                0x00000000000213e8       0x5c _build/nrf52832_xxaa_spim.c.o
                0x00000000000213e8                init_SPIM1
 .text.send_data_SPIM1
                0x0000000000021444       0x4c _build/nrf52832_xxaa_spim.c.o
                0x0000000000021444                send_data_SPIM1
 .text.init_STMcommunication
                0x0000000000021490       0x34 _build/nrf52832_xxaa_stm_communication.c.o
                0x0000000000021490                init_STMcommunication
 .text.write_register_STMcommunication
                0x00000000000214c4       0x4c _build/nrf52832_xxaa_stm_communication.c.o
                0x00000000000214c4                write_register_STMcommunication
 .text.write_image_packet_STMcommunication
                0x0000000000021510       0xac _build/nrf52832_xxaa_stm_communication.c.o
                0x0000000000021510                write_image_packet_STMcommunication
 .text.sd_flash_write
                0x00000000000215bc        0x4 _build/nrf52832_xxaa_flash.c.o
 .text.sd_flash_page_erase
                0x00000000000215c0        0x4 _build/nrf52832_xxaa_flash.c.o
 .text.flash_sys_event_handler
                0x00000000000215c4       0x34 _build/nrf52832_xxaa_flash.c.o
                0x00000000000215c4                flash_sys_event_handler
 .text.erase_FLASH
                0x00000000000215f8       0x5c _build/nrf52832_xxaa_flash.c.o
                0x00000000000215f8                erase_FLASH
 .text.write_FLASH
                0x0000000000021654       0x58 _build/nrf52832_xxaa_flash.c.o
                0x0000000000021654                write_FLASH
 .text.update_step_count
                0x00000000000216ac      0x108 _build/nrf52832_xxaa_step_count_db.c.o
                0x00000000000216ac                update_step_count
 .text.get_most_recent_step_count
                0x00000000000217b4       0x90 _build/nrf52832_xxaa_step_count_db.c.o
                0x00000000000217b4                get_most_recent_step_count
 .text.init_RTC2
                0x0000000000021844       0x30 _build/nrf52832_xxaa_rtc.c.o
                0x0000000000021844                init_RTC2
 .text.set_RTC2_IRQ_callback
                0x0000000000021874        0xc _build/nrf52832_xxaa_rtc.c.o
                0x0000000000021874                set_RTC2_IRQ_callback
 .text.RTC2_IRQHandler
                0x0000000000021880       0x1c _build/nrf52832_xxaa_rtc.c.o
                0x0000000000021880                RTC2_IRQHandler
 .text.nrf_log_backend_serial_std_handler
                0x000000000002189c      0x1ac _build/nrf52832_xxaa_nrf_log_backend_serial.c.o
 .text.nrf_log_backend_serial_hexdump_handler
                0x0000000000021a48      0x194 _build/nrf52832_xxaa_nrf_log_backend_serial.c.o
 .text.nrf_log_backend_init
                0x0000000000021bdc       0x28 _build/nrf52832_xxaa_nrf_log_backend_serial.c.o
                0x0000000000021bdc                nrf_log_backend_init
 .text.nrf_log_backend_std_handler_get
                0x0000000000021c04        0x8 _build/nrf52832_xxaa_nrf_log_backend_serial.c.o
                0x0000000000021c04                nrf_log_backend_std_handler_get
 .text.nrf_log_backend_hexdump_handler_get
                0x0000000000021c0c        0x8 _build/nrf52832_xxaa_nrf_log_backend_serial.c.o
                0x0000000000021c0c                nrf_log_backend_hexdump_handler_get
 .text.nrf_log_init
                0x0000000000021c14       0x34 _build/nrf52832_xxaa_nrf_log_frontend.c.o
                0x0000000000021c14                nrf_log_init
 .text.nrf_log_blocking_backend_set
                0x0000000000021c48        0x8 _build/nrf52832_xxaa_nrf_log_frontend.c.o
                0x0000000000021c48                nrf_log_blocking_backend_set
 .text.nrf_log_frontend_std_0
                0x0000000000021c50       0xa0 _build/nrf52832_xxaa_nrf_log_frontend.c.o
                0x0000000000021c50                nrf_log_frontend_std_0
 .text.nrf_log_frontend_std_1
                0x0000000000021cf0       0xbc _build/nrf52832_xxaa_nrf_log_frontend.c.o
                0x0000000000021cf0                nrf_log_frontend_std_1
 .text.nrf_log_frontend_std_2
                0x0000000000021dac       0xc0 _build/nrf52832_xxaa_nrf_log_frontend.c.o
                0x0000000000021dac                nrf_log_frontend_std_2
 .text.nrf_log_frontend_dequeue
                0x0000000000021e6c      0x144 _build/nrf52832_xxaa_nrf_log_frontend.c.o
                0x0000000000021e6c                nrf_log_frontend_dequeue
 .text.app_error_handler_bare
                0x0000000000021fb0       0x20 _build/nrf52832_xxaa_app_error.c.o
                0x0000000000021fb0                app_error_handler_bare
 .text.app_error_fault_handler
                0x0000000000021fd0       0x58 _build/nrf52832_xxaa_app_error_weak.c.o
                0x0000000000021fd0                app_error_fault_handler
 .text.RTC1_IRQHandler
                0x0000000000022028       0xa0 _build/nrf52832_xxaa_app_timer.c.o
                0x0000000000022028                RTC1_IRQHandler
 .text.SWI0_EGU0_IRQHandler
                0x00000000000220c8      0x664 _build/nrf52832_xxaa_app_timer.c.o
                0x00000000000220c8                SWI0_EGU0_IRQHandler
 .text.app_timer_init
                0x000000000002272c      0x180 _build/nrf52832_xxaa_app_timer.c.o
                0x000000000002272c                app_timer_init
 .text.app_timer_create
                0x00000000000228ac       0x24 _build/nrf52832_xxaa_app_timer.c.o
                0x00000000000228ac                app_timer_create
 .text.app_timer_start
                0x00000000000228d0       0xac _build/nrf52832_xxaa_app_timer.c.o
                0x00000000000228d0                app_timer_start
 .text.app_timer_stop
                0x000000000002297c       0x74 _build/nrf52832_xxaa_app_timer.c.o
                0x000000000002297c                app_timer_stop
 .text.app_util_critical_region_enter
                0x00000000000229f0       0x4c _build/nrf52832_xxaa_app_util_platform.c.o
                0x00000000000229f0                app_util_critical_region_enter
 .text.app_util_critical_region_exit
                0x0000000000022a3c       0x30 _build/nrf52832_xxaa_app_util_platform.c.o
                0x0000000000022a3c                app_util_critical_region_exit
 .text.record_find_by_desc
                0x0000000000022a6c       0xd0 _build/nrf52832_xxaa_fds.c.o
 .text.gc_record_find_next
                0x0000000000022b3c       0xb8 _build/nrf52832_xxaa_fds.c.o
 .text.queue_process
                0x0000000000022bf4      0x8d8 _build/nrf52832_xxaa_fds.c.o
 .text.fs_event_handler
                0x00000000000234cc        0x8 _build/nrf52832_xxaa_fds.c.o
 .text.fds_register
                0x00000000000234d4       0x28 _build/nrf52832_xxaa_fds.c.o
                0x00000000000234d4                fds_register
 .text.fds_init
                0x00000000000234fc      0x2e4 _build/nrf52832_xxaa_fds.c.o
                0x00000000000234fc                fds_init
 .text.fds_record_open
                0x00000000000237e0       0x48 _build/nrf52832_xxaa_fds.c.o
                0x00000000000237e0                fds_record_open
 .text.fds_record_close
                0x0000000000023828       0x48 _build/nrf52832_xxaa_fds.c.o
                0x0000000000023828                fds_record_close
 .text.fds_reserve
                0x0000000000023870       0x80 _build/nrf52832_xxaa_fds.c.o
                0x0000000000023870                fds_reserve
 .text.fds_reserve_cancel
                0x00000000000238f0       0x58 _build/nrf52832_xxaa_fds.c.o
                0x00000000000238f0                fds_reserve_cancel
 .text.fds_record_write
                0x0000000000023948      0x204 _build/nrf52832_xxaa_fds.c.o
                0x0000000000023948                fds_record_write
 .text.fds_record_write_reserved
                0x0000000000023b4c      0x1a4 _build/nrf52832_xxaa_fds.c.o
                0x0000000000023b4c                fds_record_write_reserved
 .text.fds_record_update
                0x0000000000023cf0      0x218 _build/nrf52832_xxaa_fds.c.o
                0x0000000000023cf0                fds_record_update
 .text.fds_file_delete
                0x0000000000023f08       0x74 _build/nrf52832_xxaa_fds.c.o
                0x0000000000023f08                fds_file_delete
 .text.fds_gc   0x0000000000023f7c       0x6c _build/nrf52832_xxaa_fds.c.o
                0x0000000000023f7c                fds_gc
 .text.fds_record_find
                0x0000000000023fe8       0xc0 _build/nrf52832_xxaa_fds.c.o
                0x0000000000023fe8                fds_record_find
 .text.fds_record_find_by_key
                0x00000000000240a8       0xb4 _build/nrf52832_xxaa_fds.c.o
                0x00000000000240a8                fds_record_find_by_key
 .text.fds_record_find_in_file
                0x000000000002415c       0xb4 _build/nrf52832_xxaa_fds.c.o
                0x000000000002415c                fds_record_find_in_file
 .text.fds_record_id_from_desc
                0x0000000000024210       0x10 _build/nrf52832_xxaa_fds.c.o
                0x0000000000024210                fds_record_id_from_desc
 .text.sd_flash_write
                0x0000000000024220        0x4 _build/nrf52832_xxaa_fstorage.c.o
 .text.sd_flash_page_erase
                0x0000000000024224        0x4 _build/nrf52832_xxaa_fstorage.c.o
 .text.queue_process
                0x0000000000024228       0xd0 _build/nrf52832_xxaa_fstorage.c.o
 .text.fs_init  0x00000000000242f8       0xb8 _build/nrf52832_xxaa_fstorage.c.o
                0x00000000000242f8                fs_init
 .text.fs_store
                0x00000000000243b0       0xe4 _build/nrf52832_xxaa_fstorage.c.o
                0x00000000000243b0                fs_store
 .text.fs_erase
                0x0000000000024494       0xe0 _build/nrf52832_xxaa_fstorage.c.o
                0x0000000000024494                fs_erase
 .text.fs_queued_op_count_get
                0x0000000000024574       0x14 _build/nrf52832_xxaa_fstorage.c.o
                0x0000000000024574                fs_queued_op_count_get
 .text.fs_sys_event_handler
                0x0000000000024588      0x2fc _build/nrf52832_xxaa_fstorage.c.o
                0x0000000000024588                fs_sys_event_handler
 .text.sdk_mapped_flags_first_key_index_get
                0x0000000000024884       0x30 _build/nrf52832_xxaa_sdk_mapped_flags.c.o
                0x0000000000024884                sdk_mapped_flags_first_key_index_get
 .text.sdk_mapped_flags_update_by_key
                0x00000000000248b4       0x38 _build/nrf52832_xxaa_sdk_mapped_flags.c.o
                0x00000000000248b4                sdk_mapped_flags_update_by_key
 .text.sdk_mapped_flags_bulk_update_by_key
                0x00000000000248ec      0x100 _build/nrf52832_xxaa_sdk_mapped_flags.c.o
                0x00000000000248ec                sdk_mapped_flags_bulk_update_by_key
 .text.sdk_mapped_flags_get_by_key
                0x00000000000249ec       0x38 _build/nrf52832_xxaa_sdk_mapped_flags.c.o
                0x00000000000249ec                sdk_mapped_flags_get_by_key
 .text.sdk_mapped_flags_key_list_get
                0x0000000000024a24       0x34 _build/nrf52832_xxaa_sdk_mapped_flags.c.o
                0x0000000000024a24                sdk_mapped_flags_key_list_get
 .text.POWER_CLOCK_IRQHandler
                0x0000000000024a58       0x7c _build/nrf52832_xxaa_nrf_drv_clock.c.o
                0x0000000000024a58                POWER_CLOCK_IRQHandler
 .text.nrf_drv_clock_on_soc_event
                0x0000000000024ad4       0x24 _build/nrf52832_xxaa_nrf_drv_clock.c.o
                0x0000000000024ad4                nrf_drv_clock_on_soc_event
 .text.nrf_drv_clock_on_sd_enable
                0x0000000000024af8       0x68 _build/nrf52832_xxaa_nrf_drv_clock.c.o
                0x0000000000024af8                nrf_drv_clock_on_sd_enable
 .text.nrf_drv_common_irq_enable
                0x0000000000024b60       0x48 _build/nrf52832_xxaa_nrf_drv_common.c.o
                0x0000000000024b60                nrf_drv_common_irq_enable
 .text.GPIOTE_IRQHandler
                0x0000000000024ba8      0x4f8 _build/nrf52832_xxaa_nrf_drv_gpiote.c.o
                0x0000000000024ba8                GPIOTE_IRQHandler
 .text.UARTE0_UART0_IRQHandler
                0x00000000000250a0      0x2dc _build/nrf52832_xxaa_nrf_drv_uart.c.o
                0x00000000000250a0                UARTE0_UART0_IRQHandler
 .text.SEGGER_RTT_WriteNoLock
                0x000000000002537c      0x17c _build/nrf52832_xxaa_SEGGER_RTT.c.o
                0x000000000002537c                SEGGER_RTT_WriteNoLock
 .text.SEGGER_RTT_Init
                0x00000000000254f8       0x64 _build/nrf52832_xxaa_SEGGER_RTT.c.o
                0x00000000000254f8                SEGGER_RTT_Init
 .text.sd_ble_gap_addr_get
                0x000000000002555c        0x4 _build/nrf52832_xxaa_ble_advdata.c.o
 .text.sd_ble_gap_adv_data_set
                0x0000000000025560        0x4 _build/nrf52832_xxaa_ble_advdata.c.o
 .text.sd_ble_gap_appearance_get
                0x0000000000025564        0x4 _build/nrf52832_xxaa_ble_advdata.c.o
 .text.sd_ble_gap_device_name_get
                0x0000000000025568        0x4 _build/nrf52832_xxaa_ble_advdata.c.o
 .text.sd_ble_uuid_encode
                0x000000000002556c        0x4 _build/nrf52832_xxaa_ble_advdata.c.o
 .text.uuid_list_sized_encode.isra.0
                0x0000000000025570       0xec _build/nrf52832_xxaa_ble_advdata.c.o
 .text.adv_data_encode
                0x000000000002565c      0x408 _build/nrf52832_xxaa_ble_advdata.c.o
                0x000000000002565c                adv_data_encode
 .text.ble_advdata_set
                0x0000000000025a64       0x68 _build/nrf52832_xxaa_ble_advdata.c.o
                0x0000000000025a64                ble_advdata_set
 .text.sd_ble_gap_adv_start
                0x0000000000025acc        0x4 _build/nrf52832_xxaa_ble_advertising.c.o
 .text.ble_advertising_start.part.1
                0x0000000000025ad0      0x244 _build/nrf52832_xxaa_ble_advertising.c.o
 .text.ble_advertising_init
                0x0000000000025d14      0x180 _build/nrf52832_xxaa_ble_advertising.c.o
                0x0000000000025d14                ble_advertising_init
 .text.ble_advertising_start
                0x0000000000025e94       0x40 _build/nrf52832_xxaa_ble_advertising.c.o
                0x0000000000025e94                ble_advertising_start
 .text.ble_advertising_on_ble_evt
                0x0000000000025ed4       0xbc _build/nrf52832_xxaa_ble_advertising.c.o
                0x0000000000025ed4                ble_advertising_on_ble_evt
 .text.ble_advertising_on_sys_evt
                0x0000000000025f90       0x60 _build/nrf52832_xxaa_ble_advertising.c.o
                0x0000000000025f90                ble_advertising_on_sys_evt
 .text.sd_ble_gap_conn_param_update
                0x0000000000025ff0        0x4 _build/nrf52832_xxaa_ble_conn_params.c.o
 .text.sd_ble_gap_disconnect
                0x0000000000025ff4        0x4 _build/nrf52832_xxaa_ble_conn_params.c.o
 .text.sd_ble_gap_ppcp_set
                0x0000000000025ff8        0x4 _build/nrf52832_xxaa_ble_conn_params.c.o
 .text.sd_ble_gap_ppcp_get
                0x0000000000025ffc        0x4 _build/nrf52832_xxaa_ble_conn_params.c.o
 .text.update_timeout_handler
                0x0000000000026000       0x74 _build/nrf52832_xxaa_ble_conn_params.c.o
 .text.conn_params_negotiation
                0x0000000000026074       0x90 _build/nrf52832_xxaa_ble_conn_params.c.o
 .text.ble_conn_params_init
                0x0000000000026104       0x74 _build/nrf52832_xxaa_ble_conn_params.c.o
                0x0000000000026104                ble_conn_params_init
 .text.ble_conn_params_on_ble_evt
                0x0000000000026178       0xbc _build/nrf52832_xxaa_ble_conn_params.c.o
                0x0000000000026178                ble_conn_params_on_ble_evt
 .text.ble_conn_state_on_ble_evt
                0x0000000000026234      0x114 _build/nrf52832_xxaa_ble_conn_state.c.o
                0x0000000000026234                ble_conn_state_on_ble_evt
 .text.ble_conn_state_role
                0x0000000000026348       0x2c _build/nrf52832_xxaa_ble_conn_state.c.o
                0x0000000000026348                ble_conn_state_role
 .text.ble_conn_state_encrypted
                0x0000000000026374       0x10 _build/nrf52832_xxaa_ble_conn_state.c.o
                0x0000000000026374                ble_conn_state_encrypted
 .text.ble_conn_state_mitm_protected
                0x0000000000026384       0x10 _build/nrf52832_xxaa_ble_conn_state.c.o
                0x0000000000026384                ble_conn_state_mitm_protected
 .text.ble_conn_state_conn_handles
                0x0000000000026394       0x18 _build/nrf52832_xxaa_ble_conn_state.c.o
                0x0000000000026394                ble_conn_state_conn_handles
 .text.ble_conn_state_user_flag_acquire
                0x00000000000263ac       0x30 _build/nrf52832_xxaa_ble_conn_state.c.o
                0x00000000000263ac                ble_conn_state_user_flag_acquire
 .text.ble_conn_state_user_flag_get
                0x00000000000263dc       0x28 _build/nrf52832_xxaa_ble_conn_state.c.o
                0x00000000000263dc                ble_conn_state_user_flag_get
 .text.ble_conn_state_user_flag_set
                0x0000000000026404       0x28 _build/nrf52832_xxaa_ble_conn_state.c.o
                0x0000000000026404                ble_conn_state_user_flag_set
 .text.ble_conn_state_user_flag_collection
                0x000000000002642c       0x1c _build/nrf52832_xxaa_ble_conn_state.c.o
                0x000000000002642c                ble_conn_state_user_flag_collection
 .text.ble_srv_is_notification_enabled
                0x0000000000026448        0x8 _build/nrf52832_xxaa_ble_srv_common.c.o
                0x0000000000026448                ble_srv_is_notification_enabled
 .text.local_db_apply_in_evt.part.1
                0x0000000000026450       0x94 _build/nrf52832_xxaa_gatt_cache_manager.c.o
 .text.service_changed_pending_flags_check.part.2
                0x00000000000264e4       0xf8 _build/nrf52832_xxaa_gatt_cache_manager.c.o
 .text.local_db_update_in_evt
                0x00000000000265dc       0x9c _build/nrf52832_xxaa_gatt_cache_manager.c.o
 .text.gcm_gscm_evt_handler
                0x0000000000026678       0x80 _build/nrf52832_xxaa_gatt_cache_manager.c.o
                0x0000000000026678                gcm_gscm_evt_handler
 .text.gcm_im_evt_handler
                0x00000000000266f8       0x38 _build/nrf52832_xxaa_gatt_cache_manager.c.o
                0x00000000000266f8                gcm_im_evt_handler
 .text.gcm_smd_evt_handler
                0x0000000000026730       0x10 _build/nrf52832_xxaa_gatt_cache_manager.c.o
                0x0000000000026730                gcm_smd_evt_handler
 .text.gcm_init
                0x0000000000026740       0x54 _build/nrf52832_xxaa_gatt_cache_manager.c.o
                0x0000000000026740                gcm_init
 .text.gcm_ble_evt_handler
                0x0000000000026794      0x124 _build/nrf52832_xxaa_gatt_cache_manager.c.o
                0x0000000000026794                gcm_ble_evt_handler
 .text.gcm_local_database_has_changed
                0x00000000000268b8       0x70 _build/nrf52832_xxaa_gatt_cache_manager.c.o
                0x00000000000268b8                gcm_local_database_has_changed
 .text.sd_ble_gatts_service_changed
                0x0000000000026928        0x4 _build/nrf52832_xxaa_gatts_cache_manager.c.o
 .text.sd_ble_gatts_sys_attr_set
                0x000000000002692c        0x4 _build/nrf52832_xxaa_gatts_cache_manager.c.o
 .text.sd_ble_gatts_sys_attr_get
                0x0000000000026930        0x4 _build/nrf52832_xxaa_gatts_cache_manager.c.o
 .text.gscm_pdb_evt_handler
                0x0000000000026934       0x8c _build/nrf52832_xxaa_gatts_cache_manager.c.o
                0x0000000000026934                gscm_pdb_evt_handler
 .text.gscm_init
                0x00000000000269c0       0x10 _build/nrf52832_xxaa_gatts_cache_manager.c.o
                0x00000000000269c0                gscm_init
 .text.gscm_local_db_cache_update
                0x00000000000269d0       0x98 _build/nrf52832_xxaa_gatts_cache_manager.c.o
                0x00000000000269d0                gscm_local_db_cache_update
 .text.gscm_local_db_cache_apply
                0x0000000000026a68       0x84 _build/nrf52832_xxaa_gatts_cache_manager.c.o
                0x0000000000026a68                gscm_local_db_cache_apply
 .text.gscm_local_database_has_changed
                0x0000000000026aec       0x60 _build/nrf52832_xxaa_gatts_cache_manager.c.o
                0x0000000000026aec                gscm_local_database_has_changed
 .text.gscm_service_changed_ind_needed
                0x0000000000026b4c       0x24 _build/nrf52832_xxaa_gatts_cache_manager.c.o
                0x0000000000026b4c                gscm_service_changed_ind_needed
 .text.gscm_service_changed_ind_send
                0x0000000000026b70       0x2c _build/nrf52832_xxaa_gatts_cache_manager.c.o
                0x0000000000026b70                gscm_service_changed_ind_send
 .text.gscm_db_change_notification_done
                0x0000000000026b9c       0x24 _build/nrf52832_xxaa_gatts_cache_manager.c.o
                0x0000000000026b9c                gscm_db_change_notification_done
 .text.sd_ecb_block_encrypt
                0x0000000000026bc0        0x4 _build/nrf52832_xxaa_id_manager.c.o
 .text.im_ble_evt_handler
                0x0000000000026bc4      0x264 _build/nrf52832_xxaa_id_manager.c.o
                0x0000000000026bc4                im_ble_evt_handler
 .text.im_pdb_evt_handler
                0x0000000000026e28      0x118 _build/nrf52832_xxaa_id_manager.c.o
                0x0000000000026e28                im_pdb_evt_handler
 .text.im_init  0x0000000000026f40       0x34 _build/nrf52832_xxaa_id_manager.c.o
                0x0000000000026f40                im_init
 .text.im_peer_id_get_by_conn_handle
                0x0000000000026f74       0x40 _build/nrf52832_xxaa_id_manager.c.o
                0x0000000000026f74                im_peer_id_get_by_conn_handle
 .text.im_ble_addr_get
                0x0000000000026fb4       0x50 _build/nrf52832_xxaa_id_manager.c.o
                0x0000000000026fb4                im_ble_addr_get
 .text.im_master_ids_compare
                0x0000000000027004       0x44 _build/nrf52832_xxaa_id_manager.c.o
                0x0000000000027004                im_master_ids_compare
 .text.im_peer_id_get_by_master_id
                0x0000000000027048       0xf4 _build/nrf52832_xxaa_id_manager.c.o
                0x0000000000027048                im_peer_id_get_by_master_id
 .text.im_conn_handle_get
                0x000000000002713c       0x38 _build/nrf52832_xxaa_id_manager.c.o
                0x000000000002713c                im_conn_handle_get
 .text.im_master_id_is_valid
                0x0000000000027174       0x30 _build/nrf52832_xxaa_id_manager.c.o
                0x0000000000027174                im_master_id_is_valid
 .text.im_new_peer_id
                0x00000000000271a4       0x3c _build/nrf52832_xxaa_id_manager.c.o
                0x00000000000271a4                im_new_peer_id
 .text.im_peer_free
                0x00000000000271e0       0x7c _build/nrf52832_xxaa_id_manager.c.o
                0x00000000000271e0                im_peer_free
 .text.sd_ble_gap_data_length_update
                0x000000000002725c        0x4 _build/nrf52832_xxaa_nrf_ble_gatt.c.o
 .text.sd_ble_gattc_exchange_mtu_request
                0x0000000000027260        0x4 _build/nrf52832_xxaa_nrf_ble_gatt.c.o
 .text.sd_ble_gatts_exchange_mtu_reply
                0x0000000000027264        0x4 _build/nrf52832_xxaa_nrf_ble_gatt.c.o
 .text.nrf_ble_gatt_init
                0x0000000000027268       0x34 _build/nrf52832_xxaa_nrf_ble_gatt.c.o
                0x0000000000027268                nrf_ble_gatt_init
 .text.nrf_ble_gatt_on_ble_evt
                0x000000000002729c      0x210 _build/nrf52832_xxaa_nrf_ble_gatt.c.o
                0x000000000002729c                nrf_ble_gatt_on_ble_evt
 .text.peer_data_delete
                0x00000000000274ac       0x90 _build/nrf52832_xxaa_peer_data_storage.c.o
 .text.fds_evt_handler
                0x000000000002753c      0x134 _build/nrf52832_xxaa_peer_data_storage.c.o
 .text.pds_init
                0x0000000000027670       0x6c _build/nrf52832_xxaa_peer_data_storage.c.o
                0x0000000000027670                pds_init
 .text.pds_peer_data_read
                0x00000000000276dc       0x88 _build/nrf52832_xxaa_peer_data_storage.c.o
                0x00000000000276dc                pds_peer_data_read
 .text.pds_peer_data_iterate_prepare
                0x0000000000027764       0x10 _build/nrf52832_xxaa_peer_data_storage.c.o
                0x0000000000027764                pds_peer_data_iterate_prepare
 .text.pds_peer_data_iterate
                0x0000000000027774       0x50 _build/nrf52832_xxaa_peer_data_storage.c.o
                0x0000000000027774                pds_peer_data_iterate
 .text.pds_space_reserve
                0x00000000000277c4       0x30 _build/nrf52832_xxaa_peer_data_storage.c.o
                0x00000000000277c4                pds_space_reserve
 .text.pds_space_reserve_cancel
                0x00000000000277f4       0x18 _build/nrf52832_xxaa_peer_data_storage.c.o
                0x00000000000277f4                pds_space_reserve_cancel
 .text.pds_peer_data_store
                0x000000000002780c       0xd4 _build/nrf52832_xxaa_peer_data_storage.c.o
                0x000000000002780c                pds_peer_data_store
 .text.pds_peer_id_allocate
                0x00000000000278e0        0x8 _build/nrf52832_xxaa_peer_data_storage.c.o
                0x00000000000278e0                pds_peer_id_allocate
 .text.pds_peer_id_free
                0x00000000000278e8       0x18 _build/nrf52832_xxaa_peer_data_storage.c.o
                0x00000000000278e8                pds_peer_id_free
 .text.pds_peer_id_is_allocated
                0x0000000000027900        0x4 _build/nrf52832_xxaa_peer_data_storage.c.o
                0x0000000000027900                pds_peer_id_is_allocated
 .text.pds_next_peer_id_get
                0x0000000000027904        0x4 _build/nrf52832_xxaa_peer_data_storage.c.o
                0x0000000000027904                pds_next_peer_id_get
 .text.pds_next_deleted_peer_id_get
                0x0000000000027908        0x4 _build/nrf52832_xxaa_peer_data_storage.c.o
                0x0000000000027908                pds_next_deleted_peer_id_get
 .text.pdb_init
                0x000000000002790c      0x114 _build/nrf52832_xxaa_peer_database.c.o
                0x000000000002790c                pdb_init
 .text.pdb_peer_allocate
                0x0000000000027a20        0x4 _build/nrf52832_xxaa_peer_database.c.o
                0x0000000000027a20                pdb_peer_allocate
 .text.pdb_peer_data_ptr_get
                0x0000000000027a24        0x8 _build/nrf52832_xxaa_peer_database.c.o
                0x0000000000027a24                pdb_peer_data_ptr_get
 .text.pdb_write_buf_get
                0x0000000000027a2c      0x508 _build/nrf52832_xxaa_peer_database.c.o
                0x0000000000027a2c                pdb_write_buf_get
 .text.pdb_write_buf_release
                0x0000000000027f34      0x24c _build/nrf52832_xxaa_peer_database.c.o
                0x0000000000027f34                pdb_write_buf_release
 .text.pdb_peer_free
                0x0000000000028180      0x198 _build/nrf52832_xxaa_peer_database.c.o
                0x0000000000028180                pdb_peer_free
 .text.pdb_write_buf_store_prepare
                0x0000000000028318      0x244 _build/nrf52832_xxaa_peer_database.c.o
                0x0000000000028318                pdb_write_buf_store_prepare
 .text.pdb_write_buf_store
                0x000000000002855c      0x2a8 _build/nrf52832_xxaa_peer_database.c.o
                0x000000000002855c                pdb_write_buf_store
 .text.pdb_pds_evt_handler
                0x0000000000028804      0x594 _build/nrf52832_xxaa_peer_database.c.o
                0x0000000000028804                pdb_pds_evt_handler
 .text.pdb_next_peer_id_get
                0x0000000000028d98        0x4 _build/nrf52832_xxaa_peer_database.c.o
                0x0000000000028d98                pdb_next_peer_id_get
 .text.pdb_next_deleted_peer_id_get
                0x0000000000028d9c        0x4 _build/nrf52832_xxaa_peer_database.c.o
                0x0000000000028d9c                pdb_next_deleted_peer_id_get
 .text.pdb_raw_store
                0x0000000000028da0        0x8 _build/nrf52832_xxaa_peer_database.c.o
                0x0000000000028da0                pdb_raw_store
 .text.peer_id_init
                0x0000000000028da8       0x2c _build/nrf52832_xxaa_peer_id.c.o
                0x0000000000028da8                peer_id_init
 .text.peer_id_allocate
                0x0000000000028dd4       0x3c _build/nrf52832_xxaa_peer_id.c.o
                0x0000000000028dd4                peer_id_allocate
 .text.peer_id_delete
                0x0000000000028e10       0x24 _build/nrf52832_xxaa_peer_id.c.o
                0x0000000000028e10                peer_id_delete
 .text.peer_id_free
                0x0000000000028e34       0x28 _build/nrf52832_xxaa_peer_id.c.o
                0x0000000000028e34                peer_id_free
 .text.peer_id_is_allocated
                0x0000000000028e5c       0x14 _build/nrf52832_xxaa_peer_id.c.o
                0x0000000000028e5c                peer_id_is_allocated
 .text.peer_id_get_next_used
                0x0000000000028e70       0x70 _build/nrf52832_xxaa_peer_id.c.o
                0x0000000000028e70                peer_id_get_next_used
 .text.peer_id_get_next_deleted
                0x0000000000028ee0       0x40 _build/nrf52832_xxaa_peer_id.c.o
                0x0000000000028ee0                peer_id_get_next_deleted
 .text.pm_pdb_evt_handler
                0x0000000000028f20      0x21c _build/nrf52832_xxaa_peer_manager.c.o
                0x0000000000028f20                pm_pdb_evt_handler
 .text.pm_sm_evt_handler
                0x000000000002913c      0x1c8 _build/nrf52832_xxaa_peer_manager.c.o
                0x000000000002913c                pm_sm_evt_handler
 .text.pm_gcm_evt_handler
                0x0000000000029304       0xac _build/nrf52832_xxaa_peer_manager.c.o
                0x0000000000029304                pm_gcm_evt_handler
 .text.pm_im_evt_handler
                0x00000000000293b0       0x74 _build/nrf52832_xxaa_peer_manager.c.o
                0x00000000000293b0                pm_im_evt_handler
 .text.pm_on_ble_evt
                0x0000000000029424       0x24 _build/nrf52832_xxaa_peer_manager.c.o
                0x0000000000029424                pm_on_ble_evt
 .text.pm_init  0x0000000000029448       0x84 _build/nrf52832_xxaa_peer_manager.c.o
                0x0000000000029448                pm_init
 .text.pm_register
                0x00000000000294cc       0x38 _build/nrf52832_xxaa_peer_manager.c.o
                0x00000000000294cc                pm_register
 .text.pm_sec_params_set
                0x0000000000029504       0x14 _build/nrf52832_xxaa_peer_manager.c.o
                0x0000000000029504                pm_sec_params_set
 .text.pm_conn_sec_config_reply
                0x0000000000029518        0x4 _build/nrf52832_xxaa_peer_manager.c.o
                0x0000000000029518                pm_conn_sec_config_reply
 .text.pm_local_database_has_changed
                0x000000000002951c       0x10 _build/nrf52832_xxaa_peer_manager.c.o
                0x000000000002951c                pm_local_database_has_changed
 .text.pm_buffer_init
                0x000000000002952c       0x3c _build/nrf52832_xxaa_pm_buffer.c.o
                0x000000000002952c                pm_buffer_init
 .text.pm_buffer_block_acquire
                0x0000000000029568       0x90 _build/nrf52832_xxaa_pm_buffer.c.o
                0x0000000000029568                pm_buffer_block_acquire
 .text.pm_buffer_ptr_get
                0x00000000000295f8       0x30 _build/nrf52832_xxaa_pm_buffer.c.o
                0x00000000000295f8                pm_buffer_ptr_get
 .text.pm_buffer_release
                0x0000000000029628       0x30 _build/nrf52832_xxaa_pm_buffer.c.o
                0x0000000000029628                pm_buffer_release
 .text.pm_mutex_init
                0x0000000000029658       0x10 _build/nrf52832_xxaa_pm_mutex.c.o
                0x0000000000029658                pm_mutex_init
 .text.pm_mutex_lock
                0x0000000000029668       0x54 _build/nrf52832_xxaa_pm_mutex.c.o
                0x0000000000029668                pm_mutex_lock
 .text.pm_mutex_unlock
                0x00000000000296bc       0x44 _build/nrf52832_xxaa_pm_mutex.c.o
                0x00000000000296bc                pm_mutex_unlock
 .text.pm_mutex_lock_first_available
                0x0000000000029700       0x78 _build/nrf52832_xxaa_pm_mutex.c.o
                0x0000000000029700                pm_mutex_lock_first_available
 .text.pm_mutex_lock_status_get
                0x0000000000029778       0x20 _build/nrf52832_xxaa_pm_mutex.c.o
                0x0000000000029778                pm_mutex_lock_status_get
 .text.sd_ble_gap_authenticate
                0x0000000000029798        0x4 _build/nrf52832_xxaa_security_dispatcher.c.o
 .text.sd_ble_gap_sec_params_reply
                0x000000000002979c        0x4 _build/nrf52832_xxaa_security_dispatcher.c.o
 .text.sd_ble_gap_encrypt
                0x00000000000297a0        0x4 _build/nrf52832_xxaa_security_dispatcher.c.o
 .text.sd_ble_gap_sec_info_reply
                0x00000000000297a4        0x4 _build/nrf52832_xxaa_security_dispatcher.c.o
 .text.pairing_failure
                0x00000000000297a8       0x80 _build/nrf52832_xxaa_security_dispatcher.c.o
 .text.smd_pdb_evt_handler
                0x0000000000029828       0x3c _build/nrf52832_xxaa_security_dispatcher.c.o
                0x0000000000029828                smd_pdb_evt_handler
 .text.smd_init
                0x0000000000029864       0x58 _build/nrf52832_xxaa_security_dispatcher.c.o
                0x0000000000029864                smd_init
 .text.smd_params_reply
                0x00000000000298bc      0x1b4 _build/nrf52832_xxaa_security_dispatcher.c.o
                0x00000000000298bc                smd_params_reply
 .text.smd_link_secure
                0x0000000000029a70      0x26c _build/nrf52832_xxaa_security_dispatcher.c.o
                0x0000000000029a70                smd_link_secure
 .text.smd_ble_evt_handler
                0x0000000000029cdc      0x3a0 _build/nrf52832_xxaa_security_dispatcher.c.o
                0x0000000000029cdc                smd_ble_evt_handler
 .text.link_secure
                0x000000000002a07c      0x150 _build/nrf52832_xxaa_security_manager.c.o
 .text.smd_params_reply_perform
                0x000000000002a1cc      0x15c _build/nrf52832_xxaa_security_manager.c.o
 .text.sm_smd_evt_handler
                0x000000000002a328       0x80 _build/nrf52832_xxaa_security_manager.c.o
                0x000000000002a328                sm_smd_evt_handler
 .text.sm_pdb_evt_handler
                0x000000000002a3a8      0x178 _build/nrf52832_xxaa_security_manager.c.o
                0x000000000002a3a8                sm_pdb_evt_handler
 .text.sm_init  0x000000000002a520       0xbc _build/nrf52832_xxaa_security_manager.c.o
                0x000000000002a520                sm_init
 .text.sm_ble_evt_handler
                0x000000000002a5dc       0x80 _build/nrf52832_xxaa_security_manager.c.o
                0x000000000002a5dc                sm_ble_evt_handler
 .text.sm_sec_params_set
                0x000000000002a65c       0x78 _build/nrf52832_xxaa_security_manager.c.o
                0x000000000002a65c                sm_sec_params_set
 .text.sm_conn_sec_config_reply
                0x000000000002a6d4       0x14 _build/nrf52832_xxaa_security_manager.c.o
                0x000000000002a6d4                sm_conn_sec_config_reply
 .text          0x000000000002a6e8       0x3c _build/nrf52832_xxaa_gcc_startup_nrf52.S.o
                0x000000000002a6e8                Reset_Handler
                0x000000000002a710                NMI_Handler
                0x000000000002a712                HardFault_Handler
                0x000000000002a714                MemoryManagement_Handler
                0x000000000002a716                BusFault_Handler
                0x000000000002a718                UsageFault_Handler
                0x000000000002a71a                SVC_Handler
                0x000000000002a71c                DebugMon_Handler
                0x000000000002a71e                PendSV_Handler
                0x000000000002a720                SysTick_Handler
                0x000000000002a722                TIMER2_IRQHandler
                0x000000000002a722                RTC0_IRQHandler
                0x000000000002a722                PWM1_IRQHandler
                0x000000000002a722                RADIO_IRQHandler
                0x000000000002a722                PDM_IRQHandler
                0x000000000002a722                TEMP_IRQHandler
                0x000000000002a722                QDEC_IRQHandler
                0x000000000002a722                TIMER3_IRQHandler
                0x000000000002a722                FPU_IRQHandler
                0x000000000002a722                SPIM0_SPIS0_TWIM0_TWIS0_SPI0_TWI0_IRQHandler
                0x000000000002a722                TIMER4_IRQHandler
                0x000000000002a722                I2S_IRQHandler
                0x000000000002a722                SWI4_EGU4_IRQHandler
                0x000000000002a722                TIMER0_IRQHandler
                0x000000000002a722                TIMER1_IRQHandler
                0x000000000002a722                PWM2_IRQHandler
                0x000000000002a722                ECB_IRQHandler
                0x000000000002a722                SPIM1_SPIS1_TWIM1_TWIS1_SPI1_TWI1_IRQHandler
                0x000000000002a722                Default_Handler
                0x000000000002a722                SAADC_IRQHandler
                0x000000000002a722                CCM_AAR_IRQHandler
                0x000000000002a722                WDT_IRQHandler
                0x000000000002a722                SWI5_EGU5_IRQHandler
                0x000000000002a722                RNG_IRQHandler
                0x000000000002a722                PWM0_IRQHandler
                0x000000000002a722                SWI3_EGU3_IRQHandler
                0x000000000002a722                SWI1_EGU1_IRQHandler
                0x000000000002a722                SPIM2_SPIS2_SPI2_IRQHandler
                0x000000000002a722                NFCT_IRQHandler
                0x000000000002a722                MWU_IRQHandler
                0x000000000002a722                COMP_LPCOMP_IRQHandler
 .text.SystemInit
                0x000000000002a724      0x33c _build/nrf52832_xxaa_system_nrf52.c.o
                0x000000000002a724                SystemInit
 .text.sd_evt_get
                0x000000000002aa60        0x4 _build/nrf52832_xxaa_softdevice_handler.c.o
 .text.sd_softdevice_enable
                0x000000000002aa64        0x4 _build/nrf52832_xxaa_softdevice_handler.c.o
 .text.sd_ble_enable
                0x000000000002aa68        0x4 _build/nrf52832_xxaa_softdevice_handler.c.o
 .text.sd_ble_evt_get
                0x000000000002aa6c        0x4 _build/nrf52832_xxaa_softdevice_handler.c.o
 .text.softdevice_fault_handler
                0x000000000002aa70        0x4 _build/nrf52832_xxaa_softdevice_handler.c.o
                0x000000000002aa70                softdevice_fault_handler
 .text.intern_softdevice_events_execute.part.1
                0x000000000002aa74       0xd4 _build/nrf52832_xxaa_softdevice_handler.c.o
 .text.softdevice_handler_is_enabled
                0x000000000002ab48        0xc _build/nrf52832_xxaa_softdevice_handler.c.o
                0x000000000002ab48                softdevice_handler_is_enabled
 .text.softdevice_handler_init
                0x000000000002ab54       0x90 _build/nrf52832_xxaa_softdevice_handler.c.o
                0x000000000002ab54                softdevice_handler_init
 .text.softdevice_ble_evt_handler_set
                0x000000000002abe4       0x14 _build/nrf52832_xxaa_softdevice_handler.c.o
                0x000000000002abe4                softdevice_ble_evt_handler_set
 .text.softdevice_sys_evt_handler_set
                0x000000000002abf8       0x14 _build/nrf52832_xxaa_softdevice_handler.c.o
                0x000000000002abf8                softdevice_sys_evt_handler_set
 .text.SWI2_EGU2_IRQHandler
                0x000000000002ac0c       0x30 _build/nrf52832_xxaa_softdevice_handler.c.o
                0x000000000002ac0c                SWI2_EGU2_IRQHandler
 .text.softdevice_app_ram_start_get
                0x000000000002ac3c       0x14 _build/nrf52832_xxaa_softdevice_handler.c.o
                0x000000000002ac3c                softdevice_app_ram_start_get
 .text.softdevice_enable
                0x000000000002ac50       0x68 _build/nrf52832_xxaa_softdevice_handler.c.o
                0x000000000002ac50                softdevice_enable
 .text          0x000000000002acb8      0x378 /usr/local/bin/../lib/gcc/arm-none-eabi/8.3.1/thumb/v7e-m+fp/hard/libgcc.a(_arm_addsubdf3.o)
                0x000000000002acb8                __aeabi_drsub
                0x000000000002acc0                __aeabi_dsub
                0x000000000002acc0                __subdf3
                0x000000000002acc4                __adddf3
                0x000000000002acc4                __aeabi_dadd
                0x000000000002af3c                __aeabi_ui2d
                0x000000000002af3c                __floatunsidf
                0x000000000002af5c                __floatsidf
                0x000000000002af5c                __aeabi_i2d
                0x000000000002af80                __extendsfdf2
                0x000000000002af80                __aeabi_f2d
                0x000000000002afc4                __aeabi_ul2d
                0x000000000002afc4                __floatundidf
                0x000000000002afd4                __floatdidf
                0x000000000002afd4                __aeabi_l2d
 .text          0x000000000002b030      0x424 /usr/local/bin/../lib/gcc/arm-none-eabi/8.3.1/thumb/v7e-m+fp/hard/libgcc.a(_arm_muldivdf3.o)
                0x000000000002b030                __aeabi_dmul
                0x000000000002b030                __muldf3
                0x000000000002b284                __aeabi_ddiv
                0x000000000002b284                __divdf3
 .text          0x000000000002b454      0x110 /usr/local/bin/../lib/gcc/arm-none-eabi/8.3.1/thumb/v7e-m+fp/hard/libgcc.a(_arm_cmpdf2.o)
                0x000000000002b454                __gtdf2
                0x000000000002b454                __gedf2
                0x000000000002b45c                __ltdf2
                0x000000000002b45c                __ledf2
                0x000000000002b464                __cmpdf2
                0x000000000002b464                __eqdf2
                0x000000000002b464                __nedf2
                0x000000000002b4e0                __aeabi_cdrcmple
                0x000000000002b4f0                __aeabi_cdcmple
                0x000000000002b4f0                __aeabi_cdcmpeq
                0x000000000002b500                __aeabi_dcmpeq
                0x000000000002b514                __aeabi_dcmplt
                0x000000000002b528                __aeabi_dcmple
                0x000000000002b53c                __aeabi_dcmpge
                0x000000000002b550                __aeabi_dcmpgt
 .text          0x000000000002b564       0x50 /usr/local/bin/../lib/gcc/arm-none-eabi/8.3.1/thumb/v7e-m+fp/hard/libgcc.a(_arm_fixdfsi.o)
                0x000000000002b564                __fixdfsi
                0x000000000002b564                __aeabi_d2iz
 .text.memcmp   0x000000000002b5b4       0x1c /usr/local/bin/../lib/gcc/arm-none-eabi/8.3.1/../../../../arm-none-eabi/lib/thumb/v7e-m+fp/hard/libc_nano.a(lib_a-memcmp.o)
                0x000000000002b5b4                memcmp
 .text.memcpy   0x000000000002b5d0       0x1c /usr/local/bin/../lib/gcc/arm-none-eabi/8.3.1/../../../../arm-none-eabi/lib/thumb/v7e-m+fp/hard/libc_nano.a(lib_a-memcpy-stub.o)
                0x000000000002b5d0                memcpy
 .text.snprintf
                0x000000000002b5ec       0x68 /usr/local/bin/../lib/gcc/arm-none-eabi/8.3.1/../../../../arm-none-eabi/lib/thumb/v7e-m+fp/hard/libc_nano.a(lib_a-snprintf.o)
                0x000000000002b5ec                snprintf
                0x000000000002b5ec                sniprintf
 .text.strcpy   0x000000000002b654       0x10 /usr/local/bin/../lib/gcc/arm-none-eabi/8.3.1/../../../../arm-none-eabi/lib/thumb/v7e-m+fp/hard/libc_nano.a(lib_a-strcpy.o)
                0x000000000002b654                strcpy
 .text          0x000000000002b664       0x10 /usr/local/bin/../lib/gcc/arm-none-eabi/8.3.1/../../../../arm-none-eabi/lib/thumb/v7e-m+fp/hard/libc_nano.a(lib_a-strlen.o)
                0x000000000002b664                strlen
 .text.__ssputs_r
                0x000000000002b674       0xb6 /usr/local/bin/../lib/gcc/arm-none-eabi/8.3.1/../../../../arm-none-eabi/lib/thumb/v7e-m+fp/hard/libc_nano.a(lib_a-nano-svfprintf.o)
                0x000000000002b674                __ssputs_r
 *fill*         0x000000000002b72a        0x2 
 .text._svfprintf_r
                0x000000000002b72c      0x1f0 /usr/local/bin/../lib/gcc/arm-none-eabi/8.3.1/../../../../arm-none-eabi/lib/thumb/v7e-m+fp/hard/libc_nano.a(lib_a-nano-svfprintf.o)
                0x000000000002b72c                _svfprintf_r
                0x000000000002b72c                _svfiprintf_r
 .text._printf_common
                0x000000000002b91c       0xea /usr/local/bin/../lib/gcc/arm-none-eabi/8.3.1/../../../../arm-none-eabi/lib/thumb/v7e-m+fp/hard/libc_nano.a(lib_a-nano-vfprintf_i.o)
                0x000000000002b91c                _printf_common
 *fill*         0x000000000002ba06        0x2 
 .text._printf_i
                0x000000000002ba08      0x228 /usr/local/bin/../lib/gcc/arm-none-eabi/8.3.1/../../../../arm-none-eabi/lib/thumb/v7e-m+fp/hard/libc_nano.a(lib_a-nano-vfprintf_i.o)
                0x000000000002ba08                _printf_i
 .text          0x000000000002bc30       0xa0 /usr/local/bin/../lib/gcc/arm-none-eabi/8.3.1/../../../../arm-none-eabi/lib/thumb/v7e-m+fp/hard/libc_nano.a(lib_a-memchr.o)
                0x000000000002bc30                memchr
 .text.memmove  0x000000000002bcd0       0x34 /usr/local/bin/../lib/gcc/arm-none-eabi/8.3.1/../../../../arm-none-eabi/lib/thumb/v7e-m+fp/hard/libc_nano.a(lib_a-memmove.o)
                0x000000000002bcd0                memmove
 .text._free_r  0x000000000002bd04       0x9c /usr/local/bin/../lib/gcc/arm-none-eabi/8.3.1/../../../../arm-none-eabi/lib/thumb/v7e-m+fp/hard/libc_nano.a(lib_a-nano-freer.o)
                0x000000000002bd04                _free_r
 .text._malloc_r
                0x000000000002bda0       0xb4 /usr/local/bin/../lib/gcc/arm-none-eabi/8.3.1/../../../../arm-none-eabi/lib/thumb/v7e-m+fp/hard/libc_nano.a(lib_a-nano-mallocr.o)
                0x000000000002bda0                _malloc_r
 .text._realloc_r
                0x000000000002be54       0x4c /usr/local/bin/../lib/gcc/arm-none-eabi/8.3.1/../../../../arm-none-eabi/lib/thumb/v7e-m+fp/hard/libc_nano.a(lib_a-nano-reallocr.o)
                0x000000000002be54                _realloc_r
 .text._sbrk_r  0x000000000002bea0       0x20 /usr/local/bin/../lib/gcc/arm-none-eabi/8.3.1/../../../../arm-none-eabi/lib/thumb/v7e-m+fp/hard/libc_nano.a(lib_a-sbrkr.o)
                0x000000000002bea0                _sbrk_r
 .text.__malloc_lock
                0x000000000002bec0        0xc /usr/local/bin/../lib/gcc/arm-none-eabi/8.3.1/../../../../arm-none-eabi/lib/thumb/v7e-m+fp/hard/libc_nano.a(lib_a-mlock.o)
                0x000000000002bec0                __malloc_lock
 .text.__malloc_unlock
                0x000000000002becc        0xc /usr/local/bin/../lib/gcc/arm-none-eabi/8.3.1/../../../../arm-none-eabi/lib/thumb/v7e-m+fp/hard/libc_nano.a(lib_a-mlock.o)
                0x000000000002becc                __malloc_unlock
 .text._malloc_usable_size_r
                0x000000000002bed8       0x10 /usr/local/bin/../lib/gcc/arm-none-eabi/8.3.1/../../../../arm-none-eabi/lib/thumb/v7e-m+fp/hard/libc_nano.a(lib_a-nano-msizer.o)
                0x000000000002bed8                _malloc_usable_size_r
 .text.__retarget_lock_acquire_recursive
                0x000000000002bee8        0x2 /usr/local/bin/../lib/gcc/arm-none-eabi/8.3.1/../../../../arm-none-eabi/lib/thumb/v7e-m+fp/hard/libc_nano.a(lib_a-lock.o)
                0x000000000002bee8                __retarget_lock_acquire_recursive
 .text.__retarget_lock_release_recursive
                0x000000000002beea        0x2 /usr/local/bin/../lib/gcc/arm-none-eabi/8.3.1/../../../../arm-none-eabi/lib/thumb/v7e-m+fp/hard/libc_nano.a(lib_a-lock.o)
                0x000000000002beea                __retarget_lock_release_recursive
 .text._sbrk    0x000000000002beec       0x1c /usr/local/bin/../lib/gcc/arm-none-eabi/8.3.1/../../../../arm-none-eabi/lib/thumb/v7e-m+fp/hard/libnosys.a(sbrk.o)
                0x000000000002beec                _sbrk
 *(.init)
 .init          0x000000000002bf08        0x4 /usr/local/bin/../lib/gcc/arm-none-eabi/8.3.1/thumb/v7e-m+fp/hard/crti.o
                0x000000000002bf08                _init
 .init          0x000000000002bf0c        0x8 /usr/local/bin/../lib/gcc/arm-none-eabi/8.3.1/thumb/v7e-m+fp/hard/crtn.o
 *(.fini)
 .fini          0x000000000002bf14        0x4 /usr/local/bin/../lib/gcc/arm-none-eabi/8.3.1/thumb/v7e-m+fp/hard/crti.o
                0x000000000002bf14                _fini
 .fini          0x000000000002bf18        0x8 /usr/local/bin/../lib/gcc/arm-none-eabi/8.3.1/thumb/v7e-m+fp/hard/crtn.o
 *crtbegin.o(.ctors)
 *crtbegin?.o(.ctors)
 *(EXCLUDE_FILE(*crtend.o *crtend?.o) .ctors)
 *(SORT_BY_NAME(.ctors.*))
 *(.ctors)
 *crtbegin.o(.dtors)
 *crtbegin?.o(.dtors)
 *(EXCLUDE_FILE(*crtend.o *crtend?.o) .dtors)
 *(SORT_BY_NAME(.dtors.*))
 *(.dtors)
 *(.rodata*)
 .rodata._global_impure_ptr
                0x000000000002bf20        0x4 /usr/local/bin/../lib/gcc/arm-none-eabi/8.3.1/../../../../arm-none-eabi/lib/thumb/v7e-m+fp/hard/libc_nano.a(lib_a-impure.o)
                0x000000000002bf20                _global_impure_ptr
 .rodata.main.str1.4
                0x000000000002bf24      0x16c _build/nrf52832_xxaa_main.c.o
 .rodata        0x000000000002c090        0x4 _build/nrf52832_xxaa_ble_init.c.o
 .rodata.advertising_start.str1.4
                0x000000000002c094       0x39 _build/nrf52832_xxaa_ble_init.c.o
 *fill*         0x000000000002c0cd        0x3 
 .rodata.ble_evt_dispatch.str1.4
                0x000000000002c0d0       0xcd _build/nrf52832_xxaa_ble_init.c.o
 *fill*         0x000000000002c19d        0x3 
 .rodata.init_BLE.str1.4
                0x000000000002c1a0      0x610 _build/nrf52832_xxaa_ble_init.c.o
 .rodata.on_adv_evt.str1.4
                0x000000000002c7b0       0x42 _build/nrf52832_xxaa_ble_init.c.o
 *fill*         0x000000000002c7f2        0x2 
 .rodata.on_conn_params_evt.str1.4
                0x000000000002c7f4       0x3a _build/nrf52832_xxaa_ble_init.c.o
 *fill*         0x000000000002c82e        0x2 
 .rodata.pm_evt_handler.str1.4
                0x000000000002c830      0x247 _build/nrf52832_xxaa_ble_init.c.o
 *fill*         0x000000000002ca77        0x1 
 .rodata        0x000000000002ca78       0x12 _build/nrf52832_xxaa_ble_lcs.c.o
 *fill*         0x000000000002ca8a        0x2 
 .rodata.ble_lcs_data_handler.str1.4
                0x000000000002ca8c       0x4f _build/nrf52832_xxaa_ble_lcs.c.o
 *fill*         0x000000000002cadb        0x1 
 .rodata.ble_lcs_init.str1.4
                0x000000000002cadc       0x3b _build/nrf52832_xxaa_ble_lcs.c.o
 *fill*         0x000000000002cb17        0x1 
 .rodata        0x000000000002cb18       0x10 _build/nrf52832_xxaa_ble_ics.c.o
 .rodata.ble_ics_data_handler.str1.4
                0x000000000002cb28       0x29 _build/nrf52832_xxaa_ble_ics.c.o
 *fill*         0x000000000002cb51        0x3 
 .rodata.ble_ics_init.str1.4
                0x000000000002cb54       0xee _build/nrf52832_xxaa_ble_ics.c.o
 *fill*         0x000000000002cc42        0x2 
 .rodata        0x000000000002cc44       0x10 _build/nrf52832_xxaa_ble_tcs.c.o
 .rodata.ble_tcs_init.str1.4
                0x000000000002cc54      0x223 _build/nrf52832_xxaa_ble_tcs.c.o
 *fill*         0x000000000002ce77        0x1 
 .rodata.ble_tcs_on_ble_evt.str1.4
                0x000000000002ce78      0x26f _build/nrf52832_xxaa_ble_tcs.c.o
 *fill*         0x000000000002d0e7        0x1 
 .rodata        0x000000000002d0e8       0x10 _build/nrf52832_xxaa_ble_scs.c.o
 .rodata.ble_scs_init.str1.4
                0x000000000002d0f8       0xfe _build/nrf52832_xxaa_ble_scs.c.o
 *fill*         0x000000000002d1f6        0x2 
 .rodata        0x000000000002d1f8        0x7 _build/nrf52832_xxaa_print.c.o
 *fill*         0x000000000002d1ff        0x1 
 .rodata.print_double.str1.4
                0x000000000002d200        0x4 _build/nrf52832_xxaa_print.c.o
 .rodata.flash_sys_event_handler.str1.4
                0x000000000002d204       0x7b _build/nrf52832_xxaa_flash.c.o
 *fill*         0x000000000002d27f        0x1 
 .rodata.update_step_count.str1.4
                0x000000000002d280       0x30 _build/nrf52832_xxaa_step_count_db.c.o
 .rodata.nrf_log_backend_serial_std_handler.str1.4
                0x000000000002d2b0        0x7 _build/nrf52832_xxaa_nrf_log_backend_serial.c.o
 *fill*         0x000000000002d2b7        0x1 
 .rodata.nrf_log_frontend_std_0.str1.4
                0x000000000002d2b8        0xb _build/nrf52832_xxaa_nrf_log_frontend.c.o
 *fill*         0x000000000002d2c3        0x1 
 .rodata.app_error_fault_handler.str1.4
                0x000000000002d2c4       0x29 _build/nrf52832_xxaa_app_error_weak.c.o
 *fill*         0x000000000002d2ed        0x3 
 .rodata.m_fds_tl_dirty
                0x000000000002d2f0        0x4 _build/nrf52832_xxaa_fds.c.o
 .rodata.page_tag_data.8846
                0x000000000002d2f4        0x8 _build/nrf52832_xxaa_fds.c.o
 .rodata.page_tag_swap.8842
                0x000000000002d2fc        0x8 _build/nrf52832_xxaa_fds.c.o
 .rodata.SEGGER_RTT_ReadNoLock.str1.4
                0x000000000002d304       0x17 _build/nrf52832_xxaa_SEGGER_RTT.c.o
 *fill*         0x000000000002d31b        0x1 
 .rodata.m_conn_params_timer_id
                0x000000000002d31c        0x4 _build/nrf52832_xxaa_ble_conn_params.c.o
 .rodata        0x000000000002d320       0x10 _build/nrf52832_xxaa_gatts_cache_manager.c.o
 .rodata.service_changed_pending.9815
                0x000000000002d330        0x4 _build/nrf52832_xxaa_gatts_cache_manager.c.o
 .rodata.service_changed_pending.9878
                0x000000000002d334        0x4 _build/nrf52832_xxaa_gatts_cache_manager.c.o
 .rodata.nrf_ble_gatt_on_ble_evt.str1.4
                0x000000000002d338      0x185 _build/nrf52832_xxaa_nrf_ble_gatt.c.o
 *fill*         0x000000000002d4bd        0x3 
 .rodata.CSWTCH.10
                0x000000000002d4c0       0x28 _build/nrf52832_xxaa_peer_data_storage.c.o
 .rodata.m_evt_handlers
                0x000000000002d4e8       0x14 _build/nrf52832_xxaa_peer_database.c.o
 .rodata.softdevice_enable.str1.4
                0x000000000002d4fc       0xa8 _build/nrf52832_xxaa_softdevice_handler.c.o
                                         0xa5 (size before relaxing)
 .rodata._ctype_
                0x000000000002d5a4      0x101 /usr/local/bin/../lib/gcc/arm-none-eabi/8.3.1/../../../../arm-none-eabi/lib/thumb/v7e-m+fp/hard/libc_nano.a(lib_a-ctype_.o)
                0x000000000002d5a4                _ctype_
 .rodata._svfprintf_r.str1.1
                0x000000000002d6a5       0x11 /usr/local/bin/../lib/gcc/arm-none-eabi/8.3.1/../../../../arm-none-eabi/lib/thumb/v7e-m+fp/hard/libc_nano.a(lib_a-nano-svfprintf.o)
 .rodata._printf_i.str1.1
                0x000000000002d6b6       0x22 /usr/local/bin/../lib/gcc/arm-none-eabi/8.3.1/../../../../arm-none-eabi/lib/thumb/v7e-m+fp/hard/libc_nano.a(lib_a-nano-vfprintf_i.o)
 *(.eh_frame*)
 .eh_frame      0x000000000002d6d8        0x0 /usr/local/bin/../lib/gcc/arm-none-eabi/8.3.1/thumb/v7e-m+fp/hard/crtbegin.o
 .eh_frame      0x000000000002d6d8        0x4 /usr/local/bin/../lib/gcc/arm-none-eabi/8.3.1/thumb/v7e-m+fp/hard/crtend.o

.glue_7         0x000000000002d6dc        0x0
 .glue_7        0x000000000002d6dc        0x0 linker stubs

.glue_7t        0x000000000002d6dc        0x0
 .glue_7t       0x000000000002d6dc        0x0 linker stubs

.vfp11_veneer   0x000000000002d6dc        0x0
 .vfp11_veneer  0x000000000002d6dc        0x0 linker stubs

.v4_bx          0x000000000002d6dc        0x0
 .v4_bx         0x000000000002d6dc        0x0 linker stubs

.iplt           0x000000000002d6dc        0x0
 .iplt          0x000000000002d6dc        0x0 /usr/local/bin/../lib/gcc/arm-none-eabi/8.3.1/thumb/v7e-m+fp/hard/crtbegin.o

.pwr_mgmt_data  0x000000000002d6dc        0x0
                [!provide]                        PROVIDE (__start_pwr_mgmt_data = .)
 *(SORT_BY_NAME(.pwr_mgmt_data*))
                [!provide]                        PROVIDE (__stop_pwr_mgmt_data = .)

.ARM.extab
 *(.ARM.extab* .gnu.linkonce.armextab.*)
                0x000000000002d6dc                __exidx_start = .

.ARM.exidx      0x000000000002d6dc        0x8
 *(.ARM.exidx* .gnu.linkonce.armexidx.*)
 .ARM.exidx     0x000000000002d6dc        0x8 /usr/local/bin/../lib/gcc/arm-none-eabi/8.3.1/../../../../arm-none-eabi/lib/thumb/v7e-m+fp/hard/crt0.o
                0x000000000002d6e4                __exidx_end = .
                0x000000000002d6e4                __etext = .

.rel.dyn        0x000000000002d6e4        0x0
 .rel.iplt      0x000000000002d6e4        0x0 /usr/local/bin/../lib/gcc/arm-none-eabi/8.3.1/thumb/v7e-m+fp/hard/crtbegin.o

.data           0x0000000020002260       0x7c load address 0x000000000002d6e4
                0x0000000020002260                __data_start__ = .
 *(vtable)
 *(.data*)
 .data._impure_ptr
                0x0000000020002260        0x4 /usr/local/bin/../lib/gcc/arm-none-eabi/8.3.1/../../../../arm-none-eabi/lib/thumb/v7e-m+fp/hard/libc_nano.a(lib_a-impure.o)
                0x0000000020002260                _impure_ptr
 .data.impure_data
                0x0000000020002264       0x60 /usr/local/bin/../lib/gcc/arm-none-eabi/8.3.1/../../../../arm-none-eabi/lib/thumb/v7e-m+fp/hard/libc_nano.a(lib_a-impure.o)
 .data.m_conn_handle
                0x00000000200022c4        0x2 _build/nrf52832_xxaa_ble_init.c.o
                0x00000000200022c4                m_conn_handle
 .data.m_flag_sec_proc
                0x00000000200022c6        0x1 _build/nrf52832_xxaa_security_dispatcher.c.o
 .data.m_flag_sec_proc_new_peer
                0x00000000200022c7        0x1 _build/nrf52832_xxaa_security_dispatcher.c.o
 .data.m_flag_sec_proc_pairing
                0x00000000200022c8        0x1 _build/nrf52832_xxaa_security_dispatcher.c.o
 .data.m_flag_link_secure_force_repairing
                0x00000000200022c9        0x1 _build/nrf52832_xxaa_security_manager.c.o
 .data.m_flag_link_secure_null_params
                0x00000000200022ca        0x1 _build/nrf52832_xxaa_security_manager.c.o
 .data.m_flag_link_secure_pending_busy
                0x00000000200022cb        0x1 _build/nrf52832_xxaa_security_manager.c.o
 .data.m_flag_link_secure_pending_flash_full
                0x00000000200022cc        0x1 _build/nrf52832_xxaa_security_manager.c.o
 .data.m_flag_params_reply_pending_busy
                0x00000000200022cd        0x1 _build/nrf52832_xxaa_security_manager.c.o
 .data.m_flag_params_reply_pending_flash_full
                0x00000000200022ce        0x1 _build/nrf52832_xxaa_security_manager.c.o
 .data.m_flag_reject_pairing
                0x00000000200022cf        0x1 _build/nrf52832_xxaa_security_manager.c.o
 .data.SystemCoreClock
                0x00000000200022d0        0x4 _build/nrf52832_xxaa_system_nrf52.c.o
                0x00000000200022d0                SystemCoreClock
                0x00000000200022d4                . = ALIGN (0x4)
                0x00000000200022d4                PROVIDE (__preinit_array_start = .)
 *(.preinit_array)
                0x00000000200022d4                PROVIDE (__preinit_array_end = .)
                0x00000000200022d4                . = ALIGN (0x4)
                0x00000000200022d4                PROVIDE (__init_array_start = .)
 *(SORT_BY_NAME(.init_array.*))
 *(.init_array)
 .init_array    0x00000000200022d4        0x4 /usr/local/bin/../lib/gcc/arm-none-eabi/8.3.1/thumb/v7e-m+fp/hard/crtbegin.o
                0x00000000200022d8                PROVIDE (__init_array_end = .)
                0x00000000200022d8                . = ALIGN (0x4)
                [!provide]                        PROVIDE (__fini_array_start = .)
 *(SORT_BY_NAME(.fini_array.*))
 *(.fini_array)
 .fini_array    0x00000000200022d8        0x4 /usr/local/bin/../lib/gcc/arm-none-eabi/8.3.1/thumb/v7e-m+fp/hard/crtbegin.o
                [!provide]                        PROVIDE (__fini_array_end = .)
 *(.jcr*)
                0x00000000200022dc                . = ALIGN (0x4)
                0x00000000200022dc                __data_end__ = .
LOAD /usr/local/bin/../lib/gcc/arm-none-eabi/8.3.1/thumb/v7e-m+fp/hard/crti.o
LOAD /usr/local/bin/../lib/gcc/arm-none-eabi/8.3.1/thumb/v7e-m+fp/hard/crtbegin.o
LOAD /usr/local/bin/../lib/gcc/arm-none-eabi/8.3.1/../../../../arm-none-eabi/lib/thumb/v7e-m+fp/hard/crt0.o
LOAD /usr/local/bin/../lib/gcc/arm-none-eabi/8.3.1/../../../../arm-none-eabi/lib/thumb/v7e-m+fp/hard/libc_nano.a
LOAD /usr/local/bin/../lib/gcc/arm-none-eabi/8.3.1/../../../../arm-none-eabi/lib/thumb/v7e-m+fp/hard/libnosys.a
LOAD _build/nrf52832_xxaa_main.c.o
LOAD _build/nrf52832_xxaa_ble_init.c.o
LOAD _build/nrf52832_xxaa_ble_lcs.c.o
LOAD _build/nrf52832_xxaa_ble_ics.c.o
LOAD _build/nrf52832_xxaa_ble_tcs.c.o
LOAD _build/nrf52832_xxaa_ble_scs.c.o
LOAD _build/nrf52832_xxaa_gpio.c.o
LOAD _build/nrf52832_xxaa_uart.c.o
LOAD _build/nrf52832_xxaa_print.c.o
LOAD _build/nrf52832_xxaa_spim.c.o
LOAD _build/nrf52832_xxaa_stm_communication.c.o
LOAD _build/nrf52832_xxaa_flash.c.o
LOAD _build/nrf52832_xxaa_step_count_db.c.o
LOAD _build/nrf52832_xxaa_rtc.c.o
LOAD _build/nrf52832_xxaa_nrf_log_backend_serial.c.o
LOAD _build/nrf52832_xxaa_nrf_log_frontend.c.o
LOAD _build/nrf52832_xxaa_app_button.c.o
LOAD _build/nrf52832_xxaa_app_error.c.o
LOAD _build/nrf52832_xxaa_app_error_weak.c.o
LOAD _build/nrf52832_xxaa_app_scheduler.c.o
LOAD _build/nrf52832_xxaa_app_timer.c.o
LOAD _build/nrf52832_xxaa_app_util_platform.c.o
LOAD _build/nrf52832_xxaa_crc16.c.o
LOAD _build/nrf52832_xxaa_fds.c.o
LOAD _build/nrf52832_xxaa_fstorage.c.o
LOAD _build/nrf52832_xxaa_hardfault_implementation.c.o
LOAD _build/nrf52832_xxaa_nrf_assert.c.o
LOAD _build/nrf52832_xxaa_nrf_strerror.c.o
LOAD _build/nrf52832_xxaa_sdk_mapped_flags.c.o
LOAD _build/nrf52832_xxaa_sensorsim.c.o
LOAD _build/nrf52832_xxaa_boards.c.o
LOAD _build/nrf52832_xxaa_nrf_drv_clock.c.o
LOAD _build/nrf52832_xxaa_nrf_drv_common.c.o
LOAD _build/nrf52832_xxaa_nrf_drv_gpiote.c.o
LOAD _build/nrf52832_xxaa_nrf_drv_uart.c.o
LOAD _build/nrf52832_xxaa_bsp.c.o
LOAD _build/nrf52832_xxaa_bsp_btn_ble.c.o
LOAD _build/nrf52832_xxaa_bsp_nfc.c.o
LOAD _build/nrf52832_xxaa_RTT_Syscalls_GCC.c.o
LOAD _build/nrf52832_xxaa_SEGGER_RTT.c.o
LOAD _build/nrf52832_xxaa_SEGGER_RTT_printf.c.o
LOAD _build/nrf52832_xxaa_ble_advdata.c.o
LOAD _build/nrf52832_xxaa_ble_advertising.c.o
LOAD _build/nrf52832_xxaa_ble_conn_params.c.o
LOAD _build/nrf52832_xxaa_ble_conn_state.c.o
LOAD _build/nrf52832_xxaa_ble_srv_common.c.o
LOAD _build/nrf52832_xxaa_gatt_cache_manager.c.o
LOAD _build/nrf52832_xxaa_gatts_cache_manager.c.o
LOAD _build/nrf52832_xxaa_id_manager.c.o
LOAD _build/nrf52832_xxaa_nrf_ble_gatt.c.o
LOAD _build/nrf52832_xxaa_peer_data_storage.c.o
LOAD _build/nrf52832_xxaa_peer_database.c.o
LOAD _build/nrf52832_xxaa_peer_id.c.o
LOAD _build/nrf52832_xxaa_peer_manager.c.o
LOAD _build/nrf52832_xxaa_pm_buffer.c.o
LOAD _build/nrf52832_xxaa_pm_mutex.c.o
LOAD _build/nrf52832_xxaa_security_dispatcher.c.o
LOAD _build/nrf52832_xxaa_security_manager.c.o
LOAD _build/nrf52832_xxaa_gcc_startup_nrf52.S.o
LOAD _build/nrf52832_xxaa_system_nrf52.c.o
LOAD _build/nrf52832_xxaa_softdevice_handler.c.o
LOAD /usr/local/bin/../lib/gcc/arm-none-eabi/8.3.1/../../../../arm-none-eabi/lib/thumb/v7e-m+fp/hard/libm.a
START GROUP
LOAD /usr/local/bin/../lib/gcc/arm-none-eabi/8.3.1/thumb/v7e-m+fp/hard/libgcc.a
LOAD /usr/local/bin/../lib/gcc/arm-none-eabi/8.3.1/../../../../arm-none-eabi/lib/thumb/v7e-m+fp/hard/libc_nano.a
END GROUP
START GROUP
LOAD /usr/local/bin/../lib/gcc/arm-none-eabi/8.3.1/thumb/v7e-m+fp/hard/libgcc.a
LOAD /usr/local/bin/../lib/gcc/arm-none-eabi/8.3.1/../../../../arm-none-eabi/lib/thumb/v7e-m+fp/hard/libc_nano.a
END GROUP
LOAD /usr/local/bin/../lib/gcc/arm-none-eabi/8.3.1/thumb/v7e-m+fp/hard/crtend.o
LOAD /usr/local/bin/../lib/gcc/arm-none-eabi/8.3.1/thumb/v7e-m+fp/hard/crtn.o
START GROUP
LOAD /usr/local/bin/../lib/gcc/arm-none-eabi/8.3.1/thumb/v7e-m+fp/hard/libgcc.a
LOAD /usr/local/bin/../lib/gcc/arm-none-eabi/8.3.1/../../../../arm-none-eabi/lib/thumb/v7e-m+fp/hard/libc.a
LOAD /usr/local/bin/../lib/gcc/arm-none-eabi/8.3.1/../../../../arm-none-eabi/lib/thumb/v7e-m+fp/hard/libnosys.a
END GROUP

.igot.plt       0x00000000200022dc        0x0 load address 0x000000000002d760
 .igot.plt      0x00000000200022dc        0x0 /usr/local/bin/../lib/gcc/arm-none-eabi/8.3.1/thumb/v7e-m+fp/hard/crtbegin.o

.step_count_flash
                0x000000000007c000     0x3000
                0x000000000007c000                . = ALIGN (0x8)
                0x000000000007c000                _step_count_flash_start = .
 *(.step_count_flash)
 .step_count_flash
                0x000000000007c000     0x3000 _build/nrf52832_xxaa_flash.c.o
                0x000000000007c000                step_count_flash
                0x000000000007f000                . = ALIGN (0x8)
                0x000000000007f000                _step_count_flash_end = .

.user_info_flash
                0x000000000007f000        0x0
                0x000000000007f000                . = ALIGN (0x8)
                0x000000000007f000                _user_info_flash_start = .
 *(.user_info_flash)
                0x000000000007f000                . = ALIGN (0x8)
                0x000000000007f000                _user_info_flash_end = .

.fs_data        0x00000000200022dc       0x10 load address 0x000000000002d760
                0x00000000200022dc                PROVIDE (__start_fs_data = .)
 *(.fs_data)
 .fs_data       0x00000000200022dc       0x10 _build/nrf52832_xxaa_fds.c.o
                0x00000000200022ec                PROVIDE (__stop_fs_data = .)

.bss            0x00000000200022f0     0x123c load address 0x000000000002d778
                0x00000000200022f0                . = ALIGN (0x4)
                0x00000000200022f0                __bss_start__ = .
 *(.bss*)
 .bss           0x00000000200022f0       0x1c /usr/local/bin/../lib/gcc/arm-none-eabi/8.3.1/thumb/v7e-m+fp/hard/crtbegin.o
 .bss.RTC2_flag
                0x000000002000230c        0x1 _build/nrf52832_xxaa_main.c.o
                0x000000002000230c                RTC2_flag
 *fill*         0x000000002000230d        0x3 
 .bss.step_count
                0x0000000020002310        0x4 _build/nrf52832_xxaa_main.c.o
                0x0000000020002310                step_count
 .bss.BLE_EVT_BUFFER.11488
                0x0000000020002314       0x50 _build/nrf52832_xxaa_ble_init.c.o
 .bss.m_adv_uuids
                0x0000000020002364        0x0 _build/nrf52832_xxaa_ble_init.c.o
                0x0000000020002364                m_adv_uuids
 .bss.is_LED_init.9850
                0x0000000020002364        0x1 _build/nrf52832_xxaa_ble_lcs.c.o
 .bss.STMcommunication_cs_pin
                0x0000000020002365        0x1 _build/nrf52832_xxaa_stm_communication.c.o
 .bss.flash_state_
                0x0000000020002366        0x1 _build/nrf52832_xxaa_flash.c.o
                0x0000000020002366                flash_state_
 *fill*         0x0000000020002367        0x1 
 .bss.RTC2_IRQ_callback_
                0x0000000020002368        0x4 _build/nrf52832_xxaa_rtc.c.o
 .bss.m_blocking_mode
                0x000000002000236c        0x1 _build/nrf52832_xxaa_nrf_log_backend_serial.c.o
 .bss.m_initialized
                0x000000002000236d        0x1 _build/nrf52832_xxaa_nrf_log_backend_serial.c.o
 *fill*         0x000000002000236e        0x2 
 .bss.m_log_data
                0x0000000020002370      0x418 _build/nrf52832_xxaa_nrf_log_frontend.c.o
 .bss.m_op_queue
                0x0000000020002788      0x10c _build/nrf52832_xxaa_app_timer.c.o
 .bss.m_rtc1_reset
                0x0000000020002894        0x1 _build/nrf52832_xxaa_app_timer.c.o
 .bss.m_rtc1_running
                0x0000000020002895        0x1 _build/nrf52832_xxaa_app_timer.c.o
 *fill*         0x0000000020002896        0x2 
 .bss.m_ticks_elapsed
                0x0000000020002898        0x8 _build/nrf52832_xxaa_app_timer.c.o
 .bss.m_ticks_elapsed_q_read_ind
                0x00000000200028a0        0x1 _build/nrf52832_xxaa_app_timer.c.o
 .bss.m_ticks_elapsed_q_write_ind
                0x00000000200028a1        0x1 _build/nrf52832_xxaa_app_timer.c.o
 *fill*         0x00000000200028a2        0x2 
 .bss.m_ticks_latest
                0x00000000200028a4        0x4 _build/nrf52832_xxaa_app_timer.c.o
 .bss.mp_timer_id_head
                0x00000000200028a8        0x4 _build/nrf52832_xxaa_app_timer.c.o
 .bss.desc.9075
                0x00000000200028ac        0xc _build/nrf52832_xxaa_fds.c.o
 .bss.m_cb_table
                0x00000000200028b8       0x20 _build/nrf52832_xxaa_fds.c.o
 .bss.m_chunk_queue
                0x00000000200028d8       0x48 _build/nrf52832_xxaa_fds.c.o
 .bss.m_flags   0x0000000020002920        0x1 _build/nrf52832_xxaa_fds.c.o
 *fill*         0x0000000020002921        0x3 
 .bss.m_gc      0x0000000020002924       0x10 _build/nrf52832_xxaa_fds.c.o
 .bss.m_latest_rec_id
                0x0000000020002934        0x4 _build/nrf52832_xxaa_fds.c.o
 .bss.m_op_queue
                0x0000000020002938       0x78 _build/nrf52832_xxaa_fds.c.o
 .bss.m_pages   0x00000000200029b0       0x20 _build/nrf52832_xxaa_fds.c.o
 .bss.m_swap_page
                0x00000000200029d0        0x8 _build/nrf52832_xxaa_fds.c.o
 .bss.m_users   0x00000000200029d8        0x1 _build/nrf52832_xxaa_fds.c.o
 *fill*         0x00000000200029d9        0x1 
 .bss.page.9076
                0x00000000200029da        0x2 _build/nrf52832_xxaa_fds.c.o
 .bss.tok.8981  0x00000000200029dc        0x8 _build/nrf52832_xxaa_fds.c.o
 .bss.m_flags   0x00000000200029e4        0x1 _build/nrf52832_xxaa_fstorage.c.o
 *fill*         0x00000000200029e5        0x3 
 .bss.m_queue   0x00000000200029e8       0x68 _build/nrf52832_xxaa_fstorage.c.o
 .bss.m_retry_count
                0x0000000020002a50        0x1 _build/nrf52832_xxaa_fstorage.c.o
 *fill*         0x0000000020002a51        0x3 
 .bss.m_clock_cb
                0x0000000020002a54       0x14 _build/nrf52832_xxaa_nrf_drv_clock.c.o
 .bss.m_cb      0x0000000020002a68       0x58 _build/nrf52832_xxaa_nrf_drv_gpiote.c.o
 .bss.m_cb      0x0000000020002ac0       0x20 _build/nrf52832_xxaa_nrf_drv_uart.c.o
 .bss._acDownBuffer
                0x0000000020002ae0       0x10 _build/nrf52832_xxaa_SEGGER_RTT.c.o
 .bss._acUpBuffer
                0x0000000020002af0      0x200 _build/nrf52832_xxaa_SEGGER_RTT.c.o
 .bss.m_adv_evt
                0x0000000020002cf0        0x1 _build/nrf52832_xxaa_ble_advertising.c.o
 .bss.m_adv_mode_current
                0x0000000020002cf1        0x1 _build/nrf52832_xxaa_ble_advertising.c.o
 *fill*         0x0000000020002cf2        0x2 
 .bss.m_adv_modes_config
                0x0000000020002cf4       0x20 _build/nrf52832_xxaa_ble_advertising.c.o
 .bss.m_advdata
                0x0000000020002d14       0x3c _build/nrf52832_xxaa_ble_advertising.c.o
 .bss.m_advertising_start_pending
                0x0000000020002d50        0x1 _build/nrf52832_xxaa_ble_advertising.c.o
 .bss.m_conn_cfg_tag
                0x0000000020002d51        0x1 _build/nrf52832_xxaa_ble_advertising.c.o
 .bss.m_current_slave_link_conn_handle
                0x0000000020002d52        0x2 _build/nrf52832_xxaa_ble_advertising.c.o
 .bss.m_error_handler
                0x0000000020002d54        0x4 _build/nrf52832_xxaa_ble_advertising.c.o
 .bss.m_evt_handler
                0x0000000020002d58        0x4 _build/nrf52832_xxaa_ble_advertising.c.o
 .bss.m_initialized
                0x0000000020002d5c        0x1 _build/nrf52832_xxaa_ble_advertising.c.o
 *fill*         0x0000000020002d5d        0x3 
 .bss.m_manuf_data_array
                0x0000000020002d60       0x1f _build/nrf52832_xxaa_ble_advertising.c.o
 *fill*         0x0000000020002d7f        0x1 
 .bss.m_manuf_specific_data
                0x0000000020002d80        0xc _build/nrf52832_xxaa_ble_advertising.c.o
 .bss.m_peer_addr_reply_expected
                0x0000000020002d8c        0x1 _build/nrf52832_xxaa_ble_advertising.c.o
 *fill*         0x0000000020002d8d        0x3 
 .bss.m_peer_address
                0x0000000020002d90        0x7 _build/nrf52832_xxaa_ble_advertising.c.o
 *fill*         0x0000000020002d97        0x1 
 .bss.m_service_data
                0x0000000020002d98        0xc _build/nrf52832_xxaa_ble_advertising.c.o
 .bss.m_service_data_array
                0x0000000020002da4       0x1f _build/nrf52832_xxaa_ble_advertising.c.o
 *fill*         0x0000000020002dc3        0x1 
 .bss.m_slave_conn_int
                0x0000000020002dc4        0x4 _build/nrf52832_xxaa_ble_advertising.c.o
 .bss.m_whitelist_in_use
                0x0000000020002dc8        0x1 _build/nrf52832_xxaa_ble_advertising.c.o
 .bss.m_whitelist_reply_expected
                0x0000000020002dc9        0x1 _build/nrf52832_xxaa_ble_advertising.c.o
 .bss.m_whitelist_temporarily_disabled
                0x0000000020002dca        0x1 _build/nrf52832_xxaa_ble_advertising.c.o
 .bss.m_change_param
                0x0000000020002dcb        0x1 _build/nrf52832_xxaa_ble_conn_params.c.o
 .bss.m_conn_handle
                0x0000000020002dcc        0x2 _build/nrf52832_xxaa_ble_conn_params.c.o
 *fill*         0x0000000020002dce        0x2 
 .bss.m_conn_params_config
                0x0000000020002dd0       0x1c _build/nrf52832_xxaa_ble_conn_params.c.o
 .bss.m_conn_params_timer_id_data
                0x0000000020002dec       0x20 _build/nrf52832_xxaa_ble_conn_params.c.o
 .bss.m_current_conn_params
                0x0000000020002e0c        0x8 _build/nrf52832_xxaa_ble_conn_params.c.o
 .bss.m_preferred_conn_params
                0x0000000020002e14        0x8 _build/nrf52832_xxaa_ble_conn_params.c.o
 .bss.m_update_count
                0x0000000020002e1c        0x1 _build/nrf52832_xxaa_ble_conn_params.c.o
 *fill*         0x0000000020002e1d        0x3 
 .bss.m_bcs     0x0000000020002e20       0xb8 _build/nrf52832_xxaa_ble_conn_state.c.o
 .bss.m_flag_local_db_apply_pending
                0x0000000020002ed8        0x1 _build/nrf52832_xxaa_gatt_cache_manager.c.o
 .bss.m_flag_local_db_update_pending
                0x0000000020002ed9        0x1 _build/nrf52832_xxaa_gatt_cache_manager.c.o
 .bss.m_flag_service_changed_pending
                0x0000000020002eda        0x1 _build/nrf52832_xxaa_gatt_cache_manager.c.o
 .bss.m_flag_service_changed_sent
                0x0000000020002edb        0x1 _build/nrf52832_xxaa_gatt_cache_manager.c.o
 .bss.m_current_sc_store_peer_id
                0x0000000020002edc        0x2 _build/nrf52832_xxaa_gatts_cache_manager.c.o
 .bss.start_handle.9870
                0x0000000020002ede        0x2 _build/nrf52832_xxaa_gatts_cache_manager.c.o
 .bss.m_conn_state_user_flag_id
                0x0000000020002ee0        0x1 _build/nrf52832_xxaa_id_manager.c.o
 *fill*         0x0000000020002ee1        0x3 
 .bss.m_connections
                0x0000000020002ee4       0xf0 _build/nrf52832_xxaa_id_manager.c.o
 .bss.m_fds_ftok
                0x0000000020002fd4        0x8 _build/nrf52832_xxaa_peer_data_storage.c.o
 .bss.m_peer_delete_ongoing
                0x0000000020002fdc        0x1 _build/nrf52832_xxaa_peer_data_storage.c.o
 .bss.m_peer_delete_queued
                0x0000000020002fdd        0x1 _build/nrf52832_xxaa_peer_data_storage.c.o
 *fill*         0x0000000020002fde        0x2 
 .bss.buffer_memory.9892
                0x0000000020002fe0      0x280 _build/nrf52832_xxaa_peer_database.c.o
 .bss.m_n_writes
                0x0000000020003260        0x4 _build/nrf52832_xxaa_peer_database.c.o
 .bss.m_write_buffer
                0x0000000020003264       0x10 _build/nrf52832_xxaa_peer_database.c.o
 .bss.m_write_buffer_records
                0x0000000020003274       0xa0 _build/nrf52832_xxaa_peer_database.c.o
 .bss.mutex_memory.9893
                0x0000000020003314        0x1 _build/nrf52832_xxaa_peer_database.c.o
 *fill*         0x0000000020003315        0x3 
 .bss.m_pi      0x0000000020003318       0x40 _build/nrf52832_xxaa_peer_id.c.o
 .bss.m_bonding_flag_id
                0x0000000020003358        0x1 _build/nrf52832_xxaa_peer_manager.c.o
 *fill*         0x0000000020003359        0x3 
 .bss.m_current_highest_peer_rank
                0x000000002000335c        0x4 _build/nrf52832_xxaa_peer_manager.c.o
 .bss.m_deleting_all
                0x0000000020003360        0x1 _build/nrf52832_xxaa_peer_manager.c.o
 *fill*         0x0000000020003361        0x3 
 .bss.m_evt_handlers
                0x0000000020003364        0xc _build/nrf52832_xxaa_peer_manager.c.o
 .bss.m_highest_ranked_peer
                0x0000000020003370        0x2 _build/nrf52832_xxaa_peer_manager.c.o
 .bss.m_module_initialized
                0x0000000020003372        0x1 _build/nrf52832_xxaa_peer_manager.c.o
 .bss.m_n_registrants
                0x0000000020003373        0x1 _build/nrf52832_xxaa_peer_manager.c.o
 .bss.m_pairing_flag_id
                0x0000000020003374        0x1 _build/nrf52832_xxaa_peer_manager.c.o
 .bss.m_peer_rank_initialized
                0x0000000020003375        0x1 _build/nrf52832_xxaa_peer_manager.c.o
 *fill*         0x0000000020003376        0x2 
 .bss.m_peer_rank_token
                0x0000000020003378        0x4 _build/nrf52832_xxaa_peer_manager.c.o
 .bss.m_peer_pk
                0x000000002000337c       0x40 _build/nrf52832_xxaa_security_dispatcher.c.o
 .bss.m_p_public_key
                0x00000000200033bc        0x4 _build/nrf52832_xxaa_security_manager.c.o
 .bss.m_sec_params
                0x00000000200033c0        0x5 _build/nrf52832_xxaa_security_manager.c.o
 .bss.m_sec_params_valid
                0x00000000200033c5        0x1 _build/nrf52832_xxaa_security_manager.c.o
 .bss.m_ble_evt_buffer_size
                0x00000000200033c6        0x2 _build/nrf52832_xxaa_softdevice_handler.c.o
 .bss.m_ble_evt_handler
                0x00000000200033c8        0x4 _build/nrf52832_xxaa_softdevice_handler.c.o
 .bss.m_evt_schedule_func
                0x00000000200033cc        0x4 _build/nrf52832_xxaa_softdevice_handler.c.o
 .bss.m_softdevice_enabled
                0x00000000200033d0        0x1 _build/nrf52832_xxaa_softdevice_handler.c.o
 .bss.m_suspended
                0x00000000200033d1        0x1 _build/nrf52832_xxaa_softdevice_handler.c.o
 *fill*         0x00000000200033d2        0x2 
 .bss.m_sys_evt_handler
                0x00000000200033d4        0x4 _build/nrf52832_xxaa_softdevice_handler.c.o
 .bss.mp_ble_evt_buffer
                0x00000000200033d8        0x4 _build/nrf52832_xxaa_softdevice_handler.c.o
 .bss.__malloc_free_list
                0x00000000200033dc        0x4 /usr/local/bin/../lib/gcc/arm-none-eabi/8.3.1/../../../../arm-none-eabi/lib/thumb/v7e-m+fp/hard/libc_nano.a(lib_a-nano-mallocr.o)
                0x00000000200033dc                __malloc_free_list
 .bss.__malloc_sbrk_start
                0x00000000200033e0        0x4 /usr/local/bin/../lib/gcc/arm-none-eabi/8.3.1/../../../../arm-none-eabi/lib/thumb/v7e-m+fp/hard/libc_nano.a(lib_a-nano-mallocr.o)
                0x00000000200033e0                __malloc_sbrk_start
 .bss.heap_end.5501
                0x00000000200033e4        0x4 /usr/local/bin/../lib/gcc/arm-none-eabi/8.3.1/../../../../arm-none-eabi/lib/thumb/v7e-m+fp/hard/libnosys.a(sbrk.o)
 *(COMMON)
 COMMON         0x00000000200033e8       0xb0 _build/nrf52832_xxaa_ble_init.c.o
                0x00000000200033e8                ble_lcs
                0x00000000200033fc                m_gatt
                0x0000000020003418                ble_ics
                0x0000000020003434                ble_scs
                0x0000000020003450                ble_tcs
 COMMON         0x0000000020003498        0xc _build/nrf52832_xxaa_app_util_platform.c.o
                0x0000000020003498                nrf_nvic_state
 COMMON         0x00000000200034a4       0x78 _build/nrf52832_xxaa_SEGGER_RTT.c.o
                0x00000000200034a4                _SEGGER_RTT
 COMMON         0x000000002000351c        0x4 /usr/local/bin/../lib/gcc/arm-none-eabi/8.3.1/../../../../arm-none-eabi/lib/thumb/v7e-m+fp/hard/libc_nano.a(lib_a-reent.o)
                0x000000002000351c                errno
 COMMON         0x0000000020003520        0x9 /usr/local/bin/../lib/gcc/arm-none-eabi/8.3.1/../../../../arm-none-eabi/lib/thumb/v7e-m+fp/hard/libc_nano.a(lib_a-lock.o)
                0x0000000020003520                __lock___atexit_recursive_mutex
                0x0000000020003521                __lock___arc4random_mutex
                0x0000000020003522                __lock___env_recursive_mutex
                0x0000000020003523                __lock___sinit_recursive_mutex
                0x0000000020003524                __lock___malloc_recursive_mutex
                0x0000000020003525                __lock___at_quick_exit_mutex
                0x0000000020003526                __lock___dd_hash_mutex
                0x0000000020003527                __lock___tz_mutex
                0x0000000020003528                __lock___sfp_recursive_mutex
                0x000000002000352c                . = ALIGN (0x4)
 *fill*         0x0000000020003529        0x3 
                0x000000002000352c                __bss_end__ = .

.heap           0x0000000020003530     0x2000
                0x0000000020003530                __HeapBase = .
                0x0000000020003530                __end__ = .
                0x0000000020003530                PROVIDE (end = .)
 *(.heap*)
 .heap          0x0000000020003530     0x2000 _build/nrf52832_xxaa_gcc_startup_nrf52.S.o
                0x0000000020005530                __HeapLimit = .

.stack_dummy    0x0000000020003530     0x2000
 *(.stack*)
 .stack         0x0000000020003530     0x2000 _build/nrf52832_xxaa_gcc_startup_nrf52.S.o
                0x0000000020010000                __StackTop = (ORIGIN (RAM) + LENGTH (RAM))
                0x000000002000e000                __StackLimit = (__StackTop - SIZEOF (.stack_dummy))
                0x0000000020010000                PROVIDE (__stack = __StackTop)
                0x0000000000000001                ASSERT ((__StackLimit >= __HeapLimit), region RAM overflowed with stack)
OUTPUT(_build/nrf52832_xxaa.out elf32-littlearm)

.ARM.attributes
                0x0000000000000000       0x30
 .ARM.attributes
                0x0000000000000000       0x1e /usr/local/bin/../lib/gcc/arm-none-eabi/8.3.1/thumb/v7e-m+fp/hard/crti.o
 .ARM.attributes
                0x000000000000001e       0x34 /usr/local/bin/../lib/gcc/arm-none-eabi/8.3.1/thumb/v7e-m+fp/hard/crtbegin.o
 .ARM.attributes
                0x0000000000000052       0x1c /usr/local/bin/../lib/gcc/arm-none-eabi/8.3.1/../../../../arm-none-eabi/lib/thumb/v7e-m+fp/hard/crt0.o
 .ARM.attributes
                0x000000000000006e       0x34 /usr/local/bin/../lib/gcc/arm-none-eabi/8.3.1/../../../../arm-none-eabi/lib/thumb/v7e-m+fp/hard/libc_nano.a(lib_a-exit.o)
 .ARM.attributes
                0x00000000000000a2       0x32 /usr/local/bin/../lib/gcc/arm-none-eabi/8.3.1/../../../../arm-none-eabi/lib/thumb/v7e-m+fp/hard/libc_nano.a(lib_a-impure.o)
 .ARM.attributes
                0x00000000000000d4       0x34 /usr/local/bin/../lib/gcc/arm-none-eabi/8.3.1/../../../../arm-none-eabi/lib/thumb/v7e-m+fp/hard/libc_nano.a(lib_a-init.o)
 .ARM.attributes
                0x0000000000000108       0x34 /usr/local/bin/../lib/gcc/arm-none-eabi/8.3.1/../../../../arm-none-eabi/lib/thumb/v7e-m+fp/hard/libc_nano.a(lib_a-memset.o)
 .ARM.attributes
                0x000000000000013c       0x34 /usr/local/bin/../lib/gcc/arm-none-eabi/8.3.1/../../../../arm-none-eabi/lib/thumb/v7e-m+fp/hard/libnosys.a(_exit.o)
 .ARM.attributes
                0x0000000000000170       0x34 _build/nrf52832_xxaa_main.c.o
 .ARM.attributes
                0x00000000000001a4       0x34 _build/nrf52832_xxaa_ble_init.c.o
 .ARM.attributes
                0x00000000000001d8       0x34 _build/nrf52832_xxaa_ble_lcs.c.o
 .ARM.attributes
                0x000000000000020c       0x34 _build/nrf52832_xxaa_ble_ics.c.o
 .ARM.attributes
                0x0000000000000240       0x34 _build/nrf52832_xxaa_ble_tcs.c.o
 .ARM.attributes
                0x0000000000000274       0x34 _build/nrf52832_xxaa_ble_scs.c.o
 .ARM.attributes
                0x00000000000002a8       0x34 _build/nrf52832_xxaa_gpio.c.o
 .ARM.attributes
                0x00000000000002dc       0x34 _build/nrf52832_xxaa_uart.c.o
 .ARM.attributes
                0x0000000000000310       0x34 _build/nrf52832_xxaa_print.c.o
 .ARM.attributes
                0x0000000000000344       0x34 _build/nrf52832_xxaa_spim.c.o
 .ARM.attributes
                0x0000000000000378       0x34 _build/nrf52832_xxaa_stm_communication.c.o
 .ARM.attributes
                0x00000000000003ac       0x34 _build/nrf52832_xxaa_flash.c.o
 .ARM.attributes
                0x00000000000003e0       0x34 _build/nrf52832_xxaa_step_count_db.c.o
 .ARM.attributes
                0x0000000000000414       0x34 _build/nrf52832_xxaa_rtc.c.o
 .ARM.attributes
                0x0000000000000448       0x34 _build/nrf52832_xxaa_nrf_log_backend_serial.c.o
 .ARM.attributes
                0x000000000000047c       0x34 _build/nrf52832_xxaa_nrf_log_frontend.c.o
 .ARM.attributes
                0x00000000000004b0       0x34 _build/nrf52832_xxaa_app_error.c.o
 .ARM.attributes
                0x00000000000004e4       0x34 _build/nrf52832_xxaa_app_error_weak.c.o
 .ARM.attributes
                0x0000000000000518       0x34 _build/nrf52832_xxaa_app_timer.c.o
 .ARM.attributes
                0x000000000000054c       0x34 _build/nrf52832_xxaa_app_util_platform.c.o
 .ARM.attributes
                0x0000000000000580       0x34 _build/nrf52832_xxaa_fds.c.o
 .ARM.attributes
                0x00000000000005b4       0x34 _build/nrf52832_xxaa_fstorage.c.o
 .ARM.attributes
                0x00000000000005e8       0x34 _build/nrf52832_xxaa_sdk_mapped_flags.c.o
 .ARM.attributes
                0x000000000000061c       0x34 _build/nrf52832_xxaa_nrf_drv_clock.c.o
 .ARM.attributes
                0x0000000000000650       0x34 _build/nrf52832_xxaa_nrf_drv_common.c.o
 .ARM.attributes
                0x0000000000000684       0x34 _build/nrf52832_xxaa_nrf_drv_gpiote.c.o
 .ARM.attributes
                0x00000000000006b8       0x34 _build/nrf52832_xxaa_nrf_drv_uart.c.o
 .ARM.attributes
                0x00000000000006ec       0x34 _build/nrf52832_xxaa_SEGGER_RTT.c.o
 .ARM.attributes
                0x0000000000000720       0x34 _build/nrf52832_xxaa_ble_advdata.c.o
 .ARM.attributes
                0x0000000000000754       0x34 _build/nrf52832_xxaa_ble_advertising.c.o
 .ARM.attributes
                0x0000000000000788       0x34 _build/nrf52832_xxaa_ble_conn_params.c.o
 .ARM.attributes
                0x00000000000007bc       0x34 _build/nrf52832_xxaa_ble_conn_state.c.o
 .ARM.attributes
                0x00000000000007f0       0x34 _build/nrf52832_xxaa_ble_srv_common.c.o
 .ARM.attributes
                0x0000000000000824       0x34 _build/nrf52832_xxaa_gatt_cache_manager.c.o
 .ARM.attributes
                0x0000000000000858       0x34 _build/nrf52832_xxaa_gatts_cache_manager.c.o
 .ARM.attributes
                0x000000000000088c       0x34 _build/nrf52832_xxaa_id_manager.c.o
 .ARM.attributes
                0x00000000000008c0       0x34 _build/nrf52832_xxaa_nrf_ble_gatt.c.o
 .ARM.attributes
                0x00000000000008f4       0x34 _build/nrf52832_xxaa_peer_data_storage.c.o
 .ARM.attributes
                0x0000000000000928       0x34 _build/nrf52832_xxaa_peer_database.c.o
 .ARM.attributes
                0x000000000000095c       0x34 _build/nrf52832_xxaa_peer_id.c.o
 .ARM.attributes
                0x0000000000000990       0x34 _build/nrf52832_xxaa_peer_manager.c.o
 .ARM.attributes
                0x00000000000009c4       0x34 _build/nrf52832_xxaa_pm_buffer.c.o
 .ARM.attributes
                0x00000000000009f8       0x34 _build/nrf52832_xxaa_pm_mutex.c.o
 .ARM.attributes
                0x0000000000000a2c       0x34 _build/nrf52832_xxaa_security_dispatcher.c.o
 .ARM.attributes
                0x0000000000000a60       0x34 _build/nrf52832_xxaa_security_manager.c.o
 .ARM.attributes
                0x0000000000000a94       0x1c _build/nrf52832_xxaa_gcc_startup_nrf52.S.o
 .ARM.attributes
                0x0000000000000ab0       0x34 _build/nrf52832_xxaa_system_nrf52.c.o
 .ARM.attributes
                0x0000000000000ae4       0x34 _build/nrf52832_xxaa_softdevice_handler.c.o
 .ARM.attributes
                0x0000000000000b18       0x1e /usr/local/bin/../lib/gcc/arm-none-eabi/8.3.1/thumb/v7e-m+fp/hard/libgcc.a(_arm_addsubdf3.o)
 .ARM.attributes
                0x0000000000000b36       0x1e /usr/local/bin/../lib/gcc/arm-none-eabi/8.3.1/thumb/v7e-m+fp/hard/libgcc.a(_arm_muldivdf3.o)
 .ARM.attributes
                0x0000000000000b54       0x1e /usr/local/bin/../lib/gcc/arm-none-eabi/8.3.1/thumb/v7e-m+fp/hard/libgcc.a(_arm_cmpdf2.o)
 .ARM.attributes
                0x0000000000000b72       0x1e /usr/local/bin/../lib/gcc/arm-none-eabi/8.3.1/thumb/v7e-m+fp/hard/libgcc.a(_arm_fixdfsi.o)
 .ARM.attributes
                0x0000000000000b90       0x32 /usr/local/bin/../lib/gcc/arm-none-eabi/8.3.1/../../../../arm-none-eabi/lib/thumb/v7e-m+fp/hard/libc_nano.a(lib_a-ctype_.o)
 .ARM.attributes
                0x0000000000000bc2       0x34 /usr/local/bin/../lib/gcc/arm-none-eabi/8.3.1/../../../../arm-none-eabi/lib/thumb/v7e-m+fp/hard/libc_nano.a(lib_a-memcmp.o)
 .ARM.attributes
                0x0000000000000bf6       0x34 /usr/local/bin/../lib/gcc/arm-none-eabi/8.3.1/../../../../arm-none-eabi/lib/thumb/v7e-m+fp/hard/libc_nano.a(lib_a-memcpy-stub.o)
 .ARM.attributes
                0x0000000000000c2a       0x34 /usr/local/bin/../lib/gcc/arm-none-eabi/8.3.1/../../../../arm-none-eabi/lib/thumb/v7e-m+fp/hard/libc_nano.a(lib_a-snprintf.o)
 .ARM.attributes
                0x0000000000000c5e       0x34 /usr/local/bin/../lib/gcc/arm-none-eabi/8.3.1/../../../../arm-none-eabi/lib/thumb/v7e-m+fp/hard/libc_nano.a(lib_a-strcpy.o)
 .ARM.attributes
                0x0000000000000c92       0x17 /usr/local/bin/../lib/gcc/arm-none-eabi/8.3.1/../../../../arm-none-eabi/lib/thumb/v7e-m+fp/hard/libc_nano.a(lib_a-strlen.o)
 .ARM.attributes
                0x0000000000000ca9       0x34 /usr/local/bin/../lib/gcc/arm-none-eabi/8.3.1/../../../../arm-none-eabi/lib/thumb/v7e-m+fp/hard/libc_nano.a(lib_a-nano-svfprintf.o)
 .ARM.attributes
                0x0000000000000cdd       0x34 /usr/local/bin/../lib/gcc/arm-none-eabi/8.3.1/../../../../arm-none-eabi/lib/thumb/v7e-m+fp/hard/libc_nano.a(lib_a-nano-vfprintf_i.o)
 .ARM.attributes
                0x0000000000000d11       0x1c /usr/local/bin/../lib/gcc/arm-none-eabi/8.3.1/../../../../arm-none-eabi/lib/thumb/v7e-m+fp/hard/libc_nano.a(lib_a-memchr.o)
 .ARM.attributes
                0x0000000000000d2d       0x34 /usr/local/bin/../lib/gcc/arm-none-eabi/8.3.1/../../../../arm-none-eabi/lib/thumb/v7e-m+fp/hard/libc_nano.a(lib_a-memmove.o)
 .ARM.attributes
                0x0000000000000d61       0x34 /usr/local/bin/../lib/gcc/arm-none-eabi/8.3.1/../../../../arm-none-eabi/lib/thumb/v7e-m+fp/hard/libc_nano.a(lib_a-nano-freer.o)
 .ARM.attributes
                0x0000000000000d95       0x34 /usr/local/bin/../lib/gcc/arm-none-eabi/8.3.1/../../../../arm-none-eabi/lib/thumb/v7e-m+fp/hard/libc_nano.a(lib_a-nano-mallocr.o)
 .ARM.attributes
                0x0000000000000dc9       0x34 /usr/local/bin/../lib/gcc/arm-none-eabi/8.3.1/../../../../arm-none-eabi/lib/thumb/v7e-m+fp/hard/libc_nano.a(lib_a-nano-reallocr.o)
 .ARM.attributes
                0x0000000000000dfd       0x34 /usr/local/bin/../lib/gcc/arm-none-eabi/8.3.1/../../../../arm-none-eabi/lib/thumb/v7e-m+fp/hard/libc_nano.a(lib_a-sbrkr.o)
 .ARM.attributes
                0x0000000000000e31       0x34 /usr/local/bin/../lib/gcc/arm-none-eabi/8.3.1/../../../../arm-none-eabi/lib/thumb/v7e-m+fp/hard/libc_nano.a(lib_a-mlock.o)
 .ARM.attributes
                0x0000000000000e65       0x34 /usr/local/bin/../lib/gcc/arm-none-eabi/8.3.1/../../../../arm-none-eabi/lib/thumb/v7e-m+fp/hard/libc_nano.a(lib_a-nano-msizer.o)
 .ARM.attributes
                0x0000000000000e99       0x34 /usr/local/bin/../lib/gcc/arm-none-eabi/8.3.1/../../../../arm-none-eabi/lib/thumb/v7e-m+fp/hard/libc_nano.a(lib_a-reent.o)
 .ARM.attributes
                0x0000000000000ecd       0x34 /usr/local/bin/../lib/gcc/arm-none-eabi/8.3.1/../../../../arm-none-eabi/lib/thumb/v7e-m+fp/hard/libc_nano.a(lib_a-lock.o)
 .ARM.attributes
                0x0000000000000f01       0x32 /usr/local/bin/../lib/gcc/arm-none-eabi/8.3.1/thumb/v7e-m+fp/hard/crtend.o
 .ARM.attributes
                0x0000000000000f33       0x1e /usr/local/bin/../lib/gcc/arm-none-eabi/8.3.1/thumb/v7e-m+fp/hard/crtn.o
 .ARM.attributes
                0x0000000000000f51       0x34 /usr/local/bin/../lib/gcc/arm-none-eabi/8.3.1/../../../../arm-none-eabi/lib/thumb/v7e-m+fp/hard/libnosys.a(sbrk.o)

.comment        0x0000000000000000       0x76
 .comment       0x0000000000000000       0x76 _build/nrf52832_xxaa_main.c.o
                                         0x77 (size before relaxing)
 .comment       0x0000000000000076       0x77 _build/nrf52832_xxaa_ble_init.c.o
 .comment       0x0000000000000076       0x77 _build/nrf52832_xxaa_ble_lcs.c.o
 .comment       0x0000000000000076       0x77 _build/nrf52832_xxaa_ble_ics.c.o
 .comment       0x0000000000000076       0x77 _build/nrf52832_xxaa_ble_tcs.c.o
 .comment       0x0000000000000076       0x77 _build/nrf52832_xxaa_ble_scs.c.o
 .comment       0x0000000000000076       0x77 _build/nrf52832_xxaa_gpio.c.o
 .comment       0x0000000000000076       0x77 _build/nrf52832_xxaa_uart.c.o
 .comment       0x0000000000000076       0x77 _build/nrf52832_xxaa_print.c.o
 .comment       0x0000000000000076       0x77 _build/nrf52832_xxaa_spim.c.o
 .comment       0x0000000000000076       0x77 _build/nrf52832_xxaa_stm_communication.c.o
 .comment       0x0000000000000076       0x77 _build/nrf52832_xxaa_flash.c.o
 .comment       0x0000000000000076       0x77 _build/nrf52832_xxaa_step_count_db.c.o
 .comment       0x0000000000000076       0x77 _build/nrf52832_xxaa_rtc.c.o
 .comment       0x0000000000000076       0x77 _build/nrf52832_xxaa_nrf_log_backend_serial.c.o
 .comment       0x0000000000000076       0x77 _build/nrf52832_xxaa_nrf_log_frontend.c.o
 .comment       0x0000000000000076       0x77 _build/nrf52832_xxaa_app_error.c.o
 .comment       0x0000000000000076       0x77 _build/nrf52832_xxaa_app_error_weak.c.o
 .comment       0x0000000000000076       0x77 _build/nrf52832_xxaa_app_timer.c.o
 .comment       0x0000000000000076       0x77 _build/nrf52832_xxaa_app_util_platform.c.o
 .comment       0x0000000000000076       0x77 _build/nrf52832_xxaa_fds.c.o
 .comment       0x0000000000000076       0x77 _build/nrf52832_xxaa_fstorage.c.o
 .comment       0x0000000000000076       0x77 _build/nrf52832_xxaa_sdk_mapped_flags.c.o
 .comment       0x0000000000000076       0x77 _build/nrf52832_xxaa_nrf_drv_clock.c.o
 .comment       0x0000000000000076       0x77 _build/nrf52832_xxaa_nrf_drv_common.c.o
 .comment       0x0000000000000076       0x77 _build/nrf52832_xxaa_nrf_drv_gpiote.c.o
 .comment       0x0000000000000076       0x77 _build/nrf52832_xxaa_nrf_drv_uart.c.o
 .comment       0x0000000000000076       0x77 _build/nrf52832_xxaa_SEGGER_RTT.c.o
 .comment       0x0000000000000076       0x77 _build/nrf52832_xxaa_ble_advdata.c.o
 .comment       0x0000000000000076       0x77 _build/nrf52832_xxaa_ble_advertising.c.o
 .comment       0x0000000000000076       0x77 _build/nrf52832_xxaa_ble_conn_params.c.o
 .comment       0x0000000000000076       0x77 _build/nrf52832_xxaa_ble_conn_state.c.o
 .comment       0x0000000000000076       0x77 _build/nrf52832_xxaa_ble_srv_common.c.o
 .comment       0x0000000000000076       0x77 _build/nrf52832_xxaa_gatt_cache_manager.c.o
 .comment       0x0000000000000076       0x77 _build/nrf52832_xxaa_gatts_cache_manager.c.o
 .comment       0x0000000000000076       0x77 _build/nrf52832_xxaa_id_manager.c.o
 .comment       0x0000000000000076       0x77 _build/nrf52832_xxaa_nrf_ble_gatt.c.o
 .comment       0x0000000000000076       0x77 _build/nrf52832_xxaa_peer_data_storage.c.o
 .comment       0x0000000000000076       0x77 _build/nrf52832_xxaa_peer_database.c.o
 .comment       0x0000000000000076       0x77 _build/nrf52832_xxaa_peer_id.c.o
 .comment       0x0000000000000076       0x77 _build/nrf52832_xxaa_peer_manager.c.o
 .comment       0x0000000000000076       0x77 _build/nrf52832_xxaa_pm_buffer.c.o
 .comment       0x0000000000000076       0x77 _build/nrf52832_xxaa_pm_mutex.c.o
 .comment       0x0000000000000076       0x77 _build/nrf52832_xxaa_security_dispatcher.c.o
 .comment       0x0000000000000076       0x77 _build/nrf52832_xxaa_security_manager.c.o
 .comment       0x0000000000000076       0x77 _build/nrf52832_xxaa_system_nrf52.c.o
 .comment       0x0000000000000076       0x77 _build/nrf52832_xxaa_softdevice_handler.c.o

.debug_frame    0x0000000000000000     0x4668
 .debug_frame   0x0000000000000000       0x28 /usr/local/bin/../lib/gcc/arm-none-eabi/8.3.1/../../../../arm-none-eabi/lib/thumb/v7e-m+fp/hard/libc_nano.a(lib_a-exit.o)
 .debug_frame   0x0000000000000028       0x2c /usr/local/bin/../lib/gcc/arm-none-eabi/8.3.1/../../../../arm-none-eabi/lib/thumb/v7e-m+fp/hard/libc_nano.a(lib_a-init.o)
 .debug_frame   0x0000000000000054       0x20 /usr/local/bin/../lib/gcc/arm-none-eabi/8.3.1/../../../../arm-none-eabi/lib/thumb/v7e-m+fp/hard/libc_nano.a(lib_a-memset.o)
 .debug_frame   0x0000000000000074       0x20 /usr/local/bin/../lib/gcc/arm-none-eabi/8.3.1/../../../../arm-none-eabi/lib/thumb/v7e-m+fp/hard/libnosys.a(_exit.o)
 .debug_frame   0x0000000000000094       0x4c _build/nrf52832_xxaa_main.c.o
 .debug_frame   0x00000000000000e0      0x180 _build/nrf52832_xxaa_ble_init.c.o
 .debug_frame   0x0000000000000260       0xc0 _build/nrf52832_xxaa_ble_lcs.c.o
 .debug_frame   0x0000000000000320       0xdc _build/nrf52832_xxaa_ble_ics.c.o
 .debug_frame   0x00000000000003fc      0x250 _build/nrf52832_xxaa_ble_tcs.c.o
 .debug_frame   0x000000000000064c       0xe8 _build/nrf52832_xxaa_ble_scs.c.o
 .debug_frame   0x0000000000000734       0x50 _build/nrf52832_xxaa_gpio.c.o
 .debug_frame   0x0000000000000784       0x44 _build/nrf52832_xxaa_uart.c.o
 .debug_frame   0x00000000000007c8      0x168 _build/nrf52832_xxaa_print.c.o
 .debug_frame   0x0000000000000930       0xd0 _build/nrf52832_xxaa_spim.c.o
 .debug_frame   0x0000000000000a00       0xa4 _build/nrf52832_xxaa_stm_communication.c.o
 .debug_frame   0x0000000000000aa4       0x90 _build/nrf52832_xxaa_flash.c.o
 .debug_frame   0x0000000000000b34       0x68 _build/nrf52832_xxaa_step_count_db.c.o
 .debug_frame   0x0000000000000b9c       0x54 _build/nrf52832_xxaa_rtc.c.o
 .debug_frame   0x0000000000000bf0       0xc4 _build/nrf52832_xxaa_nrf_log_backend_serial.c.o
 .debug_frame   0x0000000000000cb4      0x278 _build/nrf52832_xxaa_nrf_log_frontend.c.o
 .debug_frame   0x0000000000000f2c       0x70 _build/nrf52832_xxaa_app_error.c.o
 .debug_frame   0x0000000000000f9c       0x28 _build/nrf52832_xxaa_app_error_weak.c.o
 .debug_frame   0x0000000000000fc4      0x164 _build/nrf52832_xxaa_app_timer.c.o
 .debug_frame   0x0000000000001128       0x90 _build/nrf52832_xxaa_app_util_platform.c.o
 .debug_frame   0x00000000000011b8      0x438 _build/nrf52832_xxaa_fds.c.o
 .debug_frame   0x00000000000015f0      0x164 _build/nrf52832_xxaa_fstorage.c.o
 .debug_frame   0x0000000000001754       0xe4 _build/nrf52832_xxaa_sdk_mapped_flags.c.o
 .debug_frame   0x0000000000001838      0x1f8 _build/nrf52832_xxaa_nrf_drv_clock.c.o
 .debug_frame   0x0000000000001a30       0x3c _build/nrf52832_xxaa_nrf_drv_common.c.o
 .debug_frame   0x0000000000001a6c      0x264 _build/nrf52832_xxaa_nrf_drv_gpiote.c.o
 .debug_frame   0x0000000000001cd0      0x1d4 _build/nrf52832_xxaa_nrf_drv_uart.c.o
 .debug_frame   0x0000000000001ea4      0x2d8 _build/nrf52832_xxaa_SEGGER_RTT.c.o
 .debug_frame   0x000000000000217c       0xfc _build/nrf52832_xxaa_ble_advdata.c.o
 .debug_frame   0x0000000000002278      0x168 _build/nrf52832_xxaa_ble_advertising.c.o
 .debug_frame   0x00000000000023e0      0x14c _build/nrf52832_xxaa_ble_conn_params.c.o
 .debug_frame   0x000000000000252c      0x200 _build/nrf52832_xxaa_ble_conn_state.c.o
 .debug_frame   0x000000000000272c       0xcc _build/nrf52832_xxaa_ble_srv_common.c.o
 .debug_frame   0x00000000000027f8      0x18c _build/nrf52832_xxaa_gatt_cache_manager.c.o
 .debug_frame   0x0000000000002984      0x184 _build/nrf52832_xxaa_gatts_cache_manager.c.o
 .debug_frame   0x0000000000002b08      0x3e8 _build/nrf52832_xxaa_id_manager.c.o
 .debug_frame   0x0000000000002ef0       0xec _build/nrf52832_xxaa_nrf_ble_gatt.c.o
 .debug_frame   0x0000000000002fdc      0x1fc _build/nrf52832_xxaa_peer_data_storage.c.o
 .debug_frame   0x00000000000031d8      0x20c _build/nrf52832_xxaa_peer_database.c.o
 .debug_frame   0x00000000000033e4      0x108 _build/nrf52832_xxaa_peer_id.c.o
 .debug_frame   0x00000000000034ec      0x4fc _build/nrf52832_xxaa_peer_manager.c.o
 .debug_frame   0x00000000000039e8       0xa8 _build/nrf52832_xxaa_pm_buffer.c.o
 .debug_frame   0x0000000000003a90       0xbc _build/nrf52832_xxaa_pm_mutex.c.o
 .debug_frame   0x0000000000003b4c      0x164 _build/nrf52832_xxaa_security_dispatcher.c.o
 .debug_frame   0x0000000000003cb0      0x170 _build/nrf52832_xxaa_security_manager.c.o
 .debug_frame   0x0000000000003e20       0x40 _build/nrf52832_xxaa_system_nrf52.c.o
 .debug_frame   0x0000000000003e60      0x1d0 _build/nrf52832_xxaa_softdevice_handler.c.o
 .debug_frame   0x0000000000004030       0xac /usr/local/bin/../lib/gcc/arm-none-eabi/8.3.1/thumb/v7e-m+fp/hard/libgcc.a(_arm_addsubdf3.o)
 .debug_frame   0x00000000000040dc       0x50 /usr/local/bin/../lib/gcc/arm-none-eabi/8.3.1/thumb/v7e-m+fp/hard/libgcc.a(_arm_muldivdf3.o)
 .debug_frame   0x000000000000412c       0xc4 /usr/local/bin/../lib/gcc/arm-none-eabi/8.3.1/thumb/v7e-m+fp/hard/libgcc.a(_arm_cmpdf2.o)
 .debug_frame   0x00000000000041f0       0x24 /usr/local/bin/../lib/gcc/arm-none-eabi/8.3.1/thumb/v7e-m+fp/hard/libgcc.a(_arm_fixdfsi.o)
 .debug_frame   0x0000000000004214       0x2c /usr/local/bin/../lib/gcc/arm-none-eabi/8.3.1/../../../../arm-none-eabi/lib/thumb/v7e-m+fp/hard/libc_nano.a(lib_a-memcmp.o)
 .debug_frame   0x0000000000004240       0x28 /usr/local/bin/../lib/gcc/arm-none-eabi/8.3.1/../../../../arm-none-eabi/lib/thumb/v7e-m+fp/hard/libc_nano.a(lib_a-memcpy-stub.o)
 .debug_frame   0x0000000000004268       0x7c /usr/local/bin/../lib/gcc/arm-none-eabi/8.3.1/../../../../arm-none-eabi/lib/thumb/v7e-m+fp/hard/libc_nano.a(lib_a-snprintf.o)
 .debug_frame   0x00000000000042e4       0x20 /usr/local/bin/../lib/gcc/arm-none-eabi/8.3.1/../../../../arm-none-eabi/lib/thumb/v7e-m+fp/hard/libc_nano.a(lib_a-strcpy.o)
 .debug_frame   0x0000000000004304       0x90 /usr/local/bin/../lib/gcc/arm-none-eabi/8.3.1/../../../../arm-none-eabi/lib/thumb/v7e-m+fp/hard/libc_nano.a(lib_a-nano-svfprintf.o)
 .debug_frame   0x0000000000004394       0x60 /usr/local/bin/../lib/gcc/arm-none-eabi/8.3.1/../../../../arm-none-eabi/lib/thumb/v7e-m+fp/hard/libc_nano.a(lib_a-nano-vfprintf_i.o)
 .debug_frame   0x00000000000043f4       0x28 /usr/local/bin/../lib/gcc/arm-none-eabi/8.3.1/../../../../arm-none-eabi/lib/thumb/v7e-m+fp/hard/libc_nano.a(lib_a-memmove.o)
 .debug_frame   0x000000000000441c       0x38 /usr/local/bin/../lib/gcc/arm-none-eabi/8.3.1/../../../../arm-none-eabi/lib/thumb/v7e-m+fp/hard/libc_nano.a(lib_a-nano-freer.o)
 .debug_frame   0x0000000000004454       0x30 /usr/local/bin/../lib/gcc/arm-none-eabi/8.3.1/../../../../arm-none-eabi/lib/thumb/v7e-m+fp/hard/libc_nano.a(lib_a-nano-mallocr.o)
 .debug_frame   0x0000000000004484       0x3c /usr/local/bin/../lib/gcc/arm-none-eabi/8.3.1/../../../../arm-none-eabi/lib/thumb/v7e-m+fp/hard/libc_nano.a(lib_a-nano-reallocr.o)
 .debug_frame   0x00000000000044c0       0x2c /usr/local/bin/../lib/gcc/arm-none-eabi/8.3.1/../../../../arm-none-eabi/lib/thumb/v7e-m+fp/hard/libc_nano.a(lib_a-sbrkr.o)
 .debug_frame   0x00000000000044ec       0x30 /usr/local/bin/../lib/gcc/arm-none-eabi/8.3.1/../../../../arm-none-eabi/lib/thumb/v7e-m+fp/hard/libc_nano.a(lib_a-mlock.o)
 .debug_frame   0x000000000000451c       0x20 /usr/local/bin/../lib/gcc/arm-none-eabi/8.3.1/../../../../arm-none-eabi/lib/thumb/v7e-m+fp/hard/libc_nano.a(lib_a-nano-msizer.o)
 .debug_frame   0x000000000000453c       0x5c /usr/local/bin/../lib/gcc/arm-none-eabi/8.3.1/../../../../arm-none-eabi/lib/thumb/v7e-m+fp/hard/libc_nano.a(lib_a-reent.o)
 .debug_frame   0x0000000000004598       0xb0 /usr/local/bin/../lib/gcc/arm-none-eabi/8.3.1/../../../../arm-none-eabi/lib/thumb/v7e-m+fp/hard/libc_nano.a(lib_a-lock.o)
 .debug_frame   0x0000000000004648       0x20 /usr/local/bin/../lib/gcc/arm-none-eabi/8.3.1/../../../../arm-none-eabi/lib/thumb/v7e-m+fp/hard/libnosys.a(sbrk.o)

.debug_info     0x0000000000000000    0x671f3
 .debug_info    0x0000000000000000     0x11f6 _build/nrf52832_xxaa_main.c.o
 .debug_info    0x00000000000011f6     0x527d _build/nrf52832_xxaa_ble_init.c.o
 .debug_info    0x0000000000006473     0x29e7 _build/nrf52832_xxaa_ble_lcs.c.o
 .debug_info    0x0000000000008e5a     0x2b1d _build/nrf52832_xxaa_ble_ics.c.o
 .debug_info    0x000000000000b977     0x4415 _build/nrf52832_xxaa_ble_tcs.c.o
 .debug_info    0x000000000000fd8c     0x2adf _build/nrf52832_xxaa_ble_scs.c.o
 .debug_info    0x000000000001286b      0xac7 _build/nrf52832_xxaa_gpio.c.o
 .debug_info    0x0000000000013332      0x5aa _build/nrf52832_xxaa_uart.c.o
 .debug_info    0x00000000000138dc      0xa1d _build/nrf52832_xxaa_print.c.o
 .debug_info    0x00000000000142f9      0x981 _build/nrf52832_xxaa_spim.c.o
 .debug_info    0x0000000000014c7a      0x4a5 _build/nrf52832_xxaa_stm_communication.c.o
 .debug_info    0x000000000001511f      0x4b2 _build/nrf52832_xxaa_flash.c.o
 .debug_info    0x00000000000155d1      0x32f _build/nrf52832_xxaa_step_count_db.c.o
 .debug_info    0x0000000000015900      0x7de _build/nrf52832_xxaa_rtc.c.o
 .debug_info    0x00000000000160de     0x15d7 _build/nrf52832_xxaa_nrf_log_backend_serial.c.o
 .debug_info    0x00000000000176b5     0x2178 _build/nrf52832_xxaa_nrf_log_frontend.c.o
 .debug_info    0x000000000001982d      0xc98 _build/nrf52832_xxaa_app_error.c.o
 .debug_info    0x000000000001a4c5      0xd2d _build/nrf52832_xxaa_app_error_weak.c.o
 .debug_info    0x000000000001b1f2     0x2883 _build/nrf52832_xxaa_app_timer.c.o
 .debug_info    0x000000000001da75     0x1305 _build/nrf52832_xxaa_app_util_platform.c.o
 .debug_info    0x000000000001ed7a     0x5244 _build/nrf52832_xxaa_fds.c.o
 .debug_info    0x0000000000023fbe     0x1d70 _build/nrf52832_xxaa_fstorage.c.o
 .debug_info    0x0000000000025d2e      0x67e _build/nrf52832_xxaa_sdk_mapped_flags.c.o
 .debug_info    0x00000000000263ac     0x220e _build/nrf52832_xxaa_nrf_drv_clock.c.o
 .debug_info    0x00000000000285ba      0xfc8 _build/nrf52832_xxaa_nrf_drv_common.c.o
 .debug_info    0x0000000000029582     0x3833 _build/nrf52832_xxaa_nrf_drv_gpiote.c.o
 .debug_info    0x000000000002cdb5     0x59a5 _build/nrf52832_xxaa_nrf_drv_uart.c.o
 .debug_info    0x000000000003275a     0x3380 _build/nrf52832_xxaa_SEGGER_RTT.c.o
 .debug_info    0x0000000000035ada     0x1f51 _build/nrf52832_xxaa_ble_advdata.c.o
 .debug_info    0x0000000000037a2b     0x3071 _build/nrf52832_xxaa_ble_advertising.c.o
 .debug_info    0x000000000003aa9c     0x2745 _build/nrf52832_xxaa_ble_conn_params.c.o
 .debug_info    0x000000000003d1e1     0x28b2 _build/nrf52832_xxaa_ble_conn_state.c.o
 .debug_info    0x000000000003fa93     0x16e7 _build/nrf52832_xxaa_ble_srv_common.c.o
 .debug_info    0x000000000004117a     0x3616 _build/nrf52832_xxaa_gatt_cache_manager.c.o
 .debug_info    0x0000000000044790     0x1bb9 _build/nrf52832_xxaa_gatts_cache_manager.c.o
 .debug_info    0x0000000000046349     0x4c4f _build/nrf52832_xxaa_id_manager.c.o
 .debug_info    0x000000000004af98     0x2c69 _build/nrf52832_xxaa_nrf_ble_gatt.c.o
 .debug_info    0x000000000004dc01     0x2877 _build/nrf52832_xxaa_peer_data_storage.c.o
 .debug_info    0x0000000000050478     0x2ae4 _build/nrf52832_xxaa_peer_database.c.o
 .debug_info    0x0000000000052f5c     0x116b _build/nrf52832_xxaa_peer_id.c.o
 .debug_info    0x00000000000540c7     0x4e1b _build/nrf52832_xxaa_peer_manager.c.o
 .debug_info    0x0000000000058ee2      0xcd9 _build/nrf52832_xxaa_pm_buffer.c.o
 .debug_info    0x0000000000059bbb      0xdb5 _build/nrf52832_xxaa_pm_mutex.c.o
 .debug_info    0x000000000005a970     0x4bdf _build/nrf52832_xxaa_security_dispatcher.c.o
 .debug_info    0x000000000005f54f     0x3a35 _build/nrf52832_xxaa_security_manager.c.o
 .debug_info    0x0000000000062f84      0xefc _build/nrf52832_xxaa_system_nrf52.c.o
 .debug_info    0x0000000000063e80     0x3373 _build/nrf52832_xxaa_softdevice_handler.c.o

.debug_abbrev   0x0000000000000000     0xbfa7
 .debug_abbrev  0x0000000000000000      0x322 _build/nrf52832_xxaa_main.c.o
 .debug_abbrev  0x0000000000000322      0x53a _build/nrf52832_xxaa_ble_init.c.o
 .debug_abbrev  0x000000000000085c      0x459 _build/nrf52832_xxaa_ble_lcs.c.o
 .debug_abbrev  0x0000000000000cb5      0x473 _build/nrf52832_xxaa_ble_ics.c.o
 .debug_abbrev  0x0000000000001128      0x4a0 _build/nrf52832_xxaa_ble_tcs.c.o
 .debug_abbrev  0x00000000000015c8      0x466 _build/nrf52832_xxaa_ble_scs.c.o
 .debug_abbrev  0x0000000000001a2e      0x200 _build/nrf52832_xxaa_gpio.c.o
 .debug_abbrev  0x0000000000001c2e      0x17a _build/nrf52832_xxaa_uart.c.o
 .debug_abbrev  0x0000000000001da8      0x259 _build/nrf52832_xxaa_print.c.o
 .debug_abbrev  0x0000000000002001      0x209 _build/nrf52832_xxaa_spim.c.o
 .debug_abbrev  0x000000000000220a      0x1a9 _build/nrf52832_xxaa_stm_communication.c.o
 .debug_abbrev  0x00000000000023b3      0x1d4 _build/nrf52832_xxaa_flash.c.o
 .debug_abbrev  0x0000000000002587      0x15b _build/nrf52832_xxaa_step_count_db.c.o
 .debug_abbrev  0x00000000000026e2      0x20c _build/nrf52832_xxaa_rtc.c.o
 .debug_abbrev  0x00000000000028ee      0x4e8 _build/nrf52832_xxaa_nrf_log_backend_serial.c.o
 .debug_abbrev  0x0000000000002dd6      0x4a7 _build/nrf52832_xxaa_nrf_log_frontend.c.o
 .debug_abbrev  0x000000000000327d      0x276 _build/nrf52832_xxaa_app_error.c.o
 .debug_abbrev  0x00000000000034f3      0x295 _build/nrf52832_xxaa_app_error_weak.c.o
 .debug_abbrev  0x0000000000003788      0x518 _build/nrf52832_xxaa_app_timer.c.o
 .debug_abbrev  0x0000000000003ca0      0x3e6 _build/nrf52832_xxaa_app_util_platform.c.o
 .debug_abbrev  0x0000000000004086      0x60e _build/nrf52832_xxaa_fds.c.o
 .debug_abbrev  0x0000000000004694      0x542 _build/nrf52832_xxaa_fstorage.c.o
 .debug_abbrev  0x0000000000004bd6      0x291 _build/nrf52832_xxaa_sdk_mapped_flags.c.o
 .debug_abbrev  0x0000000000004e67      0x613 _build/nrf52832_xxaa_nrf_drv_clock.c.o
 .debug_abbrev  0x000000000000547a      0x2ec _build/nrf52832_xxaa_nrf_drv_common.c.o
 .debug_abbrev  0x0000000000005766      0x59a _build/nrf52832_xxaa_nrf_drv_gpiote.c.o
 .debug_abbrev  0x0000000000005d00      0x514 _build/nrf52832_xxaa_nrf_drv_uart.c.o
 .debug_abbrev  0x0000000000006214      0x459 _build/nrf52832_xxaa_SEGGER_RTT.c.o
 .debug_abbrev  0x000000000000666d      0x448 _build/nrf52832_xxaa_ble_advdata.c.o
 .debug_abbrev  0x0000000000006ab5      0x5b4 _build/nrf52832_xxaa_ble_advertising.c.o
 .debug_abbrev  0x0000000000007069      0x504 _build/nrf52832_xxaa_ble_conn_params.c.o
 .debug_abbrev  0x000000000000756d      0x505 _build/nrf52832_xxaa_ble_conn_state.c.o
 .debug_abbrev  0x0000000000007a72      0x3be _build/nrf52832_xxaa_ble_srv_common.c.o
 .debug_abbrev  0x0000000000007e30      0x53b _build/nrf52832_xxaa_gatt_cache_manager.c.o
 .debug_abbrev  0x000000000000836b      0x4bf _build/nrf52832_xxaa_gatts_cache_manager.c.o
 .debug_abbrev  0x000000000000882a      0x687 _build/nrf52832_xxaa_id_manager.c.o
 .debug_abbrev  0x0000000000008eb1      0x499 _build/nrf52832_xxaa_nrf_ble_gatt.c.o
 .debug_abbrev  0x000000000000934a      0x507 _build/nrf52832_xxaa_peer_data_storage.c.o
 .debug_abbrev  0x0000000000009851      0x54d _build/nrf52832_xxaa_peer_database.c.o
 .debug_abbrev  0x0000000000009d9e      0x39e _build/nrf52832_xxaa_peer_id.c.o
 .debug_abbrev  0x000000000000a13c      0x573 _build/nrf52832_xxaa_peer_manager.c.o
 .debug_abbrev  0x000000000000a6af      0x2f0 _build/nrf52832_xxaa_pm_buffer.c.o
 .debug_abbrev  0x000000000000a99f      0x332 _build/nrf52832_xxaa_pm_mutex.c.o
 .debug_abbrev  0x000000000000acd1      0x579 _build/nrf52832_xxaa_security_dispatcher.c.o
 .debug_abbrev  0x000000000000b24a      0x540 _build/nrf52832_xxaa_security_manager.c.o
 .debug_abbrev  0x000000000000b78a      0x226 _build/nrf52832_xxaa_system_nrf52.c.o
 .debug_abbrev  0x000000000000b9b0      0x5f7 _build/nrf52832_xxaa_softdevice_handler.c.o

.debug_loc      0x0000000000000000    0x2fba4
 .debug_loc     0x0000000000000000       0x9b _build/nrf52832_xxaa_main.c.o
 .debug_loc     0x000000000000009b      0xc8a _build/nrf52832_xxaa_ble_init.c.o
 .debug_loc     0x0000000000000d25      0x4dc _build/nrf52832_xxaa_ble_lcs.c.o
 .debug_loc     0x0000000000001201      0x695 _build/nrf52832_xxaa_ble_ics.c.o
 .debug_loc     0x0000000000001896     0x26be _build/nrf52832_xxaa_ble_tcs.c.o
 .debug_loc     0x0000000000003f54      0x46e _build/nrf52832_xxaa_ble_scs.c.o
 .debug_loc     0x00000000000043c2       0x60 _build/nrf52832_xxaa_uart.c.o
 .debug_loc     0x0000000000004422      0xe94 _build/nrf52832_xxaa_print.c.o
 .debug_loc     0x00000000000052b6      0x478 _build/nrf52832_xxaa_spim.c.o
 .debug_loc     0x000000000000572e      0x212 _build/nrf52832_xxaa_stm_communication.c.o
 .debug_loc     0x0000000000005940      0x16a _build/nrf52832_xxaa_flash.c.o
 .debug_loc     0x0000000000005aaa      0x27b _build/nrf52832_xxaa_step_count_db.c.o
 .debug_loc     0x0000000000005d25       0x45 _build/nrf52832_xxaa_rtc.c.o
 .debug_loc     0x0000000000005d6a     0x13fe _build/nrf52832_xxaa_nrf_log_backend_serial.c.o
 .debug_loc     0x0000000000007168     0x1f27 _build/nrf52832_xxaa_nrf_log_frontend.c.o
 .debug_loc     0x000000000000908f      0x154 _build/nrf52832_xxaa_app_error.c.o
 .debug_loc     0x00000000000091e3       0x6f _build/nrf52832_xxaa_app_error_weak.c.o
 .debug_loc     0x0000000000009252     0x139f _build/nrf52832_xxaa_app_timer.c.o
 .debug_loc     0x000000000000a5f1      0x1e9 _build/nrf52832_xxaa_app_util_platform.c.o
 .debug_loc     0x000000000000a7da     0x5f7f _build/nrf52832_xxaa_fds.c.o
 .debug_loc     0x0000000000010759      0xc8b _build/nrf52832_xxaa_fstorage.c.o
 .debug_loc     0x00000000000113e4      0x5de _build/nrf52832_xxaa_sdk_mapped_flags.c.o
 .debug_loc     0x00000000000119c2      0x609 _build/nrf52832_xxaa_nrf_drv_clock.c.o
 .debug_loc     0x0000000000011fcb      0x107 _build/nrf52832_xxaa_nrf_drv_common.c.o
 .debug_loc     0x00000000000120d2     0x3725 _build/nrf52832_xxaa_nrf_drv_gpiote.c.o
 .debug_loc     0x00000000000157f7     0x31ca _build/nrf52832_xxaa_nrf_drv_uart.c.o
 .debug_loc     0x00000000000189c1     0x4e76 _build/nrf52832_xxaa_SEGGER_RTT.c.o
 .debug_loc     0x000000000001d837      0xc93 _build/nrf52832_xxaa_ble_advdata.c.o
 .debug_loc     0x000000000001e4ca      0x7bd _build/nrf52832_xxaa_ble_advertising.c.o
 .debug_loc     0x000000000001ec87      0x429 _build/nrf52832_xxaa_ble_conn_params.c.o
 .debug_loc     0x000000000001f0b0      0x4ab _build/nrf52832_xxaa_ble_conn_state.c.o
 .debug_loc     0x000000000001f55b      0x732 _build/nrf52832_xxaa_ble_srv_common.c.o
 .debug_loc     0x000000000001fc8d      0xb63 _build/nrf52832_xxaa_gatt_cache_manager.c.o
 .debug_loc     0x00000000000207f0      0x59e _build/nrf52832_xxaa_gatts_cache_manager.c.o
 .debug_loc     0x0000000000020d8e     0x2761 _build/nrf52832_xxaa_id_manager.c.o
 .debug_loc     0x00000000000234ef      0xdfa _build/nrf52832_xxaa_nrf_ble_gatt.c.o
 .debug_loc     0x00000000000242e9      0xd76 _build/nrf52832_xxaa_peer_data_storage.c.o
 .debug_loc     0x000000000002505f     0x3f58 _build/nrf52832_xxaa_peer_database.c.o
 .debug_loc     0x0000000000028fb7      0x644 _build/nrf52832_xxaa_peer_id.c.o
 .debug_loc     0x00000000000295fb     0x2541 _build/nrf52832_xxaa_peer_manager.c.o
 .debug_loc     0x000000000002bb3c      0x413 _build/nrf52832_xxaa_pm_buffer.c.o
 .debug_loc     0x000000000002bf4f      0x4f9 _build/nrf52832_xxaa_pm_mutex.c.o
 .debug_loc     0x000000000002c448     0x1ea2 _build/nrf52832_xxaa_security_dispatcher.c.o
 .debug_loc     0x000000000002e2ea     0x10d9 _build/nrf52832_xxaa_security_manager.c.o
 .debug_loc     0x000000000002f3c3      0x7e1 _build/nrf52832_xxaa_softdevice_handler.c.o

.debug_aranges  0x0000000000000000     0x1418
 .debug_aranges
                0x0000000000000000       0x30 _build/nrf52832_xxaa_main.c.o
 .debug_aranges
                0x0000000000000030       0x98 _build/nrf52832_xxaa_ble_init.c.o
 .debug_aranges
                0x00000000000000c8       0x48 _build/nrf52832_xxaa_ble_lcs.c.o
 .debug_aranges
                0x0000000000000110       0x58 _build/nrf52832_xxaa_ble_ics.c.o
 .debug_aranges
                0x0000000000000168       0x80 _build/nrf52832_xxaa_ble_tcs.c.o
 .debug_aranges
                0x00000000000001e8       0x58 _build/nrf52832_xxaa_ble_scs.c.o
 .debug_aranges
                0x0000000000000240       0x38 _build/nrf52832_xxaa_gpio.c.o
 .debug_aranges
                0x0000000000000278       0x28 _build/nrf52832_xxaa_uart.c.o
 .debug_aranges
                0x00000000000002a0       0x58 _build/nrf52832_xxaa_print.c.o
 .debug_aranges
                0x00000000000002f8       0x58 _build/nrf52832_xxaa_spim.c.o
 .debug_aranges
                0x0000000000000350       0x38 _build/nrf52832_xxaa_stm_communication.c.o
 .debug_aranges
                0x0000000000000388       0x48 _build/nrf52832_xxaa_flash.c.o
 .debug_aranges
                0x00000000000003d0       0x28 _build/nrf52832_xxaa_step_count_db.c.o
 .debug_aranges
                0x00000000000003f8       0x30 _build/nrf52832_xxaa_rtc.c.o
 .debug_aranges
                0x0000000000000428       0x48 _build/nrf52832_xxaa_nrf_log_backend_serial.c.o
 .debug_aranges
                0x0000000000000470       0x98 _build/nrf52832_xxaa_nrf_log_frontend.c.o
 .debug_aranges
                0x0000000000000508       0x30 _build/nrf52832_xxaa_app_error.c.o
 .debug_aranges
                0x0000000000000538       0x20 _build/nrf52832_xxaa_app_error_weak.c.o
 .debug_aranges
                0x0000000000000558       0x70 _build/nrf52832_xxaa_app_timer.c.o
 .debug_aranges
                0x00000000000005c8       0x48 _build/nrf52832_xxaa_app_util_platform.c.o
 .debug_aranges
                0x0000000000000610       0xd8 _build/nrf52832_xxaa_fds.c.o
 .debug_aranges
                0x00000000000006e8       0x70 _build/nrf52832_xxaa_fstorage.c.o
 .debug_aranges
                0x0000000000000758       0x48 _build/nrf52832_xxaa_sdk_mapped_flags.c.o
 .debug_aranges
                0x00000000000007a0       0xb0 _build/nrf52832_xxaa_nrf_drv_clock.c.o
 .debug_aranges
                0x0000000000000850       0x28 _build/nrf52832_xxaa_nrf_drv_common.c.o
 .debug_aranges
                0x0000000000000878       0xd8 _build/nrf52832_xxaa_nrf_drv_gpiote.c.o
 .debug_aranges
                0x0000000000000950       0x78 _build/nrf52832_xxaa_nrf_drv_uart.c.o
 .debug_aranges
                0x00000000000009c8       0xa0 _build/nrf52832_xxaa_SEGGER_RTT.c.o
 .debug_aranges
                0x0000000000000a68       0x58 _build/nrf52832_xxaa_ble_advdata.c.o
 .debug_aranges
                0x0000000000000ac0       0x70 _build/nrf52832_xxaa_ble_advertising.c.o
 .debug_aranges
                0x0000000000000b30       0x68 _build/nrf52832_xxaa_ble_conn_params.c.o
 .debug_aranges
                0x0000000000000b98       0xa0 _build/nrf52832_xxaa_ble_conn_state.c.o
 .debug_aranges
                0x0000000000000c38       0x58 _build/nrf52832_xxaa_ble_srv_common.c.o
 .debug_aranges
                0x0000000000000c90       0x70 _build/nrf52832_xxaa_gatt_cache_manager.c.o
 .debug_aranges
                0x0000000000000d00       0x78 _build/nrf52832_xxaa_gatts_cache_manager.c.o
 .debug_aranges
                0x0000000000000d78      0x128 _build/nrf52832_xxaa_id_manager.c.o
 .debug_aranges
                0x0000000000000ea0       0x68 _build/nrf52832_xxaa_nrf_ble_gatt.c.o
 .debug_aranges
                0x0000000000000f08       0x98 _build/nrf52832_xxaa_peer_data_storage.c.o
 .debug_aranges
                0x0000000000000fa0       0x90 _build/nrf52832_xxaa_peer_database.c.o
 .debug_aranges
                0x0000000000001030       0x68 _build/nrf52832_xxaa_peer_id.c.o
 .debug_aranges
                0x0000000000001098      0x158 _build/nrf52832_xxaa_peer_manager.c.o
 .debug_aranges
                0x00000000000011f0       0x38 _build/nrf52832_xxaa_pm_buffer.c.o
 .debug_aranges
                0x0000000000001228       0x40 _build/nrf52832_xxaa_pm_mutex.c.o
 .debug_aranges
                0x0000000000001268       0x68 _build/nrf52832_xxaa_security_dispatcher.c.o
 .debug_aranges
                0x00000000000012d0       0x70 _build/nrf52832_xxaa_security_manager.c.o
 .debug_aranges
                0x0000000000001340       0x28 _build/nrf52832_xxaa_system_nrf52.c.o
 .debug_aranges
                0x0000000000001368       0xb0 _build/nrf52832_xxaa_softdevice_handler.c.o

.debug_ranges   0x0000000000000000     0xa908
 .debug_ranges  0x0000000000000000       0x80 _build/nrf52832_xxaa_main.c.o
 .debug_ranges  0x0000000000000080      0x4c0 _build/nrf52832_xxaa_ble_init.c.o
 .debug_ranges  0x0000000000000540       0xd8 _build/nrf52832_xxaa_ble_lcs.c.o
 .debug_ranges  0x0000000000000618       0x70 _build/nrf52832_xxaa_ble_ics.c.o
 .debug_ranges  0x0000000000000688      0x418 _build/nrf52832_xxaa_ble_tcs.c.o
 .debug_ranges  0x0000000000000aa0       0xa8 _build/nrf52832_xxaa_ble_scs.c.o
 .debug_ranges  0x0000000000000b48       0x28 _build/nrf52832_xxaa_gpio.c.o
 .debug_ranges  0x0000000000000b70       0x30 _build/nrf52832_xxaa_uart.c.o
 .debug_ranges  0x0000000000000ba0      0x2b8 _build/nrf52832_xxaa_print.c.o
 .debug_ranges  0x0000000000000e58       0xb8 _build/nrf52832_xxaa_spim.c.o
 .debug_ranges  0x0000000000000f10       0x48 _build/nrf52832_xxaa_stm_communication.c.o
 .debug_ranges  0x0000000000000f58       0x38 _build/nrf52832_xxaa_flash.c.o
 .debug_ranges  0x0000000000000f90       0x78 _build/nrf52832_xxaa_step_count_db.c.o
 .debug_ranges  0x0000000000001008       0x58 _build/nrf52832_xxaa_rtc.c.o
 .debug_ranges  0x0000000000001060      0x128 _build/nrf52832_xxaa_nrf_log_backend_serial.c.o
 .debug_ranges  0x0000000000001188      0x338 _build/nrf52832_xxaa_nrf_log_frontend.c.o
 .debug_ranges  0x00000000000014c0       0x20 _build/nrf52832_xxaa_app_error.c.o
 .debug_ranges  0x00000000000014e0       0x10 _build/nrf52832_xxaa_app_error_weak.c.o
 .debug_ranges  0x00000000000014f0      0x720 _build/nrf52832_xxaa_app_timer.c.o
 .debug_ranges  0x0000000000001c10      0x148 _build/nrf52832_xxaa_app_util_platform.c.o
 .debug_ranges  0x0000000000001d58     0x1610 _build/nrf52832_xxaa_fds.c.o
 .debug_ranges  0x0000000000003368      0x2a8 _build/nrf52832_xxaa_fstorage.c.o
 .debug_ranges  0x0000000000003610      0x1e8 _build/nrf52832_xxaa_sdk_mapped_flags.c.o
 .debug_ranges  0x00000000000037f8      0x578 _build/nrf52832_xxaa_nrf_drv_clock.c.o
 .debug_ranges  0x0000000000003d70       0x50 _build/nrf52832_xxaa_nrf_drv_common.c.o
 .debug_ranges  0x0000000000003dc0     0x1430 _build/nrf52832_xxaa_nrf_drv_gpiote.c.o
 .debug_ranges  0x00000000000051f0      0xc38 _build/nrf52832_xxaa_nrf_drv_uart.c.o
 .debug_ranges  0x0000000000005e28      0x820 _build/nrf52832_xxaa_SEGGER_RTT.c.o
 .debug_ranges  0x0000000000006648      0x178 _build/nrf52832_xxaa_ble_advdata.c.o
 .debug_ranges  0x00000000000067c0      0x240 _build/nrf52832_xxaa_ble_advertising.c.o
 .debug_ranges  0x0000000000006a00      0x120 _build/nrf52832_xxaa_ble_conn_params.c.o
 .debug_ranges  0x0000000000006b20      0x118 _build/nrf52832_xxaa_ble_conn_state.c.o
 .debug_ranges  0x0000000000006c38      0x158 _build/nrf52832_xxaa_ble_srv_common.c.o
 .debug_ranges  0x0000000000006d90      0x3b8 _build/nrf52832_xxaa_gatt_cache_manager.c.o
 .debug_ranges  0x0000000000007148      0x170 _build/nrf52832_xxaa_gatts_cache_manager.c.o
 .debug_ranges  0x00000000000072b8      0x7b0 _build/nrf52832_xxaa_id_manager.c.o
 .debug_ranges  0x0000000000007a68      0x150 _build/nrf52832_xxaa_nrf_ble_gatt.c.o
 .debug_ranges  0x0000000000007bb8      0x340 _build/nrf52832_xxaa_peer_data_storage.c.o
 .debug_ranges  0x0000000000007ef8      0xfa8 _build/nrf52832_xxaa_peer_database.c.o
 .debug_ranges  0x0000000000008ea0      0x1b8 _build/nrf52832_xxaa_peer_id.c.o
 .debug_ranges  0x0000000000009058      0x600 _build/nrf52832_xxaa_peer_manager.c.o
 .debug_ranges  0x0000000000009658       0xa0 _build/nrf52832_xxaa_pm_buffer.c.o
 .debug_ranges  0x00000000000096f8       0xc8 _build/nrf52832_xxaa_pm_mutex.c.o
 .debug_ranges  0x00000000000097c0      0x8b0 _build/nrf52832_xxaa_security_dispatcher.c.o
 .debug_ranges  0x000000000000a070      0x460 _build/nrf52832_xxaa_security_manager.c.o
 .debug_ranges  0x000000000000a4d0      0x1c0 _build/nrf52832_xxaa_system_nrf52.c.o
 .debug_ranges  0x000000000000a690      0x278 _build/nrf52832_xxaa_softdevice_handler.c.o

.debug_macro    0x0000000000000000    0x1dd1b
 .debug_macro   0x0000000000000000      0x5d5 _build/nrf52832_xxaa_main.c.o
 .debug_macro   0x00000000000005d5      0xafc _build/nrf52832_xxaa_main.c.o
 .debug_macro   0x00000000000010d1       0x22 _build/nrf52832_xxaa_main.c.o
 .debug_macro   0x00000000000010f3       0x22 _build/nrf52832_xxaa_main.c.o
 .debug_macro   0x0000000000001115       0x56 _build/nrf52832_xxaa_main.c.o
 .debug_macro   0x000000000000116b       0x51 _build/nrf52832_xxaa_main.c.o
 .debug_macro   0x00000000000011bc      0x103 _build/nrf52832_xxaa_main.c.o
 .debug_macro   0x00000000000012bf       0x6a _build/nrf52832_xxaa_main.c.o
 .debug_macro   0x0000000000001329      0x1df _build/nrf52832_xxaa_main.c.o
 .debug_macro   0x0000000000001508       0x5e _build/nrf52832_xxaa_main.c.o
 .debug_macro   0x0000000000001566       0x18 _build/nrf52832_xxaa_main.c.o
 .debug_macro   0x000000000000157e       0x35 _build/nrf52832_xxaa_main.c.o
 .debug_macro   0x00000000000015b3       0x34 _build/nrf52832_xxaa_main.c.o
 .debug_macro   0x00000000000015e7      0x16d _build/nrf52832_xxaa_main.c.o
 .debug_macro   0x0000000000001754       0x16 _build/nrf52832_xxaa_main.c.o
 .debug_macro   0x000000000000176a       0x43 _build/nrf52832_xxaa_main.c.o
 .debug_macro   0x00000000000017ad       0x34 _build/nrf52832_xxaa_main.c.o
 .debug_macro   0x00000000000017e1       0x10 _build/nrf52832_xxaa_main.c.o
 .debug_macro   0x00000000000017f1       0x58 _build/nrf52832_xxaa_main.c.o
 .debug_macro   0x0000000000001849      0x182 _build/nrf52832_xxaa_main.c.o
 .debug_macro   0x00000000000019cb      0x35c _build/nrf52832_xxaa_main.c.o
 .debug_macro   0x0000000000001d27       0x10 _build/nrf52832_xxaa_main.c.o
 .debug_macro   0x0000000000001d37       0x35 _build/nrf52832_xxaa_main.c.o
 .debug_macro   0x0000000000001d6c      0x3ab _build/nrf52832_xxaa_main.c.o
 .debug_macro   0x0000000000002117      0x16d _build/nrf52832_xxaa_main.c.o
 .debug_macro   0x0000000000002284       0x2e _build/nrf52832_xxaa_main.c.o
 .debug_macro   0x00000000000022b2       0x22 _build/nrf52832_xxaa_main.c.o
 .debug_macro   0x00000000000022d4       0x9a _build/nrf52832_xxaa_main.c.o
 .debug_macro   0x000000000000236e       0x78 _build/nrf52832_xxaa_main.c.o
 .debug_macro   0x00000000000023e6       0x22 _build/nrf52832_xxaa_main.c.o
 .debug_macro   0x0000000000002408       0x2d _build/nrf52832_xxaa_main.c.o
 .debug_macro   0x0000000000002435       0x3b _build/nrf52832_xxaa_main.c.o
 .debug_macro   0x0000000000002470       0x50 _build/nrf52832_xxaa_main.c.o
 .debug_macro   0x00000000000024c0      0xe66 _build/nrf52832_xxaa_main.c.o
 .debug_macro   0x0000000000003326      0x392 _build/nrf52832_xxaa_main.c.o
 .debug_macro   0x00000000000036b8     0xcc8d _build/nrf52832_xxaa_main.c.o
 .debug_macro   0x0000000000010345     0x1313 _build/nrf52832_xxaa_main.c.o
 .debug_macro   0x0000000000011658       0x82 _build/nrf52832_xxaa_main.c.o
 .debug_macro   0x00000000000116da      0x491 _build/nrf52832_xxaa_main.c.o
 .debug_macro   0x0000000000011b6b       0x4b _build/nrf52832_xxaa_main.c.o
 .debug_macro   0x0000000000011bb6       0x1c _build/nrf52832_xxaa_main.c.o
 .debug_macro   0x0000000000011bd2      0x164 _build/nrf52832_xxaa_main.c.o
 .debug_macro   0x0000000000011d36       0x5e _build/nrf52832_xxaa_main.c.o
 .debug_macro   0x0000000000011d94       0x16 _build/nrf52832_xxaa_main.c.o
 .debug_macro   0x0000000000011daa       0x40 _build/nrf52832_xxaa_main.c.o
 .debug_macro   0x0000000000011dea       0x64 _build/nrf52832_xxaa_main.c.o
 .debug_macro   0x0000000000011e4e       0x2e _build/nrf52832_xxaa_main.c.o
 .debug_macro   0x0000000000011e7c       0x1c _build/nrf52832_xxaa_main.c.o
 .debug_macro   0x0000000000011e98       0x10 _build/nrf52832_xxaa_main.c.o
 .debug_macro   0x0000000000011ea8       0xbe _build/nrf52832_xxaa_main.c.o
 .debug_macro   0x0000000000011f66       0x16 _build/nrf52832_xxaa_main.c.o
 .debug_macro   0x0000000000011f7c      0x129 _build/nrf52832_xxaa_main.c.o
 .debug_macro   0x00000000000120a5       0x2b _build/nrf52832_xxaa_main.c.o
 .debug_macro   0x00000000000120d0       0x10 _build/nrf52832_xxaa_main.c.o
 .debug_macro   0x00000000000120e0       0x7f _build/nrf52832_xxaa_main.c.o
 .debug_macro   0x000000000001215f       0x28 _build/nrf52832_xxaa_main.c.o
 .debug_macro   0x0000000000012187       0x22 _build/nrf52832_xxaa_main.c.o
 .debug_macro   0x00000000000121a9      0x139 _build/nrf52832_xxaa_main.c.o
 .debug_macro   0x00000000000122e2      0x1fb _build/nrf52832_xxaa_main.c.o
 .debug_macro   0x00000000000124dd      0x46a _build/nrf52832_xxaa_main.c.o
 .debug_macro   0x0000000000012947       0x3a _build/nrf52832_xxaa_main.c.o
 .debug_macro   0x0000000000012981      0x1f7 _build/nrf52832_xxaa_main.c.o
 .debug_macro   0x0000000000012b78       0x22 _build/nrf52832_xxaa_main.c.o
 .debug_macro   0x0000000000012b9a       0xf1 _build/nrf52832_xxaa_main.c.o
 .debug_macro   0x0000000000012c8b       0x3c _build/nrf52832_xxaa_main.c.o
 .debug_macro   0x0000000000012cc7       0xa6 _build/nrf52832_xxaa_main.c.o
 .debug_macro   0x0000000000012d6d      0x2e9 _build/nrf52832_xxaa_main.c.o
 .debug_macro   0x0000000000013056       0x6a _build/nrf52832_xxaa_main.c.o
 .debug_macro   0x00000000000130c0      0x2a4 _build/nrf52832_xxaa_main.c.o
 .debug_macro   0x0000000000013364       0x16 _build/nrf52832_xxaa_main.c.o
 .debug_macro   0x000000000001337a       0x22 _build/nrf52832_xxaa_main.c.o
 .debug_macro   0x000000000001339c       0x16 _build/nrf52832_xxaa_main.c.o
 .debug_macro   0x00000000000133b2      0x261 _build/nrf52832_xxaa_main.c.o
 .debug_macro   0x0000000000013613      0x115 _build/nrf52832_xxaa_main.c.o
 .debug_macro   0x0000000000013728       0x1c _build/nrf52832_xxaa_main.c.o
 .debug_macro   0x0000000000013744       0xf7 _build/nrf52832_xxaa_main.c.o
 .debug_macro   0x000000000001383b       0x16 _build/nrf52832_xxaa_main.c.o
 .debug_macro   0x0000000000013851       0x10 _build/nrf52832_xxaa_main.c.o
 .debug_macro   0x0000000000013861       0x16 _build/nrf52832_xxaa_main.c.o
 .debug_macro   0x0000000000013877       0x2e _build/nrf52832_xxaa_main.c.o
 .debug_macro   0x00000000000138a5       0x37 _build/nrf52832_xxaa_main.c.o
 .debug_macro   0x00000000000138dc       0x16 _build/nrf52832_xxaa_main.c.o
 .debug_macro   0x00000000000138f2       0x10 _build/nrf52832_xxaa_main.c.o
 .debug_macro   0x0000000000013902       0x82 _build/nrf52832_xxaa_main.c.o
 .debug_macro   0x0000000000013984       0x40 _build/nrf52832_xxaa_main.c.o
 .debug_macro   0x00000000000139c4       0x1c _build/nrf52832_xxaa_main.c.o
 .debug_macro   0x00000000000139e0       0x22 _build/nrf52832_xxaa_main.c.o
 .debug_macro   0x0000000000013a02       0x1c _build/nrf52832_xxaa_main.c.o
 .debug_macro   0x0000000000013a1e       0x1c _build/nrf52832_xxaa_main.c.o
 .debug_macro   0x0000000000013a3a       0x1c _build/nrf52832_xxaa_main.c.o
 .debug_macro   0x0000000000013a56       0x52 _build/nrf52832_xxaa_main.c.o
 .debug_macro   0x0000000000013aa8      0x100 _build/nrf52832_xxaa_main.c.o
 .debug_macro   0x0000000000013ba8       0x82 _build/nrf52832_xxaa_main.c.o
 .debug_macro   0x0000000000013c2a       0x10 _build/nrf52832_xxaa_main.c.o
 .debug_macro   0x0000000000013c3a       0x1c _build/nrf52832_xxaa_main.c.o
 .debug_macro   0x0000000000013c56       0x82 _build/nrf52832_xxaa_main.c.o
 .debug_macro   0x0000000000013cd8       0x1c _build/nrf52832_xxaa_main.c.o
 .debug_macro   0x0000000000013cf4       0x6a _build/nrf52832_xxaa_main.c.o
 .debug_macro   0x0000000000013d5e       0x5e _build/nrf52832_xxaa_main.c.o
 .debug_macro   0x0000000000013dbc       0x3a _build/nrf52832_xxaa_main.c.o
 .debug_macro   0x0000000000013df6       0x46 _build/nrf52832_xxaa_main.c.o
 .debug_macro   0x0000000000013e3c       0x1c _build/nrf52832_xxaa_main.c.o
 .debug_macro   0x0000000000013e58       0x8e _build/nrf52832_xxaa_main.c.o
 .debug_macro   0x0000000000013ee6       0x22 _build/nrf52832_xxaa_main.c.o
 .debug_macro   0x0000000000013f08      0x556 _build/nrf52832_xxaa_ble_init.c.o
 .debug_macro   0x000000000001445e       0x35 _build/nrf52832_xxaa_ble_init.c.o
 .debug_macro   0x0000000000014493       0x22 _build/nrf52832_xxaa_ble_init.c.o
 .debug_macro   0x00000000000144b5       0x16 _build/nrf52832_xxaa_ble_init.c.o
 .debug_macro   0x00000000000144cb       0x97 _build/nrf52832_xxaa_ble_init.c.o
 .debug_macro   0x0000000000014562       0xf6 _build/nrf52832_xxaa_ble_init.c.o
 .debug_macro   0x0000000000014658      0x464 _build/nrf52832_xxaa_ble_init.c.o
 .debug_macro   0x0000000000014abc       0x34 _build/nrf52832_xxaa_ble_init.c.o
 .debug_macro   0x0000000000014af0       0x16 _build/nrf52832_xxaa_ble_init.c.o
 .debug_macro   0x0000000000014b06       0x64 _build/nrf52832_xxaa_ble_init.c.o
 .debug_macro   0x0000000000014b6a       0x46 _build/nrf52832_xxaa_ble_init.c.o
 .debug_macro   0x0000000000014bb0       0x10 _build/nrf52832_xxaa_ble_init.c.o
 .debug_macro   0x0000000000014bc0       0x16 _build/nrf52832_xxaa_ble_init.c.o
 .debug_macro   0x0000000000014bd6      0x3bd _build/nrf52832_xxaa_ble_lcs.c.o
 .debug_macro   0x0000000000014f93       0x1c _build/nrf52832_xxaa_ble_lcs.c.o
 .debug_macro   0x0000000000014faf      0x3d5 _build/nrf52832_xxaa_ble_ics.c.o
 .debug_macro   0x0000000000015384      0x3d5 _build/nrf52832_xxaa_ble_tcs.c.o
 .debug_macro   0x0000000000015759       0x40 _build/nrf52832_xxaa_ble_tcs.c.o
 .debug_macro   0x0000000000015799      0x3bd _build/nrf52832_xxaa_ble_scs.c.o
 .debug_macro   0x0000000000015b56       0x16 _build/nrf52832_xxaa_ble_scs.c.o
 .debug_macro   0x0000000000015b6c      0x290 _build/nrf52832_xxaa_gpio.c.o
 .debug_macro   0x0000000000015dfc       0xfa _build/nrf52832_xxaa_gpio.c.o
 .debug_macro   0x0000000000015ef6       0xdc _build/nrf52832_xxaa_uart.c.o
 .debug_macro   0x0000000000015fd2       0xf4 _build/nrf52832_xxaa_print.c.o
 .debug_macro   0x00000000000160c6       0x58 _build/nrf52832_xxaa_print.c.o
 .debug_macro   0x000000000001611e       0xfd _build/nrf52832_xxaa_spim.c.o
 .debug_macro   0x000000000001621b       0x88 _build/nrf52832_xxaa_spim.c.o
 .debug_macro   0x00000000000162a3       0x64 _build/nrf52832_xxaa_spim.c.o
 .debug_macro   0x0000000000016307      0x115 _build/nrf52832_xxaa_stm_communication.c.o
 .debug_macro   0x000000000001641c       0x22 _build/nrf52832_xxaa_stm_communication.c.o
 .debug_macro   0x000000000001643e      0x206 _build/nrf52832_xxaa_flash.c.o
 .debug_macro   0x0000000000016644       0x88 _build/nrf52832_xxaa_flash.c.o
 .debug_macro   0x00000000000166cc      0x215 _build/nrf52832_xxaa_step_count_db.c.o
 .debug_macro   0x00000000000168e1       0xd7 _build/nrf52832_xxaa_rtc.c.o
 .debug_macro   0x00000000000169b8      0x327 _build/nrf52832_xxaa_nrf_log_backend_serial.c.o
 .debug_macro   0x0000000000016cdf       0xa2 _build/nrf52832_xxaa_nrf_log_backend_serial.c.o
 .debug_macro   0x0000000000016d81       0x3a _build/nrf52832_xxaa_nrf_log_backend_serial.c.o
 .debug_macro   0x0000000000016dbb      0x114 _build/nrf52832_xxaa_nrf_log_backend_serial.c.o
 .debug_macro   0x0000000000016ecf      0x340 _build/nrf52832_xxaa_nrf_log_frontend.c.o
 .debug_macro   0x000000000001720f       0x22 _build/nrf52832_xxaa_nrf_log_frontend.c.o
 .debug_macro   0x0000000000017231      0x16a _build/nrf52832_xxaa_nrf_log_frontend.c.o
 .debug_macro   0x000000000001739b       0x2e _build/nrf52832_xxaa_nrf_log_frontend.c.o
 .debug_macro   0x00000000000173c9      0x2fc _build/nrf52832_xxaa_app_error.c.o
 .debug_macro   0x00000000000176c5      0x497 _build/nrf52832_xxaa_app_error.c.o
 .debug_macro   0x0000000000017b5c       0x16 _build/nrf52832_xxaa_app_error.c.o
 .debug_macro   0x0000000000017b72      0x2f6 _build/nrf52832_xxaa_app_error_weak.c.o
 .debug_macro   0x0000000000017e68      0x331 _build/nrf52832_xxaa_app_timer.c.o
 .debug_macro   0x0000000000018199       0x16 _build/nrf52832_xxaa_app_timer.c.o
 .debug_macro   0x00000000000181af      0x26d _build/nrf52832_xxaa_app_util_platform.c.o
 .debug_macro   0x000000000001841c      0x2ef _build/nrf52832_xxaa_fds.c.o
 .debug_macro   0x000000000001870b       0x9c _build/nrf52832_xxaa_fds.c.o
 .debug_macro   0x00000000000187a7       0x31 _build/nrf52832_xxaa_fds.c.o
 .debug_macro   0x00000000000187d8      0x247 _build/nrf52832_xxaa_fstorage.c.o
 .debug_macro   0x0000000000018a1f       0x4f _build/nrf52832_xxaa_fstorage.c.o
 .debug_macro   0x0000000000018a6e      0x11f _build/nrf52832_xxaa_sdk_mapped_flags.c.o
 .debug_macro   0x0000000000018b8d       0x16 _build/nrf52832_xxaa_sdk_mapped_flags.c.o
 .debug_macro   0x0000000000018ba3      0x42d _build/nrf52832_xxaa_nrf_drv_clock.c.o
 .debug_macro   0x0000000000018fd0       0x10 _build/nrf52832_xxaa_nrf_drv_clock.c.o
 .debug_macro   0x0000000000018fe0       0x28 _build/nrf52832_xxaa_nrf_drv_clock.c.o
 .debug_macro   0x0000000000019008       0x10 _build/nrf52832_xxaa_nrf_drv_clock.c.o
 .debug_macro   0x0000000000019018       0x16 _build/nrf52832_xxaa_nrf_drv_clock.c.o
 .debug_macro   0x000000000001902e      0x2d7 _build/nrf52832_xxaa_nrf_drv_common.c.o
 .debug_macro   0x0000000000019305       0x22 _build/nrf52832_xxaa_nrf_drv_common.c.o
 .debug_macro   0x0000000000019327      0x3c9 _build/nrf52832_xxaa_nrf_drv_gpiote.c.o
 .debug_macro   0x00000000000196f0       0x16 _build/nrf52832_xxaa_nrf_drv_gpiote.c.o
 .debug_macro   0x0000000000019706      0x3b6 _build/nrf52832_xxaa_nrf_drv_uart.c.o
 .debug_macro   0x0000000000019abc       0x10 _build/nrf52832_xxaa_nrf_drv_uart.c.o
 .debug_macro   0x0000000000019acc       0x43 _build/nrf52832_xxaa_nrf_drv_uart.c.o
 .debug_macro   0x0000000000019b0f      0x2b5 _build/nrf52832_xxaa_SEGGER_RTT.c.o
 .debug_macro   0x0000000000019dc4       0x34 _build/nrf52832_xxaa_SEGGER_RTT.c.o
 .debug_macro   0x0000000000019df8      0x2a0 _build/nrf52832_xxaa_ble_advdata.c.o
 .debug_macro   0x000000000001a098      0x2ee _build/nrf52832_xxaa_ble_advertising.c.o
 .debug_macro   0x000000000001a386      0x307 _build/nrf52832_xxaa_ble_conn_params.c.o
 .debug_macro   0x000000000001a68d      0x10e _build/nrf52832_xxaa_ble_conn_params.c.o
 .debug_macro   0x000000000001a79b       0x86 _build/nrf52832_xxaa_ble_conn_params.c.o
 .debug_macro   0x000000000001a821      0x2e3 _build/nrf52832_xxaa_ble_conn_state.c.o
 .debug_macro   0x000000000001ab04      0x2d1 _build/nrf52832_xxaa_ble_srv_common.c.o
 .debug_macro   0x000000000001add5      0x399 _build/nrf52832_xxaa_gatt_cache_manager.c.o
 .debug_macro   0x000000000001b16e      0x387 _build/nrf52832_xxaa_gatts_cache_manager.c.o
 .debug_macro   0x000000000001b4f5       0x10 _build/nrf52832_xxaa_gatts_cache_manager.c.o
 .debug_macro   0x000000000001b505      0x3ac _build/nrf52832_xxaa_id_manager.c.o
 .debug_macro   0x000000000001b8b1       0x40 _build/nrf52832_xxaa_id_manager.c.o
 .debug_macro   0x000000000001b8f1      0x33d _build/nrf52832_xxaa_nrf_ble_gatt.c.o
 .debug_macro   0x000000000001bc2e       0x16 _build/nrf52832_xxaa_nrf_ble_gatt.c.o
 .debug_macro   0x000000000001bc44      0x386 _build/nrf52832_xxaa_peer_data_storage.c.o
 .debug_macro   0x000000000001bfca       0x3a _build/nrf52832_xxaa_peer_data_storage.c.o
 .debug_macro   0x000000000001c004      0x3a1 _build/nrf52832_xxaa_peer_database.c.o
 .debug_macro   0x000000000001c3a5       0x3a _build/nrf52832_xxaa_peer_database.c.o
 .debug_macro   0x000000000001c3df       0x10 _build/nrf52832_xxaa_peer_database.c.o
 .debug_macro   0x000000000001c3ef       0x10 _build/nrf52832_xxaa_peer_database.c.o
 .debug_macro   0x000000000001c3ff      0x35c _build/nrf52832_xxaa_peer_id.c.o
 .debug_macro   0x000000000001c75b      0x3d2 _build/nrf52832_xxaa_peer_manager.c.o
 .debug_macro   0x000000000001cb2d      0x211 _build/nrf52832_xxaa_pm_buffer.c.o
 .debug_macro   0x000000000001cd3e      0x2b8 _build/nrf52832_xxaa_pm_mutex.c.o
 .debug_macro   0x000000000001cff6      0x395 _build/nrf52832_xxaa_security_dispatcher.c.o
 .debug_macro   0x000000000001d38b      0x39f _build/nrf52832_xxaa_security_manager.c.o
 .debug_macro   0x000000000001d72a       0xf5 _build/nrf52832_xxaa_system_nrf52.c.o
 .debug_macro   0x000000000001d81f      0x3e1 _build/nrf52832_xxaa_softdevice_handler.c.o
 .debug_macro   0x000000000001dc00       0x58 _build/nrf52832_xxaa_softdevice_handler.c.o
 .debug_macro   0x000000000001dc58       0x5c _build/nrf52832_xxaa_softdevice_handler.c.o
 .debug_macro   0x000000000001dcb4       0x57 _build/nrf52832_xxaa_softdevice_handler.c.o
 .debug_macro   0x000000000001dd0b       0x10 _build/nrf52832_xxaa_softdevice_handler.c.o

.debug_line     0x0000000000000000    0x2b5c9
 .debug_line    0x0000000000000000      0xcd9 _build/nrf52832_xxaa_main.c.o
 .debug_line    0x0000000000000cd9     0x1308 _build/nrf52832_xxaa_ble_init.c.o
 .debug_line    0x0000000000001fe1      0xa37 _build/nrf52832_xxaa_ble_lcs.c.o
 .debug_line    0x0000000000002a18      0xa87 _build/nrf52832_xxaa_ble_ics.c.o
 .debug_line    0x000000000000349f     0x16e2 _build/nrf52832_xxaa_ble_tcs.c.o
 .debug_line    0x0000000000004b81      0xa31 _build/nrf52832_xxaa_ble_scs.c.o
 .debug_line    0x00000000000055b2      0x505 _build/nrf52832_xxaa_gpio.c.o
 .debug_line    0x0000000000005ab7      0x372 _build/nrf52832_xxaa_uart.c.o
 .debug_line    0x0000000000005e29      0xd3a _build/nrf52832_xxaa_print.c.o
 .debug_line    0x0000000000006b63      0x5c6 _build/nrf52832_xxaa_spim.c.o
 .debug_line    0x0000000000007129      0x478 _build/nrf52832_xxaa_stm_communication.c.o
 .debug_line    0x00000000000075a1      0x635 _build/nrf52832_xxaa_flash.c.o
 .debug_line    0x0000000000007bd6      0x65f _build/nrf52832_xxaa_step_count_db.c.o
 .debug_line    0x0000000000008235      0x327 _build/nrf52832_xxaa_rtc.c.o
 .debug_line    0x000000000000855c      0xafc _build/nrf52832_xxaa_nrf_log_backend_serial.c.o
 .debug_line    0x0000000000009058     0x1384 _build/nrf52832_xxaa_nrf_log_frontend.c.o
 .debug_line    0x000000000000a3dc      0x6bf _build/nrf52832_xxaa_app_error.c.o
 .debug_line    0x000000000000aa9b      0x659 _build/nrf52832_xxaa_app_error_weak.c.o
 .debug_line    0x000000000000b0f4     0x143d _build/nrf52832_xxaa_app_timer.c.o
 .debug_line    0x000000000000c531      0x74a _build/nrf52832_xxaa_app_util_platform.c.o
 .debug_line    0x000000000000cc7b     0x324a _build/nrf52832_xxaa_fds.c.o
 .debug_line    0x000000000000fec5      0xe5c _build/nrf52832_xxaa_fstorage.c.o
 .debug_line    0x0000000000010d21      0x62e _build/nrf52832_xxaa_sdk_mapped_flags.c.o
 .debug_line    0x000000000001134f     0x134e _build/nrf52832_xxaa_nrf_drv_clock.c.o
 .debug_line    0x000000000001269d      0x603 _build/nrf52832_xxaa_nrf_drv_common.c.o
 .debug_line    0x0000000000012ca0     0x28cf _build/nrf52832_xxaa_nrf_drv_gpiote.c.o
 .debug_line    0x000000000001556f     0x269c _build/nrf52832_xxaa_nrf_drv_uart.c.o
 .debug_line    0x0000000000017c0b     0x24bb _build/nrf52832_xxaa_SEGGER_RTT.c.o
 .debug_line    0x000000000001a0c6      0xd65 _build/nrf52832_xxaa_ble_advdata.c.o
 .debug_line    0x000000000001ae2b      0xfb8 _build/nrf52832_xxaa_ble_advertising.c.o
 .debug_line    0x000000000001bde3      0x9c9 _build/nrf52832_xxaa_ble_conn_params.c.o
 .debug_line    0x000000000001c7ac      0x912 _build/nrf52832_xxaa_ble_conn_state.c.o
 .debug_line    0x000000000001d0be      0xa2e _build/nrf52832_xxaa_ble_srv_common.c.o
 .debug_line    0x000000000001daec      0xe1e _build/nrf52832_xxaa_gatt_cache_manager.c.o
 .debug_line    0x000000000001e90a      0xa70 _build/nrf52832_xxaa_gatts_cache_manager.c.o
 .debug_line    0x000000000001f37a     0x1b46 _build/nrf52832_xxaa_id_manager.c.o
 .debug_line    0x0000000000020ec0      0xb95 _build/nrf52832_xxaa_nrf_ble_gatt.c.o
 .debug_line    0x0000000000021a55      0xf75 _build/nrf52832_xxaa_peer_data_storage.c.o
 .debug_line    0x00000000000229ca     0x206e _build/nrf52832_xxaa_peer_database.c.o
 .debug_line    0x0000000000024a38      0x8f9 _build/nrf52832_xxaa_peer_id.c.o
 .debug_line    0x0000000000025331     0x1b97 _build/nrf52832_xxaa_peer_manager.c.o
 .debug_line    0x0000000000026ec8      0x5ed _build/nrf52832_xxaa_pm_buffer.c.o
 .debug_line    0x00000000000274b5      0x6f8 _build/nrf52832_xxaa_pm_mutex.c.o
 .debug_line    0x0000000000027bad     0x13bf _build/nrf52832_xxaa_security_dispatcher.c.o
 .debug_line    0x0000000000028f6c      0xfa8 _build/nrf52832_xxaa_security_manager.c.o
 .debug_line    0x0000000000029f14      0x7d1 _build/nrf52832_xxaa_system_nrf52.c.o
 .debug_line    0x000000000002a6e5      0xee4 _build/nrf52832_xxaa_softdevice_handler.c.o

.debug_str      0x0000000000000000    0x82997
 .debug_str     0x0000000000000000    0x71bcc _build/nrf52832_xxaa_main.c.o
                                      0x728bf (size before relaxing)
 .debug_str     0x0000000000071bcc     0x3330 _build/nrf52832_xxaa_ble_init.c.o
                                      0x73f2f (size before relaxing)
 .debug_str     0x0000000000074efc      0x2d6 _build/nrf52832_xxaa_ble_lcs.c.o
                                      0x6e5d8 (size before relaxing)
 .debug_str     0x00000000000751d2       0xfb _build/nrf52832_xxaa_ble_ics.c.o
                                      0x6ec1b (size before relaxing)
 .debug_str     0x00000000000752cd      0x17b _build/nrf52832_xxaa_ble_tcs.c.o
                                      0x6ecb6 (size before relaxing)
 .debug_str     0x0000000000075448       0x82 _build/nrf52832_xxaa_ble_scs.c.o
                                      0x6e6a8 (size before relaxing)
 .debug_str     0x00000000000754ca       0x85 _build/nrf52832_xxaa_gpio.c.o
                                      0x62081 (size before relaxing)
 .debug_str     0x000000000007554f      0x18b _build/nrf52832_xxaa_uart.c.o
                                      0x5440e (size before relaxing)
 .debug_str     0x00000000000756da       0xa8 _build/nrf52832_xxaa_print.c.o
                                      0x544a9 (size before relaxing)
 .debug_str     0x0000000000075782      0x216 _build/nrf52832_xxaa_spim.c.o
                                      0x54a63 (size before relaxing)
 .debug_str     0x0000000000075998       0x82 _build/nrf52832_xxaa_stm_communication.c.o
                                      0x54bb9 (size before relaxing)
 .debug_str     0x0000000000075a1a      0x1d8 _build/nrf52832_xxaa_flash.c.o
                                      0x6783f (size before relaxing)
 .debug_str     0x0000000000075bf2       0x80 _build/nrf52832_xxaa_step_count_db.c.o
                                      0x673de (size before relaxing)
 .debug_str     0x0000000000075c72      0x31e _build/nrf52832_xxaa_rtc.c.o
                                      0x53f67 (size before relaxing)
 .debug_str     0x0000000000075f90      0xfd1 _build/nrf52832_xxaa_nrf_log_backend_serial.c.o
                                      0x6775d (size before relaxing)
 .debug_str     0x0000000000076f61      0x677 _build/nrf52832_xxaa_nrf_log_frontend.c.o
                                      0x68498 (size before relaxing)
 .debug_str     0x00000000000775d8       0xd6 _build/nrf52832_xxaa_app_error.c.o
                                      0x67ddb (size before relaxing)
 .debug_str     0x00000000000776ae       0x78 _build/nrf52832_xxaa_app_error_weak.c.o
                                      0x67dcf (size before relaxing)
 .debug_str     0x0000000000077726      0x7f3 _build/nrf52832_xxaa_app_timer.c.o
                                      0x6720d (size before relaxing)
 .debug_str     0x0000000000077f19      0x245 _build/nrf52832_xxaa_app_util_platform.c.o
                                      0x623d9 (size before relaxing)
 .debug_str     0x000000000007815e     0x11bc _build/nrf52832_xxaa_fds.c.o
                                      0x67af4 (size before relaxing)
 .debug_str     0x000000000007931a      0x527 _build/nrf52832_xxaa_fstorage.c.o
                                      0x664b4 (size before relaxing)
 .debug_str     0x0000000000079841      0x1b5 _build/nrf52832_xxaa_sdk_mapped_flags.c.o
                                      0x60b4a (size before relaxing)
 .debug_str     0x00000000000799f6      0xb8f _build/nrf52832_xxaa_nrf_drv_clock.c.o
                                      0x6dce2 (size before relaxing)
 .debug_str     0x000000000007a585       0x53 _build/nrf52832_xxaa_nrf_drv_common.c.o
                                      0x66ebe (size before relaxing)
 .debug_str     0x000000000007a5d8     0x18d3 _build/nrf52832_xxaa_nrf_drv_gpiote.c.o
                                      0x6a215 (size before relaxing)
 .debug_str     0x000000000007beab     0x16ca _build/nrf52832_xxaa_nrf_drv_uart.c.o
                                      0x6a51c (size before relaxing)
 .debug_str     0x000000000007d575      0x323 _build/nrf52832_xxaa_SEGGER_RTT.c.o
                                      0x62936 (size before relaxing)
 .debug_str     0x000000000007d898      0x363 _build/nrf52832_xxaa_ble_advdata.c.o
                                      0x6b02d (size before relaxing)
 .debug_str     0x000000000007dbfb      0x46c _build/nrf52832_xxaa_ble_advertising.c.o
                                      0x6d15c (size before relaxing)
 .debug_str     0x000000000007e067      0x190 _build/nrf52832_xxaa_ble_conn_params.c.o
                                      0x6c5c1 (size before relaxing)
 .debug_str     0x000000000007e1f7      0x6d7 _build/nrf52832_xxaa_ble_conn_state.c.o
                                      0x6ae32 (size before relaxing)
 .debug_str     0x000000000007e8ce      0x2d5 _build/nrf52832_xxaa_ble_srv_common.c.o
                                      0x6aefd (size before relaxing)
 .debug_str     0x000000000007eba3      0xaa2 _build/nrf52832_xxaa_gatt_cache_manager.c.o
                                      0x6cc25 (size before relaxing)
 .debug_str     0x000000000007f645      0x5ba _build/nrf52832_xxaa_gatts_cache_manager.c.o
                                      0x6bb1d (size before relaxing)
 .debug_str     0x000000000007fbff      0x818 _build/nrf52832_xxaa_id_manager.c.o
                                      0x6d71d (size before relaxing)
 .debug_str     0x0000000000080417      0x433 _build/nrf52832_xxaa_nrf_ble_gatt.c.o
                                      0x6de2e (size before relaxing)
 .debug_str     0x000000000008084a      0x555 _build/nrf52832_xxaa_peer_data_storage.c.o
                                      0x6bf2a (size before relaxing)
 .debug_str     0x0000000000080d9f      0x64a _build/nrf52832_xxaa_peer_database.c.o
                                      0x6bfd3 (size before relaxing)
 .debug_str     0x00000000000813e9      0x120 _build/nrf52832_xxaa_peer_id.c.o
                                      0x6ade6 (size before relaxing)
 .debug_str     0x0000000000081509      0x67b _build/nrf52832_xxaa_peer_manager.c.o
                                      0x6daed (size before relaxing)
 .debug_str     0x0000000000081b84       0xe6 _build/nrf52832_xxaa_pm_buffer.c.o
                                      0x65186 (size before relaxing)
 .debug_str     0x0000000000081c6a       0x67 _build/nrf52832_xxaa_pm_mutex.c.o
                                      0x6645a (size before relaxing)
 .debug_str     0x0000000000081cd1      0x445 _build/nrf52832_xxaa_security_dispatcher.c.o
                                      0x6d3d2 (size before relaxing)
 .debug_str     0x0000000000082116      0x2a8 _build/nrf52832_xxaa_security_manager.c.o
                                      0x6cc48 (size before relaxing)
 .debug_str     0x00000000000823be      0x13c _build/nrf52832_xxaa_system_nrf52.c.o
                                      0x5c3f8 (size before relaxing)
 .debug_str     0x00000000000824fa      0x49d _build/nrf52832_xxaa_softdevice_handler.c.o
                                      0x6e1f1 (size before relaxing)
